:020000040800F2
:100000006097012405040008D9480108510C010833
:10001000D148010849410008598C0108000000003E
:10002000000000000000000000000000614F010817
:100030004164000800000000214B010881580108BC
:1000400023040008230400082304000823040008F4
:1000500023040008230400082304000823040008E4
:10006000230400082304000823040008F15C0008AE
:10007000015D0008115D0008215D0008315D000888
:10008000415D00082304000823040008A16400085F
:10009000C1640008B1640008D164000823040008AA
:1000A0002304000823040008230400082304000894
:1000B0002304000823040008230400082304000884
:1000C0002304000823040008230400082304000874
:1000D000D94D0108198601083986010849860108A9
:1000E00049640008230400080000000023040008FD
:1000F0002304000823040008230400082304000844
:100100002304000823040008230400082304000833
:1001100023040008016501082304000823040008E3
:100120002304000823040008230400082304000813
:100130002304000823040008230400082304000803
:1001400000000000000000000000000000000000AF
:1001500023040008230400082304000823040008E3
:1001600023040008230400082304000823040008D3
:1001700023040008230400082304000800000000F2
:100180002304000823040008216501082304000853
:1001900023040008230400082304000823040008A3
:1001A00023040008230400082304000800000000C2
:1001B0002304000823040008230400082304000883
:1001C00023040008230400080000000000000000D1
:1001D00000000000000000002304000800000000F0
:1001E000000000000000000000000000000000000F
:1001F00000000000000000002304000823040008A1
:100200002304000823040008000000002304000861
:100210002304000823040008230400082304000822
:100220002304000800000000230400080000000070
:10023000230400082304000800000000611A0008DD
:10024000230400087925000823040008230400087B
:1002500023040008230400082304000823040008E2
:1002600023040008230400082304000823040008D2
:1002700023040008230400082304000800000000F1
:1002800023040008230400082304000823040008B2
:100290000000000023040008230400080000000000
:1002A00000000000230400082304000823040008C1
:1002B000098601082304000823040008E1640008FB
:1002C000F1640008615A01082304000800F002F8F4
:1002D00000F088F80AA090E8000C82448344AAF158
:1002E0000107DA4501D100F07DF8AFF2090EBAE856
:1002F0000F0013F0010F18BFFB1A43F0010318475A
:1003000038020200580202000A444FF0000C10F8B4
:10031000013B13F0070408BF10F8014B1D1108BF83
:1003200010F8015B641E05D010F8016B641E01F823
:10033000016BF9D113F0080F1EBF10F8014BAD1C73
:100340000C1B09D16D1E58BF01F801CBFAD505E091
:1003500014F8016B01F8016B6D1EF9D59142D6D3EB
:10036000704700000023002400250026103A28BF13
:1003700078C1FBD8520728BF30C148BF0B60704717
:10038000692900F09F81642900F09C81752900F0A3
:1003900099816F2900F03082782900F05782036834
:1003A000DB0928BF41F08001632900F090877329A1
:1003B00000F09587E32900F0A087002070471FB563
:1003C0001FF0ACF99DE8030000F090FE01F070F81A
:1003D0000400002000211FF065F8401C60601FBD74
:1003E00010B510BD01F0BBFA1146FFF7E8FF19F098
:1003F000F3FF01F0D9FA03B4FFF7F2FF03BC01F0F9
:1004000009FB00000A4880470A4880470A4800471D
:10041000FEE7FEE7FEE7FEE7FEE7FEE7FEE7FEE7B4
:10042000FEE7FEE705480649064A074B704700000D
:100430007164000889590108CD0200086067012431
:1004400060970124607701246077012470B5064627
:1004500000F02CFE056806F10B0020F00704B44202
:100460009CBF002070BD2B466A68BAB11068A042DC
:1004700010D304F1080188423CBF5068586007D38C
:100480005168101941601168091B016058601460BF
:10049000101D70BD13465268002AE7D12146284638
:1004A00000F010FE0028DED170BD53EA020C00F00F
:1004B00069802DE9F04B4FF00006002B1FBFB3FA07
:1004C00083F503FA05F424FA05F65E4012BF1643DD
:1004D000B2FA82F502FA05F4C5F120051EBF22FA30
:1004E00005FC44EA0C04203556EA044C4FEA144457
:1004F00018BF641C4FF000084FF00009904271EBE8
:10050000030C39D3002919BFB1FA81F701FA07F6B4
:10051000B0FA80F700FA07F6C7F120071EBF20FAED
:1005200007FC46EA0C062037B6FBF4FCA7EB0507F0
:10053000103F07F01F0BCBF120062CFA06F60CFA41
:100540000BFB44BFB3460026202FA4BF5E464FF0EE
:10055000000B5BEA060C08BF4FF0010B19EB0B090F
:1005600048EB0608ABFB027C06FB02CC0BFB03CC82
:10057000C01B71EB0C01C1E70B46024641464846E1
:10058000BDE8F08B13B5084318BF4FF0FF300146AC
:10059000AFF30080BDE81C40704700000FB41CB5ED
:1005A000084B06AA7B4469460090059800F065FE5A
:1005B00004460020694600F073FE20461CBC5DF82E
:1005C00014FB0000F90C00000FB47CB50C0009AA64
:1005D000009001D02044401E084B7B4469460190A6
:1005E000089800F04AFE05461CB10020694600F05C
:1005F00057FE28467CBC5DF814FB0000CD0C0000C3
:1006000070B5044685690068C10601D5302600E052
:100610002026C00707D070BDD4E90121304690479D
:10062000206A401C20626D1EF6D570BD70B5044670
:1006300085690078C00707D170BDD4E90121202069
:100640009047206A401C20626D1EF6D570BD096877
:100650004A0501D540B27047C905FCD500B27047C4
:1006600009684A0501D5C0B27047C905FCD580B2FA
:10067000704770B50C460546012A05D028788006DB
:1006800000D5EA69002302E0012305E05B1C9342E8
:1006900002D2E05C0028F9D1A869E618C01AA86166
:1006A000286A184428622846FFF7AAFF04E0D5E923
:1006B000012114F8010B9047B442F8D32846FFF704
:1006C000B5FF70BD2DE9F04106460024106875297C
:1006D000314616A510D0FFF7BAFF002802DA4042D3
:1006E00013A507E031688A0701D512A502E0490782
:1006F00004D511A5012401E0FFF7B2FF00210A2271
:1007000006F1240709E0B0FBF2FCB0FBF2F302FBB8
:100710001C00303078541846491C0028F3D1234679
:100720002A463046BDE8F04100F048BD0000000018
:100730002D0000002B000000200000002DE9FF5FCD
:1007400015468A460446DFF8AC80F8440027D8E90D
:1007500000103E46CDE9001010E03AF816106A4647
:1007600002A800F053FE411C07D02178890603D56A
:10077000E269391891420DD80744761C207880062A
:1007800002D5E069B84205DDAE42E6DB3AF8160074
:100790000028E2D1A069C01BA0612046FFF730FF0E
:1007A000D8E90010CDE90010002017E03AF8181041
:1007B0006A4602A800F02AFEB0F1FF3F81460BD046
:1007C00000250DF1080B05E0D4E901211BF8050017
:1007D00090476D1C4D45F7D308F10100B0428046AB
:1007E000E4DB206A384420622046FFF71FFFBDE8A3
:1007F000FF9F0000EAEF010070B504462146106833
:10080000FFF72EFF002104F1240505E000F00702A8
:100810003032C0086A54491C0028F7D120680023F0
:1008200008A2050708D500F02000084304D0E069BD
:10083000012305A2401EE0612046BDE8704000F0A3
:10084000BDBC0000000000003000000070B5044690
:100850000D4621461068FFF703FF2188090502D5E0
:100860000F4A7A4402E00E4A7A440E32002104F123
:10087000240305E000F00F060009965D5E54491C54
:100880000028F7D120780023000704D5702D02D06E
:1008900009B1022311322046BDE8704000F08EBC41
:1008A000DAEE01002DE9F05F894604464FF0000AB8
:1008B000DFF874B1FB44C0F820A02046E168884707
:1008C000002874D0252806D0D4E901219047206A59
:1008D000401C2062F1E700265F462046E168884719
:1008E0002028054607DB312D05D2781910F8200C99
:1008F00008B10643F1E7B00701D526F00406C4F8B5
:100900001CA00027C4F818A02A2D09D028461EF0E4
:100910008FFD38B304EB8708303DC8F8185019E054
:1009200059F8041B204604EB87029161E16888476F
:10093000012F054618D1E069002820DA26F02006AC
:100940001DE0D8F8180000EB800005EB40003038BF
:10095000C8F818002046E168884705461EF068FD83
:100960000028EED1012F0AD02E2D08D12046E168B3
:1009700088477F1C0546022F46F02006C4DBA0698D
:10098000002803DA404246F00106A061F00701D0DA
:1009900026F010066C2D0BD0682D09D04C2D39D0C7
:1009A0006A2D35D0742D35D07A2D33D016E038E04D
:1009B000E1682F4620468847B842054609D16C2F8A
:1009C00026D04FF48060E1680643204688470546FC
:1009D00004E06C2F1AD04FF4807006430DB3A5F1DC
:1009E0004100192802D8203546F400664A462946B7
:1009F000204626604E46FFF7C3FC80B101280BD08D
:100A0000F61D26F0070000F1080956E74020E4E74C
:100A10008020D8E70020D6E706F104094DE72846F4
:100A200052E7206ABDE8F09FB0EE01000FB400B5B8
:100A30008DB010A9099000910B904FF0FF300A90F3
:100A400000200C90064878440690064878446A4690
:100A500007900F9909A800F071FC0DB05DF814FB28
:100A6000130900002B0900002DE9FF5F1D464FF020
:100A7000FF3B91464FF000085F46D5E90146A96962
:100A800001987F1C8847296A824688470028F6D14A
:100A9000BAF1FF3F0CD0002E24F4C06419DD6006CB
:100AA00014D5BAF12B0F09D0BAF12D0F0ED103E0F6
:100AB000584604B0BDE8F09F44F48064A9690198E9
:100AC0007F1C8847761E8246002E02DDBAF1300F69
:100AD00003D0B9F1000F26D032E0A969761E019843
:100AE0007F1C44F400748847002E824605DDBAF16D
:100AF000780F06D0BAF1580F03D0B9F1000F10D01B
:100B00001EE0B9F1000F02D0B9F1100F18D1A96998
:100B1000761E01987F1C24F40074884782461020BA
:100B200002E0082000E00A20814609E0A96908FBEC
:100B30000908761E01987F1C44F400748847824699
:100B4000002E05DD4946504600F0E3FB0028EDDAB3
:100B5000E96901988847A00502D46FF00100A8E771
:100B6000E00725D1600613D5600502D5C8F1000065
:100B700000E0404629680A1D2A600968220501D55F
:100B8000087015E0220701D5088011E008600FE029
:100B90002868011D29600068210502D580F80080C1
:100BA00006E0210702D5A0F8008001E0C0F800802F
:100BB00038467EE72DE9FF5F4FF00008994614465E
:100BC00046469169D2E901A7DDF838B00198884717
:100BD000054659EA0B0005D009E0A1690198761C89
:100BE00088470546216A284688470028F5D1681CB1
:100BF00003D05FEACA7005D015E04FF0FF3004B0B3
:100C0000BDE8F09F2068011D2160D0F800800AE057
:100C10005FEACA7001D108F8015BA169761C0198EE
:100C20007F1E88470546002F1ADD681C18D0B9F1D1
:100C3000000F0DD0E81705EBD060421120F01F0027
:100C400059F822102A1A012090400142E0D107E011
:100C5000BBF1000FDCD12846216A88470028D7D095
:100C6000E16901988847BBF1000F07D1002E05DD2F
:100C70005FEACA7002D1002188F80010A068B8426B
:100C800003DDBBF1000F03D017B16FF00100B6E731
:100C90003046B4E770B5064600F00CFA0468054625
:100CA00030460A22002100F079FB2C6070BD000064
:100CB000014A00F0CFBB00000000002440EA01031D
:100CC00010B59B070FD1042A0DD310C808C9121FF5
:100CD0009C42F8D020BA19BA884201D9012010BD2F
:100CE0004FF0FF3010BD1AB1D30703D0521C07E0FC
:100CF000002010BD10F8013B11F8014B1B1B07D160
:100D000010F8013B11F8014B1B1B01D1921EF1D1D0
:100D1000184610BD40EA0103024630B59B0710D1CA
:100D20004FF0013400E008C208C91D1B9D4315EABD
:100D3000C41FF8D013F0FF0102F8011B0DD01B0AED
:100D4000F8E711F8013B002B02F8013B05D011F840
:100D5000013B002B02F8013BF3D130BD10B5431C21
:100D600002E010F8011B71B18107FAD14FF0013296
:100D700002C88C1A8C4314EAC211F9D0C01A0A06B0
:100D800003D0C01E10BDC01A10BD0A0401D0801EC1
:100D900010BD0902FCD0401E10BD40EA010370B531
:100DA0009B072ED14FF00136042A2AD308C810C958
:100DB0009D1B9D43121F15EAC61517D0D8B2E1B28C
:100DC000401A50EA056110D198B2A1B2401A50EA17
:100DD00005410AD123F07F4024F07F41401A50EAB8
:100DE000052102D1180EA0EB146070BDA342DBD028
:100DF00018BA21BA884201D9012070BD4FF0FF30E6
:100E000070BD0AB9002070BD10F8013B11F8014B0C
:100E100063B1A3420AD1521E08D010F8013B11F869
:100E2000014B1BB1A34201D1521EEDD1181B70BD65
:100E3000032A40F2308010F0030C00F0158011F806
:100E4000013BBCF1020F624498BF11F801CB00F8DE
:100E5000013B38BF11F8013BA2F1040298BF00F832
:100E600001CB38BF00F8013B11F0030300F02580EF
:100E7000083AC0F0088051F8043B083A51F804CB16
:100E8000A0E80810F5E7121D5CBF51F8043B40F8DC
:100E9000043BAFF30080D20724BF11F8013B11F8E7
:100EA00001CB48BF11F8012B24BF00F8013B00F82B
:100EB00001CB48BF00F8012B704710B5203AC0F0B5
:100EC0000B80B1E81850A0E81850B1E81850A0E81D
:100ED0001850203ABFF4F5AF5FEA027C24BFB1E8B6
:100EE0001850A0E8185044BF18C918C0BDE81040F9
:100EF0005FEA827C24BF51F8043B40F8043B08BF02
:100F00007047D20728BF31F8023B48BF11F8012BC8
:100F100028BF20F8023B48BF00F8012B704702F0C1
:100F2000FF0343EA032242EA024200F00AB802F059
:100F3000FF0343EA032242EA024200F024B84FF0E2
:100F400000020429C0F0128010F0030C00F01B8096
:100F5000CCF1040CBCF1020F18BF00F8012BA8BFA4
:100F600020F8022BA1EB0C0100F00DB85FEAC17C68
:100F700024BF00F8012B00F8012B48BF00F8012B1B
:100F800070474FF0000200B513469446964620394C
:100F900022BFA0E80C50A0E80C50B1F12001BFF432
:100FA000F7AF090728BFA0E80C5048BF0CC05DF898
:100FB00004EB890028BF40F8042B08BF704748BFE6
:100FC00020F8022B11F0804F18BF00F8012B70475A
:100FD00010B5044610F0030F08BF11F0030F40F0E6
:100FE00015804FF0013E121FC0F20E8051F8043BF5
:100FF000A3EB0E0C2CEA030C1CEACE1C08BF40F835
:10100000043BF0D0A1F1040102F10402521E08DBFE
:1010100011F8013B00F8013B002BF7D11146FFF717
:101020008EFF204610BD000030B44FF0013C50F858
:10103000042BCCFA52F451F8043BD51A20D1FCB958
:1010400050F8042BCCFA52F451F8043BD51A17D1BE
:10105000B4B950F8042BCCFA52F451F8043BD51A29
:101060000ED16CB950F8042BCCFA52F451F8043B71
:10107000D51A05D1002CDAD030BC4FF000007047F3
:1010800029BAB1FA81F111F01801D1F120008440A0
:10109000F2D1CA40CB4012F0FF0213F0FF0330BC84
:1010A000D01A70477047704770470000004870477B
:1010B000E810002400487047E01000247047704793
:1010C0007047704738B504460A4600206946AFF3BA
:1010D0000080002808BF38BD02460099204600F075
:1010E000EBF9012038BD012000F013BCF8B5AFF3D7
:1010F0000080054600200C46102000BF0646A819B7
:10110000A0420DD9324669460020AFF300800700A7
:1011100008BF00F0FEFB0098A04218BF0546C419A6
:10112000FFF7C4FF05600746F01D20F007004619D1
:10113000284600F00AF8B44208BFF8BDA21B3146A9
:101140003868BDE8F84000F0B7B900210160C0E997
:10115000011070471020704770B50446051FFFF757
:10116000A5FF0068002C14BF446870BD002C18BF98
:10117000AC423CBF20466468F8D301680A18AA4212
:1011800018BF456003D12A680546114401602868EC
:101190004119A1421CBF6C6070BD61686960216823
:1011A0000844286070BD10B5FFF784FF006810BDCB
:1011B00010B50446FFF77EFF046010BD2DE9F0472F
:1011C0000D4699469246044600F1240801688806B7
:1011D00004D5E06921F01001216000E00120A8425F
:1011E00001DD471B00E00027A1697A1902EB090025
:1011F000081AA0612078C00602D42046FFF700FA42
:10120000002608E0D4E901211AF806009047206A78
:10121000401C761C20624E45F4DB2078C0060AD5BF
:101220002046FFF7EDF906E0D4E901213020904790
:10123000206A401C2062381EA7F10107F4DC07E099
:10124000D4E9012118F805009047206A401C20626B
:10125000281EA5F10105F3DC2046FFF7E7F9207809
:10126000000602D50220BDE8F0870120FBE7000060
:1012700001694A1C02610878704700B58FB0CDE95A
:1012800001310021059105497944CDE9031011464A
:101290006846FFF707FB0FB000BD0000E5FFFFFF4A
:1012A0000A6802F8010B0A607047D1E900239A42EC
:1012B00002D2531C0B601070704710B5436913B114
:1012C000AFF3008001E0FFF7D4F9012010BD1278E0
:1012D00000F124010A7000224A700122EDE7116832
:1012E0004FF0FF32E9E710B5436913B1AFF3008067
:1012F00001E0FFF723FA012010BD128800F124015C
:1013000082840022C2840122EDE711684FF0FF328F
:10131000E9E73A2800D2303820F02002412A01D3F0
:10132000A2F13700884201D34FF0FF307047000030
:10133000026811441378016018467047D16005496E
:1013400079445161044979441162002111611146C7
:1013500000F0D6B8EDFFFFFFA3010000426842B1E4
:10136000016811F8013B23B1521EC0E90012184672
:1013700070470121C160881E704742685AB1C36836
:10138000016843B983688B4205D0491E521CC0E9ED
:101390000012002070474FF0FF3070472DE9F047F2
:1013A00091460F4680460446002614F8015B2DB195
:1013B00000F076F80068405DC007F6D12B2D02D012
:1013C0002D2D18D0641E4A463946204600F052FAA8
:1013D00027B13968A14201D1C7F800804FF002045B
:1013E00071050BD54042002803DDFFF763FE046062
:1013F000A007BDE8F08746F48066E4E70028F8DA45
:10140000FFF758FE04606FF00040F2E72DE9F0416D
:1014100016460C46054600F043F8036893F80101B0
:10142000012807D0FF2C12D8185D80B101202C7044
:10143000BDE8F081D3F807013246214603F20713D5
:10144000C7182846BC46BDE8F041002360474FF06E
:10145000FF30EDE72DE9F04115460E46040002D1BC
:101460002C6804B90BA4204600F06AFA04442078E2
:1014700070B127463146384600F052FA04442078CD
:1014800010B1002004F8010B38462C60BDE8F08153
:101490000027F9E70000000000487047E010002432
:1014A00010B500F005F8001D10BD00BFF9DF010008
:1014B0000048704700110024034640688C4600280D
:1014C00018BF88423CBF03464068F8D318681844E8
:1014D000884207D00CF1030020F00700001D411ADC
:1014E000521A0146081D0A60FFF736BE10B50446C1
:1014F000FFF7D6FF0068005D00F0010010BD00009E
:101500002DE9F34F4FF0000A0C4656468DB00120EE
:101510000C9001F10C000B9062690B98012190472F
:10152000051E2DD0252D2CD0216A8847C0B16269B7
:101530000B9801219047216A88470028F7D16269FA
:10154000411E0B98904700E0761CA1690D988847D2
:10155000216A88470028F7D1E1690D988847DBE7C1
:10156000A1690D988847A842074601D1761CD3E7A8
:10157000E1690D9888477F1C02D1BAF1000F6FD046
:101580006BE162690B9800273D46394690472A284F
:1015900004D162690B98012190470125DFF8D082C0
:1015A00062690B9801219047A0F130010A290AD203
:1015B0004745E5DC07EB870100EB4107303FDFD40F
:1015C00045F01005ECE7E90601D46FF000476C2800
:1015D0000AD04C2814D0682815D06A280DD0742859
:1015E0001CD07A281AD01DE062690B98012190471F
:1015F0006C2802D045F0040514E045F002050DE02A
:1016000045F020050AE062690B980121904768289F
:1016100002D045F0080505E045F4006562690B98C5
:1016200001219047C4E9015765283DD019DC5828AD
:101630007AD00CDC452837D004DC252826D0412878
:101640009ED131E046282FD0472899D12CE05B2845
:1016500077D0612828D063287CD0642823D15AE031
:10166000F6E06F2848D008DC66281DD067281BD01C
:10167000692821D06E2816D127E0702845D073281C
:1016800068D0752847D078280DD14DE0A1690D9814
:101690008847252805463FF469AFE1690D988847DA
:1016A0006D1C3FF46AAFD8E00D9923466A466FF08F
:1016B0000100AFF30080C5E045F0400023464FF045
:1016C00000026060A80736D43EE0E8077FF447AF29
:1016D0002068011D21600068290501D506701BE7FF
:1016E000290701D5068017E7A90703D5F117C0E937
:1016F000006111E706600FE745F0400023464FF018
:1017000008026060A80716D41EE040F60E0125EA24
:101710000100606016E045F0400023464FF00A02E9
:101720006060A80707D40FE045F040006060A8079C
:1017300008D5234610220D996FF00100AFF3008009
:1017400080E007E0102223460D996FF00100FFF7BB
:101750008BF977E04FF0000963284F46C8464B46A7
:10176000CB4602D05B2806D038E0E80601D4012041
:10177000A060012732E06269D4F80CB00B98012117
:1017800090475E2807D14FF0010949466269D4F8B5
:101790000CB00B989047216939B900210A4603AB78
:1017A00043F82120491C0829FADBD8B3216949B341
:1017B00008F1010862690B98012190475D28F4D176
:1017C000B9F1000F09D0002003A951F82020D2431D
:1017D00041F82020401C0828F7DB03AB20690028D3
:1017E00020794FEA40701ED05B462246CDF800803B
:1017F000CDE901970D9900286FF0010020DAAFF3D1
:1018000000801FE0C11703AA00EBD1614B1121F04A
:101810001F0102EB8302411A136801208840034331
:101820001360C7E719E00D99224600286FF0010008
:10183000009702DAAFF3008004E0FFF7BBF901E0A4
:10184000AFF3008000280ADA401C06D10C9820B1C2
:101850004FF0FF300FB0BDE8F08F5046FAE7E907D0
:1018600001D10AF1010A064400200C9054E6000060
:10187000CCCCCC0C2DE9F05F824615468B46002778
:101880000AF10104B9460078302801D09DB113E077
:1018900014F8010B0127782803D0582801D045B14E
:1018A0000AE00DB1102D07D1002714F8010B102507
:1018B00002E0082500E00A250026B0460EE005FB00
:1018C000080005FB06F101271FFA80F801EB10461E
:1018D000B6F5803F00D3B94614F8010B2946FFF74F
:1018E00018FD0028EBDABBF1000F05D00FB1641E24
:1018F00000E05446CBF80040B9F1000F06D0FFF7E6
:10190000D9FB02210160C81EBDE8F09F48EA0640ED
:10191000FAE710B500F056F8BDE8104000F04DB8F9
:1019200030B503461D781DB10A4603E0AC4201D133
:10193000181A30BD12F8014B002CF7D15B1CF1E7EF
:1019400030B503461D783DB10A4612F8014B1CB173
:10195000AC42FAD15B1CF5E7181A30BD70477546EA
:10196000FFF79AFDAE4605006946534620F0070092
:10197000854618B020B5FEF755FDBDE820404FF074
:1019800000064FF000074FF000084FF0000BAC4688
:10199000ACE8C009ACE8C009ACE8C009ACE8C009D3
:1019A00021F007018D46704710B50446AFF3008063
:1019B0002046BDE81040FEF71EBD002801D000F013
:1019C00029B8704710B5012805D0002103A000F008
:1019D00027F8012010BD09A1F8E70000534947523C
:1019E000544D454D3A204F7574206F6620686561EF
:1019F00070206D656D6F7279000000003A204865B7
:101A00006170206D656D6F727920636F7272757091
:101A10007465640001491820ABBEFEE72600020091
:101A200070B505460C460A2000E06D1C00F011F868
:101A300035B128780028F8D102E0641C00F009F8DC
:101A400014B120780028F8D1BDE870400A20AFF327
:101A5000008008B569468DF800000320ABBE08BDC4
:101A600042F2B000C2F2004005F0DABE0000000011
:101A700010B50446006842F2001140F48070C4F2D0
:101A80000201884218D142F20830C4F20200006814
:101A900010F4403F18D00BF04BFB6168B1F5803F6C
:101AA00005D0B1F5403F2BD0B1F5003F29D1090C4D
:101AB000B0FBF1F025E000BF46F20830C5F60200A9
:101AC000006810F4403FE6D14FF4002000210AF0F6
:101AD0002FFA6168A1F580224FEAB2420A2A10D893
:101AE000DFE802F00606060606063C3E40424400D9
:101AF0006FF0010202EA5141B0FBF1F001E000BFDA
:101B000080084BF62141C0F2BE01884206D8206809
:101B1000816821F44071816010BD00BF47F641012A
:101B2000C0F27D11884207D820680122816862F3E3
:101B30000921816010BD00BF21684FF28102C0F20F
:101B4000FA229042886805D8022262F30920886050
:101B500010BD00BF40F44070886010BD0009D0E7A0
:101B60004009CEE78009CCE7C009CAE7000AC8E708
:101B7000B0B52DED028B044600284FF0FF005FD07A
:101B80000D4600295CD095ED020A95ED032A20EE62
:101B9000001A95ED013A20EE020A95ED002AB7EE03
:101BA000008A03EE031A02EE030A31EE011A30EE48
:101BB000000A78EE410A1CF017FE95ED002A95ED1B
:101BC000014A95ED023A95ED035A22EE031A84ED8F
:101BD000010A05EE441A31EE011AB0EEC16AB4EE04
:101BE000486AF1EE10FA0FDAB0EE410A1CF096FBEB
:101BF00095ED002A95ED014A95ED023A95ED035ACF
:101C000084ED020A09E000BF11EE100A40F6DB7114
:101C1000C3F6C97161F31E00A06023EE030A24EE2F
:101C2000031A05EE050A02EE051A30EE002A31EE1F
:101C3000010A78EE420A1CF0D7FD002084ED000A6C
:101C400040B2BDEC028BB0BDB0B500286ED0B7EE8F
:101C5000001A04460D46002981EE000A80ED040AB0
:101C60004FF07E5020604FF00000C4E90100E060BA
:101C700059D095ED010A95ED001AB7EEC00AB7EEFE
:101C8000C11A1CF0CDFC95ED001AB5EE401AF1EE2C
:101C900010FA0DD195ED011AB5EE401AF1EE10FAD9
:101CA00006D195ED021AB5EE401AF1EE10FA41D0C8
:101CB000B7EEC00B9FED351AB4EE410AF1EE10FA03
:101CC0004CDCB5EE400AF1EE10FA47DB9FED302A0E
:101CD000B4EE420AF1EE10FA2CDCB4EE410AF1EE59
:101CE00010FA27DB9FED2B1AB4EE410AF1EE10FA41
:101CF00004DCB4EE420AF1EE10FA43DA40F2C560B9
:101D000044F62D21C3F64D70C3F60D4120604AF212
:101D10005640616044F2AD71CBF63930C3F61971AB
:101D2000C4E90201002040B2B0BD00BFFF2040B2B4
:101D3000B0BD00BF40F2C56044F62D21C3F64D7022
:101D4000C3F60D4120604AF25640616044F2AD7125
:101D5000CBF63930C3F6197112E000BF45F66E10AC
:101D600045F20C31C3F67F70C3F6B011206048F61F
:101D7000AB00616049F28551CBF6BB30C3F6975199
:101D8000C4E90201002040B2B0BD00BFDB0FC9BFF3
:101D9000DB0F49C00000B4C200218160C0E900111E
:101DA0007047000000000000B0B52DED108B8EB024
:101DB000044600284FF0FF0003D0002918BF002A76
:101DC00004D140B20EB0BDEC108BB0BD40F218058E
:101DD0004EF69E70C2F20045002BC3F627502860D5
:101DE00000F0D28193ED009A93ED01AAB5EE409AEE
:101DF00093ED028AF1EE10FA04BFB5EE40AAF1EEBF
:101E000010FA00F0BB8192ED000A94ED011A92EDF8
:101E1000016A92ED027A94ED004A21EE405A60EE9A
:101E2000040A94ED022A66EE041A94ED033A67EE72
:101E3000042AD1ED004A06EE425AF5EE404A47EE3A
:101E4000020A47EE411A46EE012A07EE435A46EED1
:101E5000430AB6EE006A40EE031A40EE422A91EDC4
:101E6000010AF1EE10FA65EE063A91ED025A60EEC3
:101E7000860A21EE867A22EE866A04BFB5EE400A13
:101E8000F1EE10FA00F088818DED080A20EE000ACC
:101E90008DED0D6A8DED0C7A04EEA40ACDED0B3AB2
:101EA000CDED0A0A8DED095A05EE050ACDED074A7A
:101EB0000EF0D2FE2AEE0A1A8DED060A09EE091A74
:101EC00008EE081AB0EE410A0EF0C6FE94ED00CA04
:101ED00029EE00FA7CEE0CBA94ED03BA6AEE008AA1
:101EE00094ED013A28EE00EAD4ED029A2FEE2B0A87
:101EF0002CEE0C8A8DED010A68EEABAA20EE0B0ADF
:101F00002FEE081A2EEE2B2A08EE880A73EE03EA4B
:101F10000AEECB1A03EE420A6FEE2ECA02EE291A1F
:101F200023EE034A09EEAC0A8DED034A28EEAE2AF1
:101F30000FEE041A08EEC40A69EEA9FA39EEA99A5E
:101F400009EE821A08EEAF0A2EEE2E2A2EEE094A6C
:101F50002BEE0BDA02EE0B1A0BEE040A2CEE03AAA0
:101F60000FEE6F1A08EECD0A63EE0BDA0FEE4D1A84
:101F700020EE000A01EE010A23EE291A8DED021A65
:101F80003BEE0B1A8DED051A2CEE291A8DED041A75
:101F90000EF062FE94ED011A94ED022A2AEE813AC7
:101FA0009DED014ADDED031A28EE897A3DEEAD5A2A
:101FB000DDED070A04EE423A94ED034A3AEE0A6A6E
:101FC000F6EE004A0BEEE95ADDED047A0EEE083A21
:101FD000F0EE616A09EE0B6ADDED02AA7DEEE72AFA
:101FE0009DED058A0CEE843A09EE8BAA4CEE4BAAC5
:101FF0000EEE613A07EE043A9DED067A00EEC75AFE
:10200000DDED080A00EEC76AF0EE473A0EEE6F3AD1
:10201000B7EE007A71EEA10A74EEEF1A0EEE0D3AE9
:1020200087EE000A37EE607A7FEEAF0A28EE05BA37
:1020300028EE068A37EE607A71EECD0A62EE831AD8
:10204000DDED092A02EEE37A6AEE032A40EE201A59
:10205000F1EE000A0BEEC58A40EE2A2A61EE203A24
:1020600062EE200A0BEE86BA2EEE86AA00EEC78A32
:1020700074EEE60AF8EE004A2EEE85CA07EE63BA61
:1020800070EEEF0A09EE45AA09EE06CA31EECF5A04
:1020900032EEE86A62EE031A61EE032A60EE043A59
:1020A00037EEAD7A60EE830A01EEC5AA72EEE35A0E
:1020B00060EE244A40EE070A94ED007A05EE86AA07
:1020C00044EE842A24EE034A60EE025A67EE036A65
:1020D00033EE033A20EE077A75EEA67A52EE246AC2
:1020E00041EE433A04EE05BA71EEC71A02EE437AA6
:1020F00030EECE2A20EE011A07EE86BA06EE858A69
:1021000031EE040A03EE82BA02EE85CA00EE068AB8
:1021100005EE82AA01EE86CA07EE028A2BEE0B0AB2
:1021200001EE02CA0AEE0A0A08EE080A0CEE0C0AD0
:102130000EF092FD20EE0A1ADDED0A0A20EE0B2ABF
:10214000DDED0B3A20EE083A9DED0C7A20EE0C0AFC
:102150009DED0D6A95ED004A44EE413A94ED011A69
:1021600044EE420A94ED022A04EE437A94ED033AD7
:1021700004EE406A94ED004A14E000BFB5EE408AD8
:10218000F1EE10FA7FF43FAE20460EB0BDEC108B9E
:10219000BDE8B04000F040B8B5EE405AF1EE10FA9C
:1021A0007FF472AE94ED045A00EE851A03EE854A70
:1021B00007EE052A06EE053A84ED011A84ED004A81
:1021C00021EE010A84ED022A84ED033A04EE040AAA
:1021D00002EE020A03EE030A0EF03EFD94ED001A31
:1021E00094ED012A94ED023A94ED034A20EE011A8F
:1021F000002020EE022A84ED001A20EE031A84ED5E
:10220000012A20EE040A84ED021A84ED030A40B28A
:102210000EB0BDEC108BB0BDB0B52DED108B0446EB
:1022200000284FF0FF0003D0002918BF002A03D177
:1022300040B2BDEC108BB0BD40F2180542F6023042
:10224000C2F20045C3F6075094ED011A92ED016AFF
:10225000286092ED027A92ED000A94ED003A21EEA8
:10226000405A94ED022A60EE030A94ED034A66EEAA
:10227000031A91ED00EA67EE032AB5EE40EA06EE96
:10228000425A91ED01DA47EE020A91ED02CA47EE99
:10229000411A46EE012A07EE445A46EE440AB6EECB
:1022A000006A40EE041A40EE422AF1EE10FA04BF32
:1022B000B5EE40DAF1EE10FA25EE06AA20EE86BA67
:1022C00021EE869A22EE868A00F090802DEE0D0A8D
:1022D0000EEE0E0A0CEE0C0A0EF0BEFCB1EE001A69
:1022E00094ED013A94ED034A94ED007A24EE046AE9
:1022F000D4ED023A23EE015A67EE071A2EEE002AB9
:1023000074EE040A65EE062A61EE811A77EE074A3A
:1023100042EE602A61EEA35A63EE816A43EE212AFF
:102320006DEE001A42EE245A2CEE000A41EEE42A29
:1023300046EE865A33EEA36A27EE017A41EEE05A62
:10234000F2EE000A22EE06DA32EEC5CA63EEA32AE6
:1023500063EE204A63EE037A07EE22DA63EEA00A08
:1023600004EEA7CA07EE27DA35EEE6EA04EEA2CAC3
:1023700027EE817A07EEA0EA33EE033A27EE04FA5D
:1023800000EE05CA00EEA2EA02EE43FA22EE811A3E
:1023900001EEC3DA00EE26EA04EE01FA2CEE0C0A96
:1023A00001EEC6FA0DEE0D0A0EEE0E0A0FEE0F0A42
:1023B0000EF052FC20EE0D1A95ED004A20EE0C2A8C
:1023C00020EE0E3A20EE0F0A04EE41AA94ED011A17
:1023D00004EE42BA94ED022A04EE439A94ED003AD8
:1023E00004EE408A94ED034A06E000BFB5EE40CA11
:1023F000F1EE10FA7FF46AAF94ED045A0BEE051A71
:102400000AEE053A09EE052A08EE054A84ED011A9E
:1024100084ED003A21EE010A84ED022A84ED034A9C
:1024200003EE030A02EE020A04EE040A0EF014FCA4
:1024300094ED001A94ED012A94ED023A94ED034ACA
:1024400020EE011A002020EE022A84ED001A20EE70
:10245000031A84ED012A20EE040A84ED021A84EDA9
:10246000030A40B2BDEC108BB0BD000000000000BC
:10247000A0B1B0B504460D4600F09AFB48212046B5
:10248000FEF75DFD287803226988A56400F090FCC2
:102490000020BDE8B04040B2704700BFFE2040B20F
:1024A0007047000000000000002908BF704770B5A9
:1024B00096B00C46816C01AA002308780026498852
:1024C00000F01AFB20B116B0BDE87040704700BFA5
:1024D0009DF812009DF814209DF813109DF81530FA
:1024E0009DF817509FED1C1A090341EA00510006A0
:1024F0009DF8160041EA021103F00F0241EA1311A0
:102500004FEA004048BF01F1704140EA02609DF887
:10251000182040EA052000EE101A1044190748BFA1
:1025200000F17040B8EEC00A02EE100A9DF81100EA
:10253000207080EE010AB8EEC22A84ED010AC4E9D7
:102540000366C4E9056682EE010A84ED020A16B04C
:10255000BDE87040704700BF8096184B0000000037
:10256000B1EE601A80FE602AB4EE401AF1EE10FA65
:1025700031FE020A7047000042F29810C2F2004099
:1025800006F0B2B80000000041F290200821C2F22B
:102590000040406818F0CCB910B50320002101F0CC
:1025A0007BFA41F290249220C2F2004401220023DF
:1025B00004F8010F0020214601F06AFBE11D002014
:1025C0001322012301F03CFB002010BD000000009D
:1025D000022001214FF0FF3218F0EEB90000000098
:1025E0009FED010A704700BF0000C84300000000D3
:1025F00041F290201021C2F20040406818F098B9D2
:1026000010B50720002101F047FA41F29024822002
:10261000C2F200440122002304F8010F00202146E9
:1026200001F036FB04F10E0100200622012301F027
:1026300007FB002010BD0000042001214FF0FF32F5
:1026400018F0BAB9000000002DE9F04100284FF061
:10265000FE0700F08F810E46002900F08B8141F2C9
:1026600090280546C2F2004898F8000020B1FD27E6
:1026700078B2BDE8F08100BF18F052FA0028C8F81F
:10268000040000F07F8144464BF27E60EE6224F845
:10269000010F012001F014FB0320002101F0FCF9DF
:1026A000002002220023214601F0F2FA032001213A
:1026B00001F0F2F94BF214602080012001F000FBE0
:1026C0000720002101F0E8F9002002220023214622
:1026D00001F0DEFA0720012101F0DEF91E2001F0F1
:1026E000EFFA012001F0ECFA0320002101F0D4F907
:1026F0009E202070002001220023214601F0C8FA0C
:10270000002002220023214601F09AFA0320012131
:1027100001F0C2F9012001F0D3FA0320002101F0F9
:10272000BBF900200122002321468026267001F0FB
:10273000AFFA002002220023214601F081FA032093
:10274000012101F0A9F960781E2840F017810120CD
:10275000012501F0B5FA0720002101F09DF944465A
:1027600000200122002304F8016F214601F090FAB5
:10277000002002220023214601F062FA07200121F5
:1027800001F08AF920780F2840F0F8800A2001F043
:10279000EBF80B2001F0E8F842F699220020C0F691
:1027A00000020121002701F063FA42F289510A2058
:1027B000C0F6000101F018F942F2F1510B20C0F609
:1027C000000101F011F944464AF6402024F8010FB7
:1027D000012001F075FA0320002101F05DF90020CD
:1027E00002220023214601F053FA0320012101F0C7
:1027F00053F940F241102080012001F061FA0320DA
:10280000002101F049F9002002220023214601F0B5
:102810003FFA0320012101F03FF940F653002080E8
:10282000012001F04DFA0320002101F035F90020CC
:1028300002220023214601F02BFA0320012101F09E
:102840002BF94FF48B602080012001F039FA03202E
:10285000002101F021F9002002220023214601F08D
:1028600017FA0320012101F017F940F27D40208082
:10287000012001F025FA0320002101F00DF90020CC
:1028800002220023214601F003FA0320012101F076
:1028900003F9322001F014FA40F20F1020800120D9
:1028A00001F00EFA0720002101F0F6F800200222C4
:1028B0000023214601F0ECF90720012101F0ECF89A
:1028C0004FF444702080012001F0FAF90720002124
:1028D00001F0E2F8002002220023214601F0D8F99D
:1028E0000720012101F0D8F816202080012001F0F6
:1028F000E7F90720002101F0CFF800200222002391
:10290000214601F0C5F90720012101F0C5F84FF477
:102910008C702080012001F0D3F90720002101F004
:10292000BBF8002002220023214601F0B1F9072064
:10293000012101F0B1F848F215002080012001F0DA
:10294000BFF90720002101F0A7F800200222002390
:10295000214601F09DF90720012101F09DF80A2090
:1029600001F0AEF90A2088F8005001F011F80B20B0
:1029700001F00EF878B2BDE8F08100BFFC2778B214
:10298000BDE8F081FE2778B2BDE8F08100000000CC
:1029900000283FD041F290219FED203AC2F2004141
:1029A000B1F90920B1F90DC0B1F90B3000EE102AD0
:1029B00002EE10CA01EE103A4FF60003CFF6FF7395
:1029C000B8EEC00AB8EEC11AB8EEC22A80EE030A09
:1029D00081EE031A80ED040A82EE030A80ED051AE7
:1029E00080ED060AB4EE001A4A7EB3EE072A897E0D
:1029F000D20042EA51120021B1EB922F18BF1A43C4
:102A000000EE102AB8EEC00A00EE012A80ED0A2A74
:102A100048B27047FE2148B2704700BF00A0AA45E7
:102A200090B341F290219FED1A3AC2F200419FED1E
:102A3000194AB1F90F20B1F91130B1F9131000EEB4
:102A4000102A01EE103A02EE101AC16AB8EEC00A5E
:102A500091ED015AB8EEC11AB8EEC22A80EE030A0F
:102A600081EE031A82EE032A91ED003A10EE043A49
:102A700091ED020A11EE045A12EE040A80ED073AB3
:102A800080ED085A80ED090A6FF00100704700BF21
:102A90006F12034235FA8E3C10B5032000F08CFF14
:102AA00041F29024C2F2004438B90320012100F021
:102AB000F3FF6068022117F03BFF072000F07CFF66
:102AC000002818BF10BD0720012100F0E5FF606855
:102AD0000421BDE8104017F02BBF000000000000EB
:102AE000182001214FF0FF3217F066BF00000000F0
:102AF00070470000000000002DE9F04141F2202461
:102B0000C2F200442778012F0ED1154682B10E463D
:102B10000746A0686421984617F076FE60B1FB2056
:102B200040B2BDE8F08100BFFD2040B2BDE8F081B9
:102B3000FE2040B2BDE8F081E06800E0006978B3B3
:102B40000178B94202D14168B14217D0006938B367
:102B50000178B94202D14168B1420FD00069F8B1A1
:102B60000178B94202D14168B14207D00069B8B1D9
:102B70000178B942E2D14168B142DFD18668A068EC
:102B800017F0AEFE7EB1002230462946434617F0CC
:102B90003FFD002818BF4FF0FF3040B2BDE8F08184
:102BA000A06817F09DFEFC2040B2BDE8F081000057
:102BB0002DE9F04F89B041F22027C2F20047387862
:102BC00020B1FD2040B209B0BDE8F08F07F1100040
:102BD0006021FEF7D6F943F6C02041F60811C2F293
:102BE000004041F60C120024C0F8804CC0F8844C20
:102BF000445042F29051845042F2945244508450D6
:102C000042F6F120C0F600007860002017F028FEA0
:102C10000028B86000F0C68042F2684501AEC2F2FA
:102C2000004541F21009284631464FF0010A87F865
:102C300000A0CDE901444FF0020BC0F20209CDE93A
:102C400003BACDE90544079406F05AFF28463146F9
:102C5000CDF808A04FF08048CDF80480CDE903BA44
:102C6000CDE90544079406F04BFF00210022002324
:102C70002846009406F08CFFA9F10F010022284697
:102C800006F07AFE3878012809D142F6C160C0F614
:102C90000000F86143F2F170C0F60000386142F2C2
:102CA0006840C2F2004007F0EBFD42F2085501AE69
:102CB000C2F20045314628460024CDE90144CDE961
:102CC00003BBCDE90544079406F01AFF01A831467D
:102CD000CDE904B480E8000D2846CDE9064406F0AD
:102CE0000FFF0121012200232846009406F050FF27
:102CF00000222846494606F03FFE387843F2492A2A
:102D0000C0F6000A012806D143F2F170C7F844A0CA
:102D1000C0F60000386342F20850C2F2004007F0EB
:102D2000AFFD42F2A8550DF10408C2F2004541463C
:102D300028460226CDE90144CDE90366CDE90544E4
:102D4000079406F0DDFE012002904FF080400190D4
:102D500028464146CDE90366CDE90544079406F0CF
:102D6000CFFE0121012200232846009406F010FF27
:102D700000222846494606F0FFFD3878012806D192
:102D800043F2F170C7F864A0C0F60000386542F263
:102D9000A850C2F2004007F073FD002040B209B015
:102DA000BDE8F08FFF2040B209B0BDE8F08F000011
:102DB0002DE9F04141F22028C2F2004898F8003095
:102DC000012B0FD114460D460646002A08BF0A24DF
:102DD000D8F80800642117F017FD38B1FB2040B285
:102DE000BDE8F081FD2040B2BDE8F081D8F80C00CC
:102DF00001E000BF0069F8B10178B14202D1416839
:102E0000A94240D00069B8B10178B14202D141680D
:102E1000A94238D0006978B10178B14202D1416845
:102E2000A94230D0006938B10178B142E2D141689D
:102E3000A942DFD127E000BF142000F045FEB8B161
:102E4000074654210022204617F02AFCB860B8B18A
:102E5000D8F80C003861D8F808003E707D603C73EB
:102E6000C8F80C7017F03CFD002040B2BDE8F081BE
:102E7000D8F8080017F034FDFE2040B2BDE8F0811C
:102E8000384600F06DFDD8F8080017F029FDFF2046
:102E900040B2BDE8F081000041F22021C2F20041C1
:102EA0000A78012A04D138B14860002040B2704746
:102EB000FD2040B2704700BFFE2040B270470000C6
:102EC0002DE9F04FAFB06846402100F10D0942F204
:102ED0006840C2F2004006F0A3FE41F2202800281C
:102EE000C2F2004800F0868042F268460DF1940A72
:102EF000C2F200460DF1540B06E000BF40213046FF
:102F000006F08EFE002875D04021304652465B46C2
:102F100006F092FE00286DD126986FF060410028DF
:102F20004FF0020708BF40F2FF71259AB0F1804FC1
:102F300001EA020500F14041B1FA81F0279B08BF88
:102F40000327D8F80420B3F1005F18BF47092846CB
:102F500012B1284639469047D8F80C1001E000BF5E
:102F600009690029CAD00A7812B94A68824218D081
:102F700009690029C2D00A7812B94A68824210D081
:102F800009690029BAD00A7812B94A68824208D081
:102F900009690029B2D00A78002AE1D14A68824240
:102FA000DED18C68002CA9D028998DF80070CDE96D
:102FB00001504FF6C03001F00F01C0F601006F461E
:102FC000455C0F398DF80C5007EB050000F10D0042
:102FD00018BFC5F14001FDF7B2FF484659462A46E1
:102FE000FDF726FF002200232046394617F0A4FBF8
:102FF00084E700BF42F208504021C2F2004006F0D0
:103000000FFE002800F0888042F208560DF1940A65
:10301000C2F200460DF1540B06E000BF40213046DD
:1030200006F0FEFD002877D04021304652465B4630
:1030300006F002FE00286FD126986FF0604100284C
:103040004FF0020708BF40F2FF71259AB0F1804FA0
:1030500001EA020500F14041B1FA81F0279B08BF67
:103060000327D8F80420B3F1005F18BF47092846AA
:1030700012B1284639469047D8F80C1001E000BF3D
:1030800009690029CAD00A78012A02D14A68824215
:103090001AD009690029C1D00A78012A02D14A68E8
:1030A000824211D009690029B8D00A78012A02D1D8
:1030B0004A68824208D009690029AFD00A78012AFB
:1030C000DED14A688242DBD18C68002CA6D02899D8
:1030D0008DF80070CDE901504FF6C03001F00F01BE
:1030E000C0F601006F46455C0F398DF80C5007EBB8
:1030F000050000F10D0018BFC5F14001FDF71FFFED
:10310000484659462A46FDF793FE002200232046F2
:10311000394617F011FB81E742F2A8504021C2F274
:10312000004006F07DFD002800F0888042F2A8569D
:103130000DF1940AC2F200460DF1540B06E000BFF7
:103140004021304606F06CFD002877D04021304603
:1031500052465B4606F070FD00286FD126986FF04E
:10316000604100284FF0020708BF40F2FF71259A26
:10317000B0F1804F01EA020500F14041B1FA81F05F
:10318000279B08BF0327D8F80420B3F1005F18BFBE
:103190004709284612B1284639469047D8F80C10FE
:1031A00001E000BF09690029CAD00A78022A02D1C9
:1031B0004A6882421AD009690029C1D00A78022AD5
:1031C00002D14A68824211D009690029B8D00A7830
:1031D000022A02D14A68824208D009690029AFD088
:1031E0000A78022ADED14A688242DBD18C68002C40
:1031F000A6D028998DF80070CDE901504FF6C03067
:1032000001F00F01C0F601006F46455C0F398DF8E3
:103210000C5007EB050000F10D0018BFC5F140018F
:10322000FDF78DFE484659462A46FDF701FE00226D
:1032300000232046394617F07FFA81E72FB0BDE81A
:10324000F08F0000000000002DE9F04FAFB068469D
:10325000412100F10D0942F26840C2F2004006F03F
:10326000DFFC41F220280028C2F2004800F08680EE
:1032700042F268460DF1940AC2F200460DF1540B79
:1032800006E000BF4121304606F0CAFC002875D098
:103290004121304652465B4606F0CEFC00286DD1F7
:1032A00026986FF0604100284FF0020708BF40F2F7
:1032B000FF71259AB0F1804F01EA020500F140410B
:1032C000B1FA81F0279B08BF0327D8F80420B3F197
:1032D000005F18BF4709284612B128463946904773
:1032E000D8F80C1001E000BF09690029CAD00A789B
:1032F00012B94A68824218D009690029C2D00A78F6
:1033000012B94A68824210D009690029BAD00A78F5
:1033100012B94A68824208D009690029B2D00A78F5
:10332000002AE1D14A688242DED18C68002CA9D003
:1033300028998DF80070CDE901504FF6C03001F0AA
:103340000F01C0F601006F46455C0F398DF80C5037
:1033500007EB050000F10D0018BFC5F14001FDF7B6
:10336000EEFD484659462A46FDF762FD002200233D
:103370002046394617F0E0F984E700BF42F20850D2
:103380004121C2F2004006F04BFC002800F088808A
:1033900042F208560DF1940AC2F200460DF1540BA8
:1033A00006E000BF4121304606F03AFC002877D005
:1033B0004121304652465B4606F03EFC00286FD164
:1033C00026986FF0604100284FF0020708BF40F2D6
:1033D000FF71259AB0F1804F01EA020500F14041EA
:1033E000B1FA81F0279B08BF0327D8F80420B3F176
:1033F000005F18BF4709284612B128463946904752
:10340000D8F80C1001E000BF09690029CAD00A7879
:10341000012A02D14A6882421AD009690029C1D022
:103420000A78012A02D14A68824211D0096900292A
:10343000B8D00A78012A02D14A68824208D00969C4
:103440000029AFD00A78012ADED14A688242DBD156
:103450008C68002CA6D028998DF80070CDE9015019
:103460004FF6C03001F00F01C0F601006F46455C19
:103470000F398DF80C5007EB050000F10D0018BF57
:10348000C5F14001FDF75BFD484659462A46FDF768
:10349000CFFC002200232046394617F04DF981E782
:1034A00042F2A8504121C2F2004006F0B9FB0028C8
:1034B00000F0888042F2A8560DF1940AC2F200464C
:1034C0000DF1540B06E000BF4121304606F0A8FB89
:1034D000002877D04121304652465B4606F0ACFBCF
:1034E00000286FD126986FF0604100284FF0020746
:1034F00008BF40F2FF71259AB0F1804F01EA020542
:1035000000F14041B1FA81F0279B08BF0327D8F8AA
:103510000420B3F1005F18BF4709284612B12846BE
:1035200039469047D8F80C1001E000BF096900291E
:10353000CAD00A78022A02D14A6882421AD009699E
:103540000029C1D00A78022A02D14A68824211D0E9
:1035500009690029B8D00A78022A02D14A68824251
:1035600008D009690029AFD00A78022ADED14A685A
:103570008242DBD18C68002CA6D028998DF800708F
:10358000CDE901504FF6C03001F00F01C0F6010047
:103590006F46455C0F398DF80C5007EB050000F1C4
:1035A0000D0018BFC5F14001FDF7C9FC484659465A
:1035B0002A46FDF73DFC002200232046394617F03D
:1035C000BBF881E72FB0BDE8F08F000000000000DD
:1035D0002DE9F0479AB041F22027C2F200473F7828
:1035E000012F0FD10446022817D801F0FE001D4616
:1035F00017460E4602280BD055B9FE2040B21AB02D
:10360000BDE8F087FD2040B21AB0BDE8F08700BFEA
:10361000DDF888A0BAF1400F04D9FF2040B21AB0FB
:10362000BDE8F0870DF1040864214046FDF7A9FCD0
:10363000032EF2D860B24FF6BC02C0F6010252F877
:103640002090DFE806F0030D071100BF019700216D
:1036500000200EE001974FF00050002109E000BF6C
:103660000197002003E000BF4FF0005001974FF09A
:1036700080410390D9F808000291B0F5407F07D04F
:10368000B0F5807F0AD14FF40010002108E000BFA0
:103690004FF400104FF4801102E000BF0021002021
:1036A000CDE90610002005904FF400000890BAF113
:1036B000090F4FF001000990504622D3BAF10D0FC7
:1036C00002D209201DE000BFBAF1110F02D20A2078
:1036D00017E000BFBAF1150F02D20B2011E000BFB6
:1036E000BAF1190F02D20C200BE000BFBAF1210F82
:1036F00002D20D2005E000BF0F20BAF1310F38BF14
:103700000E2008F12407049038465146FDF739FC95
:10371000002D18BFBAF1000F04D1484606F0E0FBB7
:1037200048B90EE0384629465246FDF781FB484627
:1037300006F0D6FB28B101A948463A4606F064F9DE
:1037400030B343F6C02040F68841C2F2004014FB7B
:103750000102D2F8803CD2F8846C013303F01F05DB
:10376000B5420CD002F5486714FB010064213A68A9
:1037700002FB010001A96422FDF79FFB3D600020D0
:10378000B54208BF4FF0FF3040B21AB0BDE8F08735
:10379000002040B21AB0BDE8F08700000000000031
:1037A00061B180B582B091F804C00A684B1D012157
:1037B000CDF800C0FFF70CFF02B080BD6FF0010034
:1037C000704700000000000061B180B582B091F840
:1037D00004C00A684B1D0021CDF800C0FFF7F8FEB9
:1037E00002B080BD6FF001007047000000000000D3
:1037F0002DE9F04FA3B0684642F2684500F1240875
:10380000C2F2004519AE00BF2846314606F008FB5B
:103810000028F9D043F6C02742F26845C2F20047BB
:10382000C2F2004564246E46D7F8800CD7F8841C99
:10383000884220D0284606F053FB00281EBFD7F848
:10384000800CD7F8841C884215D0D7F8840C6422E9
:1038500000FB04713046FDF730FBD7F8840C31468D
:103860000130424600F01F00C7F8840C284606F0DD
:10387000CBF80028D8D042F2085519AEC2F2004564
:103880002846314606F0CCFA0028F9D042F2085515
:1038900041F6081441F60C16C2F200454FF0640AD6
:1038A000E9463859B95988421DD0284606F018FB18
:1038B00000281EBF3859B959884214D0B85964221B
:1038C00000FB0A7000F688414846FDF7F6FAB85941
:1038D00049460130424600F01F00B851284606F024
:1038E00093F80028DDD042F2A85519AEC2F2004587
:1038F0002846314606F094FA0028F9D042F2A85939
:1039000042F2905442F29455C2F200494FF0640AD8
:1039100041F6101B6E463859795988421DD04846E9
:1039200006F0DEFA00281EBF38597959884214D0B3
:103930007859642200FB0A7000EB0B013046FDF75A
:10394000BCFA785931460130424600F01F007851E8
:10395000484606F059F80028DDD023B0BDE8F08FC6
:1039600018F01ABC0000000000F0FE000A2809D17F
:1039700080B5282007F054FA0020BDE8804040B20E
:10398000704700BFFF2040B27047000000000000F9
:1039900000F0FE000A2809D180B5282007F054FA6B
:1039A0000020BDE8804040B2704700BFFF2040B219
:1039B00070470000000000000C2801D9002070476B
:1039C00080B54FF6D801C0F6010101EBC00231F815
:1039D0003010506807F060F90138B0FA80F0400903
:1039E00080BD00000000000021B10C2806D9FF2096
:1039F00040B27047FE2040B2704700BF4FF6D80279
:103A0000C0F6010232F83000C2071FD182071FD46E
:103A100042071FD402071FD4C2061FD482061FD438
:103A200042061FD402061FD4C2051FD482051FD42C
:103A300042051FD402051FD4C2041FD482041FD420
:103A400042041FD4000424D50F201CE000201AE0FB
:103A5000012018E0022016E0032014E0042012E008
:103A6000052010E006200EE007200CE008200AE008
:103A7000092008E00A2006E00B2004E00C2002E008
:103A80000D2000E00E2041F2E042C2F2004242F876
:103A90002010002040B270470C2803D9FF2040B20C
:103AA000704700BF80B50A464FF6D801C0F6010145
:103AB00001EBC00331F83010586807F0F5F800202A
:103AC000BDE8804040B2704717F042BE00000000E1
:103AD000062803D9FF2040B2704700BF4FF674118B
:103AE000B7EE001AC0F60101062851F8301080FE2A
:103AF000410A9FED1E1A0A6880FE010AD16A01F18F
:103B0000010101EE101AB8EE411A20EE010ABCEED6
:103B1000C00A10EE101A11D8DFE800F004100A10E5
:103B20000A10040002F134000160002040B2704726
:103B300002F138000160002040B2704700F0FB0342
:103B4000012B05D102F13C000160002040B270471A
:103B5000032805D102F140000160002040B2704707
:103B600002F15C000160002040B2704700000000DC
:103B700010B52DED028B062804D9FF2040B2BDEC14
:103B8000028B10BD0446B0EE408A09F0F9FA4FF6F8
:103B90007411BFEE001AC0F6010151F834104A68E2
:103BA0000132B0FBF2F000EE100A0022B8EE400A3B
:103BB00080EE080A30EE010ABCEEC00A10EE100AD0
:103BC000B2EB104F04D0FF2040B2BDEC028B10BD11
:103BD0000A68D062C860002040B2BDEC028B10BD04
:103BE000062803D9FF2040B2704700BF80B54FF6CA
:103BF0007412C0F6010202EBC00152F8300089884D
:103C00000BF072FD0020BDE8804040B2704700001C
:103C1000062803D9FF2040B2704700BF80B54FF699
:103C20007412C0F6010202EBC00152F8300089881C
:103C30000BF02AFE0020BDE8804040B27047000033
:103C400080B518B1FF2040B280BD00BF42F61040E1
:103C5000C2F2004013B10AF0BBFB02E014230AF0E9
:103C6000BBF9002818BF012040B280BD0000000051
:103C700052B141F22853C2F2004303EB401040F826
:103C80002120002040B27047FE2040B27047000063
:103C900080B518B1FF2040B280BD00BF42F6104091
:103CA000C2F2004013B10AF047FE02E014230AF00A
:103CB00087FC002818BF012040B280BD0000000032
:103CC00070B5044616F02CFC0546FF2616F00CFCD9
:103CD000411C05290CD80120884010F0310F0CD16F
:103CE00010F0060F0CD0204605F032FE13E000BFA6
:103CF0006FF00041884218BF002670B270BD00BF4F
:103D00004FF47A70B0FBF5F1B4FBF1F0A14288BF3B
:103D1000012016F0BDFB002670B270BD000000004F
:103D200019F0A2BF000000002DE9F04116F0F8FBE9
:103D3000044619F099FF4EF218074FF47A78CEF244
:103D40000007B8FBF4F404FB00F63D6819F08CFFA3
:103D500060433968864200FB08F008BF294657F8DF
:103D6000042C01FB08F10132B1FBF2F1401A0021F1
:103D700000F57A70BDE8F08142F6146243F2640106
:103D8000C2F20042012818BF0022C2F200410028FE
:103D900018BF1146084670470068C169C90658BF78
:103DA000704745F200010323C4F2000101F54042CF
:103DB000904241F2485208BF0123411AC2F2004228
:103DC00018BF194601EBC10102EB8101102202620A
:103DD000086A08B1004700BF7047000000000000FB
:103DE00080B5012802D9FF2040B280BD8446FE2064
:103DF000002918BF002A01D140B280BD42F6146EDE
:103E000043F26400C2F2004EBCF1010F18BF4FF044
:103E1000000EC2F20040BCF1000F18BF70461BB18B
:103E20000CF03EFC40B280BD0CF032FD40B280BDD3
:103E300032B1FF23012898BF082905D958B270472D
:103E4000FE2358B2704700BF00EBC00041F2485358
:103E5000C2F2004303EB8000002340F8212058B257
:103E6000704700000000000080B5012802D9FF2043
:103E700040B280BD8446FE20002918BF002A01D12F
:103E800040B280BD42F6146E43F26400C2F2004EAE
:103E9000BCF1010F18BF4FF0000EC2F20040BCF1A0
:103EA000000F18BF70461BB10CF08AFD40B280BDF8
:103EB0000CF0F6FD40B280BDB0B578B10446017497
:103EC00001202070FFF72CFF217C0025C4E90205AA
:103ED0000846FFF79DFE68B2B0BD00BFFF2568B27F
:103EE000B0BD0000000000002DE9F0472DED0A8B69
:103EF00070B104460078002800F08A8071B1012971
:103F000040F086804FF6401AC0F6010A0AE000BF72
:103F1000FF2568B2BDEC0A8BBDE8F0874FF6AC1AFE
:103F2000C0F6010AB2EE08AAB6EE008A4FF0000809
:103F30004FF001099FED4DBA00279FED4DCA00BF1C
:103F40001AF827000AEB8706FF283ED0717801EBAC
:103F5000410100EB81000C3000EE100AB8EEC00AFF
:103F600030EE0B0A80EE0A0A1AF03CFE20EE0C9AA4
:103F70002078B5EE409AF1EE10FA25DD002847D002
:103F800084F80090FFF7CCFE217CB0EE490AC4E92A
:103F900002080846FFF7ECFD217CB0EE480A054612
:103FA0000846FFF795FD28434CD1207880B384F86C
:103FB0000090FFF7B5FE217CC4E902080846FFF730
:103FC0000FFE60B13EE000BF48B184F80090FFF7FB
:103FD000A7FE217CC4E902080846FFF719FE708895
:103FE000FFF76EFE207848B184F80090FFF798FE46
:103FF000217CC4E902080846FFF70AFE1420FFF7F7
:104000005FFE20780C2F09D0002807F1010797D117
:10401000FF2568B2BDEC0A8BBDE8F08700284FF0A1
:1040200000053FF476AF01202070FFF779FE217C78
:10403000C4E902050846FFF7EBFD68B2BDEC0A8B48
:10404000BDE8F08720780028E2D001202070FFF73B
:1040500067FE217C0022C4E902020846FFF7D8FD72
:10406000FF2568B2BDEC0A8BBDE8F08700008AC26C
:104070000000DC430000000010B52DED048B18B3E8
:104080000446007800B3B0EE608AB0EE409A01209A
:104090002070FFF745FE217CB0EE490A0022C4E9FA
:1040A00002020846FFF764FD217CB0EE480A044690
:1040B0000846FFF70DFD204318BF4FF0FF3040B218
:1040C000BDEC048B10BD00BFFF2040B2BDEC048BE3
:1040D00010BD00000000000010B598B10446007843
:1040E00080B101202070FFF71BFE217C0022C4E973
:1040F00002020846FFF774FD002818BF4FF0FF309A
:1041000040B210BDFF2040B210BD00000000000012
:1041100010B598B10446007880B101202070FFF7F7
:10412000FFFD217C0022C4E902020846FFF770FD72
:10413000002818BF4FF0FF3040B210BDFF2040B242
:1041400010BD000000000000FEE7000000000000BD
:104150002DE9F04381B02DED108B84B0044600288A
:104160004FF0FE0000F0C5840F46002900F0C18426
:10417000FFF7DAFDD4E90023801A99411BF09EFA7B
:1041800000EE100A9FEDE6DA80EE0D0A84ED020AD9
:10419000FFF7CAFD3E78227DC4E90001B24200F07B
:1041A0009D80E0680EF0E0F9E06806300EF0DCF982
:1041B000E0680C300EF0D8F9E06812300EF0D4F957
:1041C000E06818300DF08CFFE0681E300DF088FFBD
:1041D00004F5A26004F5797510F07EFC04F24C50F1
:1041E00010F07AFC284610F077FC04F5846010F09B
:1041F00073FC04F25C4010F06FFC04F5936010F067
:104200006BFC04F2D44010F067FC04F521700DF053
:10421000C7FA04F544700DF0C3FA9FEDD58A04F592
:10422000C060B0EE480A0DF0EBFBB0EE480A04F5B2
:10423000C4600DF0E5FBB0EE480A04F5C8600DF06F
:10424000DFFBB0EE480A04F5CC600DF0D9FBB0EE10
:10425000480A04F5D0600DF0D3FBB0EE480A04F52F
:10426000D4600DF0CDFB04F5DC600CF0C9FFE06814
:104270000025C4E9E755C4E9E955C4F8AC539FEDFE
:10428000BD0AC4F8B05394ED1EAA90ED868A9FED46
:10429000BABA38EE009AB0EE480AF0EE4A0AB0EE2A
:1042A0004B1A01F0E5FCB0EE40CAB0EE490AF0EE60
:1042B0004A0AB0EE4B1A01F0DBFCB0EECC1AB0EEBD
:1042C000C00AB4EE401AF1EE10FAC8BF012539FE5B
:1042D000080A267584EDED0A84F8C053387D40B194
:1042E000B01E022805D894F8C40310B9012084F840
:1042F000C50304F1C40694ED060AD4ED0A0A94ED50
:10430000291AD4ED261A304614F042FD04F5D2796C
:10431000D4ED0E0A94ED120A94ED291AD4ED261A62
:10432000484614F035FD9FED959A94ED3EFAB0EEB7
:10433000490A9FED93AAB7EE00BA9FED92CAB0EE7C
:104340004CEA0FEE4F0A80EE0A8AB0EEC80AB4EECD
:104350004B0AF1EE10FA37DCB0EE480A19F052FFC2
:104360001AF0A2FD9FED881AB0EE402A9FED874A11
:1043700028EE013A20EE044A9FED850A03EE004A3A
:1043800002EE410A9FED831A31EE433AB0EEC44A81
:1043900020EE000A03EE030A9FED7F3A24EE033A73
:1043A00023EE013AB1EEC01A22EE038AB4EE411AAE
:1043B000F1EE10FA80F1A4839FED780A21EE000A55
:1043C0002FEE000A88EE00EAB0EE490A94ED76FA84
:1043D0000FEE4F0A80EE0A8AB0EEC80AB4EE4B0A1E
:1043E000F1EE10FA37DCB0EE480A19F00BFF1AF0C4
:1043F0005BFD9FED651AB0EE402A9FED644A28EE02
:10440000013A20EE044A9FED620A03EE004A02EEF2
:10441000410A9FED601A31EE433AB0EEC44A20EEF5
:10442000000A03EE030A9FED5C3A24EE033A23EE02
:10443000013AB1EEC01A22EE038AB4EE411AF1EE4F
:1044400010FA80F163839FED550A21EE000A2FEEEA
:10445000000A88EE00CA1EEE100A40F20108C7F6F4
:10446000807820F00040B0F1FF4F2BD91CEE100AED
:1044700020F0004040453CD3207D04284DD8DFE8A3
:1044800000F003CF515B8F00E0680EF095FAE06812
:1044900006300EF091FAE0680C300EF08DFAE0680C
:1044A00012300EF089FAE06818300DF0C1FEE068B5
:1044B0001E300DF0BDFE2046394600F0C1FC002044
:1044C00017E300BF94ED5D0AB3EE041A3EEE000A56
:1044D000002084ED5D0AB4EE410AF1EE10FAC8BF87
:1044E000012084F878011CEE100A20F000404045BD
:1044F000C2D294ED950AB3EE041A3CEE000A0020F5
:1045000084ED950AB4EE410AF1EE10FAC8BF01201D
:1045100084F85802207D0428B1D9FD20E9E200BFCB
:10452000002474492046394600F08AFC204601F0F8
:10453000C7F80020DDE200BF2046394600F080FCCD
:1045400097ED020A94ED2F1A9FEDAA2A204600EE5D
:10455000021A94ED300A84ED2F1A97ED021A01EE3B
:10456000420A84ED300A01F0ABF80020C1E200BF3E
:1045700000000000DB0F4940DB0FC9402ECCE23DBC
:10458000BDAEDF3D0000C07FCDCC4C3DC52030BC72
:1045900031082C3DF6285C3E0000B4434A0C823EB4
:1045A000FFF7C2FBD4E90023801A99411BF086F87B
:1045B00000EE100A0020C4F8BC00C4F8C00080EE71
:1045C0000D0A97ED048A84ED020AFFF7ADFB4FF464
:1045D0007A720023FBF769FF94F8C513D4F8C83347
:1045E00094F8C4230029A0EB030100F0F580002A11
:1045F00040F0F2800122A4F8C423C4F8C803E268A2
:104600001FED25CAD2F8E431994292ED7D0AC0F03F
:104610001581022184F8C413C4F8C8030EE100BF59
:104620002046394600F00CFCB0EE490A94ED3EEA13
:104630001FED2CCAB0EE4CDA0EEE4E0A80EE0A8A5E
:10464000B0EEC80AB4EE4B0AF1EE10FA37DCB0EE69
:10465000480A19F0D7FD1AF027FC1FED351AB0EE05
:10466000402A1FED364A28EE013A20EE044A1FED9B
:10467000380A03EE004A02EE410A1FED3A1A31EE03
:10468000433AB0EEC44A20EE000A03EE030A1FEDDF
:104690003E3A24EE033A23EE013AB1EEC01A22EE7E
:1046A000038AB4EE411AF1EE10FA80F135821FED63
:1046B000450A21EE000A2EEE000A88EE00DA94ED9B
:1046C00076EA0EEE4E9A89EE0A8AB0EEC80AB4EE89
:1046D0004B0AF1EE10FA37DCB0EE480A19F092FD01
:1046E0001AF0E2FB1FED581AB0EE402A1FED594AAE
:1046F00028EE013A20EE044A1FED5B0A03EE004A61
:1047000002EE410A1FED5D1A31EE433AB0EEC44AA3
:1047100020EE000A03EE030A1FED613A24EE033A8D
:1047200023EE013AB1EEC01A22EE038AB4EE411A2A
:10473000F1EE10FA80F1F6811FED680A21EE000A11
:104740002EEE000A88EE00CA1DEE100ABBEE048AA7
:104750001CEE101A1FED7A9AF0EE490A20F0004084
:1047600038EE4D1A4045B0EE480A21F0004038EED0
:104770004C2A38BFB0EE410A4045304638BFB0EE53
:10478000428A14F0FDFD04F1AC0104F1B0023046A0
:1047900014F06EFDB0EE480AF0EE490A484614F0F7
:1047A000EFFD04F1B80104F1B402484614F060FDD5
:1047B00097ED010A9FED0F1A20EE010A204684EDC5
:1047C0002F0A97ED010A20EE010A84ED300A00F06D
:1047D00077FF00208DE100BF9FEDE30A042A08EE79
:1047E000000A9FEDD9CA26D8DFE802F0280608148F
:1047F000200000BFCDCC4C3E01E700BFE2689FED3A
:10480000DB0AD2F8E831994292ED7ECA16D3032131
:1048100000E700BFE268D2F8EC3192ED80CA99421D
:1048200092ED7F0A0AD30421F4E600BFE068D0F8D5
:10483000F001814202D3002084F8C40302AF9FED4F
:10484000CB1A0021002230463B4680FE41DA9FED24
:10485000C8EA0025009514F02BFD3B1D0021002225
:104860004846009514F024FDB0EE490AD4ED3E8A86
:104870009FEDB6FA08EEE80A80EE0A8AB0EEC80AA2
:10488000B4EE4B0AB0EE4F0AF1EE10FA37DCB0EEA0
:10489000480A19F0B7FC1AF007FB9FEDAD1AB0EE0D
:1048A000402A9FEDAC4A28EE013A20EE044A9FEDE3
:1048B000AA0A03EE004A02EE410A9FEDA91A31EE60
:1048C000433AB0EEC44A20EE000A03EE030A9FED1D
:1048D000A33A24EE033A23EE013AB1EEC01A22EED7
:1048E000038AB4EE411AF1EE10FA80F121819FEDB6
:1048F0009D0A21EE000A28EE800A88EE000AD4ED17
:10490000768A10EE100A08EEE89A8DFE0E8A20F0E4
:104910000040404589EE0AAA9FED8B9AB0EE49DA35
:1049200038BFB0EE40DAB0EECA1AB4EE4B1AF1EE70
:1049300010FA37DCB0EE4A0A19F064FC1AF0B4FA47
:104940009FED831AB0EE402A9FED824A2AEE013A8B
:1049500020EE044A9FED800A03EE004A02EE410A6F
:104960009FED7F1A31EE433AB0EEC44A20EE000AC2
:1049700003EE030A9FED793A24EE033A23EE013A5F
:10498000B1EEC01A22EE03AAB4EE411AF1EE10FA0B
:1049900080F1D4809FED730A21EE000A28EE800A90
:1049A0008AEE00FA1FEE100AB0EE480AB0EE49BADD
:1049B00020F00040404504F5A26038BFB0EE4FBA89
:1049C000D4ED021A9DED021AD4ED3E0A0FF088FFD5
:1049D0009FED68AAF0EE490A30EE0A0A304630EE42
:1049E0004D0A3CEE000A14F0CBFC18B10020C4E9DB
:1049F0002B0006E004F1AC0104F1B002304614F0E3
:104A000037FCB0EE480A04F24C50D4ED021A9DED8A
:104A1000031AD4ED760A0FF063FF30EE0A0ADFEDD9
:104A20004A0A484630EE4B0A3CEE000A14F0A8FC55
:104A300020B10020C4E92D0007E000BF04F1B80157
:104A400004F1B402484614F013FC9FED4B0A94EDB8
:104A50002B1AB0EE403AB4EE401AF1EE10FA08DB31
:104A6000B0EE4A3AB4EE4A1AF1EE10FA01DCB0EEBA
:104A7000413AB0EE401A94ED2C2AB4EE402A84ED6F
:104A80002B3AF1EE10FA08DB9FED3A1AB4EE412A08
:104A9000F1EE10FA01DCB0EE421A84ED2C1AB0EE01
:104AA000401A94ED2D2AB4EE402AF1EE10FA08DBFC
:104AB0009FED301AB4EE412AF1EE10FA01DCB0EEAF
:104AC000421A94ED2E2A84ED2D1AB4EE402AF1EE0E
:104AD00010FA08DB9FED270AB4EE402AF1EE10FA37
:104AE00001DCB0EE420A204684ED2E0A00F0E8FD1B
:104AF000002040B204B0BDEC108B01B0BDE8F083E3
:104B00001AF09AFAB0EE401A56E400BF1AF094FA7E
:104B1000B0EE401A97E400BF1AF08EFAB0EE401AD9
:104B2000C5E500BF1AF088FAB0EE401A04E600BFEF
:104B30001AF082FAB0EE401AD9E600BF1AF07CFAF9
:104B4000B0EE401A26E700BF000000000000C07F62
:104B5000CDCC4C3DC52030BC31082C3D0000B443C9
:104B6000F6285C3E4A0C823E0AD7233E0AD7A33E73
:104B70008FC2F53D00007042000070C200000000CE
:104B8000F0B581B02DED028BFF2600281CBF0D462D
:104B9000002905D170B2BDEC028B01B0F0BD00BFA1
:104BA000B0EE408AB5EE400AF1EE10FAF2DD0446AE
:104BB000C56000202075FDF7FBFF0DF051FDE0689A
:104BC0000DF06EFEC0B9E06806300DF069FE98B9D0
:104BD000E0680C300DF064FE70B9E06812300DF042
:104BE0005FFE48B9E06818300DF09AFA20B9E06825
:104BF0001E300DF095FA28B1FF2670B2BDEC028B85
:104C000001B0F0BDE06824300DF066F8B0EE480A5F
:104C100004F1C40005F12C0114F06AFBB0EE480A5F
:104C200004F5D27005F1480114F062FBB0EE480AB9
:104C300005F5D27704F5A26001213A4604F57976AC
:104C40000FF0FEFEB0EE480A04F24C5001213A4645
:104C50000FF0F6FEB0EE480A05F5927201213046DB
:104C60000FF0EEFEB0EE480A04F5846005F5A2727E
:104C700001210FF0E5FEB0EE480A04F25C4005F5B4
:104C8000B27201210FF0DCFEB0EE480A05F5C276E3
:104C900004F59360012132460FF0D2FEB0EE480ACF
:104CA00004F2D440012132460FF0CAFE05F1640639
:104CB00004F5217031460CF057FD04F5447031467F
:104CC0000CF052FDB0EE480A04F5C060D5ED8B0A39
:104CD0000CF03EFEB0EE480A04F5C460D5ED8B0A38
:104CE0000CF036FEB0EE480A04F5C860D5ED8B0A2C
:104CF0000CF02EFEB0EE480A04F5CC60D5ED8B0A20
:104D00000CF026FEB0EE480A04F5D060D5ED8B0A13
:104D10000CF01EFEB0EE480A04F5D460D5ED8B0A07
:104D20000CF016FEF3EE0E0AB0EE480A04F5D86059
:104D30000CF00EFE04F5DC600221002202230026A6
:104D40000CF016F84FF6E031D4F8D807C0F60101A0
:104D5000B7EE000A4FF07E55D1F800C0C0F800C091
:104D60004B6843608F688760C968C160D4F8E0070A
:104D700080EE080A056080ED010AC0E902654FF681
:104D8000D035D4F8F407C0F601052A6802606A68D5
:104D90004260AA688260EA68C260D4F800074DF2F7
:104DA0000A724CF6CD45C3F6A332C3F6CC55C0E922
:104DB0000025D4F8EC0784F8EF66C0E900C3C0E929
:104DC00002714FF6F031D4F8F807C0F601010A6815
:104DD00002604A6842608A688260C968C160E068AF
:104DE0000DF0C2FBE06806300DF0BEFBE0680C3051
:104DF0000DF0BAFBE06812300DF0B6FBE068183039
:104E00000DF06EF9E0681E300DF06AF904F5677078
:104E10002A21C4F8C863FCF7B4F8E068D0F8F411AC
:104E2000C4F8CC13D0F8F811C4F8D013D0F8FC01B2
:104E3000C4F8D40370B2BDEC028B01B0F0BD000029
:104E40002DE9F04381B02DED108B90B00446002881
:104E50004FF0FE0000F002848846002900F0FE8337
:104E600098ED010A94ED021A30EE000A94EDEA2A58
:104E700084EDEB0A04F5217684EDEC0A0AAF00EE2E
:104E8000012A94ED250AD4F800010A90D4F804010F
:104E90000B90D4F89C030C90D4F8A0030D90D4F898
:104EA000A4000E90B1EE400A3046394684EDEA2A5D
:104EB0008DED0F0A0CF0D0FC04F54475D4E97801AF
:104EC000CDE90A01284639460CF0C6FC94ED3E0AAD
:104ED00030460CF0FDFA94ED760A28460CF0F8FA0C
:104EE000D4F8A803069098F80000002798ED020A6D
:104EF000D4F8AC1303280997CDE90477CDE9071757
:104F000020D1B5EE400AF1EE10FA1BD094F87801EA
:104F100000285CD004A930460CF052FC30460CF05E
:104F2000CFFB94F8580200286DD004A928460CF055
:104F300047FC28460CF0C4FB94EDD70A94EDEF1A19
:104F40007DE000BF9FEDC11AE06820EE010AD4EDBC
:104F50001E0AC4EDEE0A9FEDBE2A90ED861A9FED63
:104F6000BDAA31EE022A30EE018AB0EE4A1A30EEC6
:104F7000029AB0EE480A00F07BFEB0EE40BAB0EE06
:104F8000490AB0EE4A1AD4EDEE0A00F071FEB0EE16
:104F9000CB1A04F57970B0EEC00AB4EE401A9FED5A
:104FA000AE1AF1EE10FAC8BF012739FE080AD4ED97
:104FB000021AD4ED1E0A84EDED0A84F8C0730FF0D6
:104FC0008FFC84EDEF0A94F878010028A2D104A99F
:104FD0003046002704970CF0F3FB94ED410A94ED62
:104FE000BE1A20EE410A94ED401A94EDBD2AC4F891
:104FF000D072C4F8BC7302EE410A84EDB50A94F88D
:105000005802002891D104A92846002604960CF0E5
:10501000D7FB94ED790A94EDE02A94EDE11AC4F8F7
:105020005C6320EE410A94ED781AC4F8BC6302EE8A
:10503000410A84EDD80A9FED880AB0EE401AB1EE1D
:10504000022A94EDB43AE06894ED2AAA83EE023A7B
:1050500080EE020A33EE012A30EE410AB6EE001A63
:1050600084ED2F2A84ED300A90ED850A20EE01CAE6
:1050700094ED760A94ED3E1A30EE41DAB0EE4A0A2B
:1050800019F008FDB0EE408AB0EE4A0A3CEE0CEA98
:1050900019F00AFFB0EE409AB0EE4A0A19F004FF88
:1050A000B0EE40BAB0EE4A0A19F0F4FC2EEE003A27
:1050B0009FEDD82A9FED680A0DEE4B3AB0EEC31A69
:1050C000B4EE421AB0EE401AB0EE402AF1EE10FAF9
:1050D00009DD2EEE091A0DEE081A81EE031A2CEEE8
:1050E000412A2CEE011A94F8780104F1C40604F563
:1050F000D27940B194F858020FF28C51002808BFC1
:10510000043191ED000AB1EE403A9FED539A82FED0
:10511000404A04F25C4081FE400AD4ED021AB4EE2B
:10512000423AD4ED2A0AF1EE10FAB4EE413A94ED87
:10513000251A33FE04AAF1EE10FA33FE00BAB0EEDF
:10514000490A0FF0CDFBB0EE408A98ED04CAFEF795
:10515000EBFD4FF47A720023FBF7A7F994F8C5131F
:10516000D4F8C83394F8C4230029A0EB03010FD06E
:1051700072B90122A4F8C423C4F8C803E268D2F8C3
:10518000E4319942D2ED7D8A18D2B0EE680A69E026
:10519000042A2CD8DFE802F02E04061A260000BFED
:1051A000ECE700BFE268DFED9C8AD2F8E831994273
:1051B00092ED7E9AE9D3032101E000BF022184F839
:1051C000C413B0EE680AC4F8C8034BE0E268D2F832
:1051D000EC3192ED809A9942D2ED7F8AD5D30421A9
:1051E000EDE700BFE068D0F8F001814202D3002073
:1051F00084F8C4039FED890A0CEE000A3AEE001A07
:105200003BEE002AB4EE421AF1EE10FA0CDA9FEDF2
:10521000840AB4EE401AF1EE10FA1FDA30EE411AA9
:1052200072EE018A1EE000BFB4EE412AF1EE10FAE0
:1052300014DADFED7B8AB4EE682AF1EE10FA0DDAAB
:1052400038EEC20A31EE000A0CE000BFDB0FC93FA6
:10525000DB0F4940DB0FC94000000000F0EE428A3E
:10526000B0EE410ADFED6CCA02AF80FE6C0ADFEDE2
:105270006C9A0021002230463B4680FE29CA002558
:10528000009514F015F83B1D0021002248460095BA
:1052900014F00EF8D4ED021A94ED411AD4ED400A40
:1052A00004F5936094ED780AD4ED3EDA0FF018FB24
:1052B000B0EE40BAD4ED021A94ED400A94ED791A9A
:1052C000D4ED780A04F2D44094ED76FA0FF008FB9E
:1052D000B0EE40AAB0EE4C0A04F5A260D4ED021A7A
:1052E000D4ED3E0A9DED021A0FF0FAFADFEDE8AABE
:1052F000D4ED3EEAB0EE6A1ADFEDE6BAB7EE00EAA8
:10530000B0EE40CA0EEEEE1A81EE2BDAB0EECD1AF8
:10531000B4EE4E1AF1EE10FA02DD9FEDDF0A37E02F
:10532000B0EE4D0A18F06EFF19F0BEFD9FEDDB1ACE
:10533000B0EE402A9FEDDA4A2DEE013A20EE044A03
:105340009FEDD80A03EE004A02EE410A9FEDD71AFC
:1053500031EE433AB0EEC44A20EE000A03EE030AEF
:105360009FEDD13A24EE033A23EE013AB1EEC01A92
:1053700022EE03DAB4EE411AF1EE10FA80F17681F2
:105380009FEDCB0A21EE000A2EEE800A8DEE000A78
:1053900094F8C403B2EE04DAC8FEEC8A012701389F
:1053A000C7F68077022807D839EE0C0A0020C4E936
:1053B0002F00DFEDB40A23E010EE100A2DEE8D1A57
:1053C000DFEDB0CA20F0004021EE0BBAB84238BF82
:1053D000F0EE40CA94ED400AD4EDB5DA19F064FD60
:1053E0000DEE80CA9FEDB30A94EDB51A7BEE010A6B
:1053F0003CEE000A30EE6C0A39EE000A38EE000A84
:10540000304688FEA9BA13F0BBFF58B10020C4E9AA
:105410002B000EE06F12833A0AD7A33E0AD7233E31
:105420008FC2F53D04F1AC0104F1B002304613F037
:105430001FFFB0EE4B0A04F24C50D4ED021A9DED62
:10544000031AD4ED760A0FF04BFAD4ED768AB0EE5B
:1054500040BA48EEE8AA8AEEABCAB0EECC1AB4EE77
:105460004E1AF1EE10FA33DD9FED8B0A94F8C40367
:105470000138022869D910EE100A2FEE0D1A9FED9F
:1054800081CA20F0004021EE0AAAB84238BFB0EE2F
:1054900040CA94ED780A94EDD8DA19F005FD0DEEC6
:1054A00000BA9FED840A94EDD81A7AEE010A3BEE19
:1054B000000A30EE4C0A39EE000A30EE480A48463F
:1054C00013F05EFF002849D00020C4E92D004CE015
:1054D000B0EE4C0A18F096FE19F0E6FC9FED6F1A3C
:1054E000B0EE402A9FED6E4A2CEE013A20EE044ABF
:1054F0009FED6C0A03EE004A02EE410A9FED6B1A23
:1055000031EE433AB0EEC44A20EE000A03EE030A3D
:105510009FED653A24EE033A23EE013AB1EEC01A4C
:1055200022EE03CAB4EE411AF1EE10FA80F1A48023
:105530009FED5F0A21EE000A28EE800A8CEE000A39
:1055400094F8C4030138022895D839EE0B0ADFED30
:105550004D0A484613F014FF0028B5D104F1B801F4
:1055600004F1B402484613F083FEBFEE001A94ED36
:105570002F0AB0EE412AB4EE410AF1EE10FA08DB30
:10558000B0EE4E2AB4EE4E0AF1EE10FA01DCB0EEA7
:10559000402A94ED300A84ED2F2AB4EE410AF1EE50
:1055A00010FA08DBB7EE001AB4EE410AF1EE10FA79
:1055B00001DCB0EE401A9FED400A84ED301AB0EEE7
:1055C000401A94ED2B2AB4EE402AF1EE10FA08DBD3
:1055D0009FED381AB4EE412AF1EE10FA01DCB0EE7C
:1055E000421A84ED2B1AB0EE401A94ED2C2AB4EE38
:1055F000402AF1EE10FA08DB9FED2E1AB4EE412A94
:10560000F1EE10FA01DCB0EE421A84ED2C1AB0EE85
:10561000401A94ED2D2AB4EE402AF1EE10FA08DB80
:105620009FED241AB4EE412AF1EE10FA01DCB0EE3F
:10563000421A94ED2E2A84ED2D1AB4EE402AF1EE92
:1056400010FA08DB9FED1B0AB4EE402AF1EE10FAC7
:1056500001DCB0EE420A002084ED2E0A40B210B008
:10566000BDEC108B01B0BDE8F08300BF19F0E4FC85
:10567000B0EE401A84E600BF19F0DEFCB0EE401A2E
:1056800056E700BF000000008FC2F53D000000009B
:105690002ECCE23DBDAEDF3D0000C07FCDCC4C3D09
:1056A000C52030BC31082C3D0000B443F6285C3ED8
:1056B0004A0C823E00007042000070C200000000F0
:1056C000002808BF7047B0B586B0044601AD002081
:1056D000CDE90300CDE90100E068D4F8AC100591F4
:1056E00029460CF0C9FFE068D4F8B01005910630E7
:1056F00029460CF0C1FFE068D4F8B41005910C30D5
:1057000029460CF0B9FFE068D4F8B81005911230C2
:1057100029460CF0B1FFE068183094ED2F0A0CF028
:105720008FFDE06894ED300A1E300CF089FD06B064
:10573000BDE8B0407047000010B52DED108B00287B
:1057400000F09E8104460DF0A3FA0CF0B1FEE06873
:105750000CF02EFF40B100F11C0304F1180C806A1C
:105760000ECB8CE80E00606294ED060A9FEDCA8AAB
:1057700030EE081A9FEDC99AB4EE490AE068F1EEDE
:1057800010FA31FE000AB1EE400A84ED060A90EDEF
:10579000811A063030EE410A84ED060A0CF008FF4B
:1057A00040B100F11C0304F1280C806A0ECB8CE898
:1057B0000E00606394ED0A0AE06830EE081AB4EE59
:1057C000490AF1EE10FA31FE000AB1EE400A84ED0A
:1057D0000A0A90ED821A0C3030EE410A84ED0A0A72
:1057E0000CF0E6FE40B100F11C0304F1380C806AB5
:1057F0000ECB8CE80E00606494ED0E0AE06830EE8B
:10580000081AB4EE490AF1EE10FA31FE000AB1EEC0
:10581000400A84ED0E0A90ED831A123030EE410AF0
:1058200084ED0E0A0CF0C4FE40B100F11C0304F13B
:10583000480C806A0ECB8CE80E00606594ED120A6D
:10584000E06830EE081AB4EE490AF1EE10FA31FEC3
:10585000000AB1EE400A84ED120A90ED841A183065
:1058600030EE410A84ED120A0CF0F2FB40B100F177
:105870001C0304F1580C806A0ECB8CE80E006066A5
:10588000E0681E300CF0E4FB40B100F11C0304F1B1
:10589000680C806A0ECB8CE80E00606794ED0B0AF2
:1058A0009FED7F1A94ED0F2A20EE010A22EE012AC5
:1058B00094ED173A94ED1B4A03EE010A04EE012A17
:1058C00094ED261A30EE418A94ED3E0A32EE419A6A
:1058D00094ED411A20EE01AA94ED400A19F0DAF88D
:1058E0002AEE00AA9FED6FBA94ED400A08EE0BAACB
:1058F00094ED3F8A19F0D8FA08EE00AA94ED760AE2
:1059000094ED791A20EE018A94ED780A19F0C2F824
:1059100028EE008A94ED780A09EE0B8A94ED779AC6
:1059200019F0C2FA09EE008AB6EE001AD4F8A00304
:10593000C4F8A40394ED22EA94ED23FA94ED24DA5A
:1059400094ED2A9A3AEE080A94ED298A20EE01CACB
:10595000B0EE480A19F0A8FAB0EE40AAB0EE490A33
:1059600019F0A2FADFED508A60EE289AB0EE480AEC
:1059700019F090F8B0EE40BAB0EE490A19F08AF882
:1059800060EE28AAB0EE480A19F084F80AEEC0DAF0
:10599000B0EE480A0AEE28EA09EECBFA19F07AF8D6
:1059A000B0EE40AAB0EE490A19F07EFAB0EE40BA65
:1059B000B0EE480A19F078FA2BEE000A2FEE00BA82
:1059C000B0EE490A0EEE0ABA19F064F8B0EE409A49
:1059D000B0EE480A19F068FA29EE000A94ED021AAE
:1059E0009FED322AD4F8E007B4EE421A9FED302A38
:1059F000F1EE10FA0DEE00BAB5EE401A32FE018A51
:105A00000022F1EE10FAD8BFB0EE428A8260D4F8DC
:105A1000E426B3EE040A4FF07E51016080ED018A66
:105A2000C16004F5DC6082ED00CA82ED01BA94ED3C
:105A30005D1AB4EE401AF1EE10FA09DA94ED951AF7
:105A4000B4EE401AF1EE10FA02DA9FED1A0A01E004
:105A50009FED190AD4F8F81781ED000A0BF0ECFB62
:105A6000A0B190ED000A94EDE71A08EE001A0020AC
:105A700084EDE80A84EDE71A40B2BDEC108B10BD4E
:105A8000FE2040B2BDEC108B10BD00BF002040B224
:105A9000BDEC108B10BD00BFDB0FC9C0DB0F494050
:105AA00035FA8E3C96438B3DC3F51C41CDCCCC3DA5
:105AB0006F12833A0050C3470000C8420000000044
:105AC00090ED001AF5EE400A31EE000AF1EE10FA00
:105AD0000BDDB4EE600AF1EE10FA09DAB5EE400A19
:105AE000F1EE10FA01DA30EE200A80ED000A70477C
:105AF00030EE600A80ED000A7047000000000000F0
:105B000010B52DED088B002844D030EEC11AB0EE50
:105B1000429A9FED262A04469FED253AB0EE628A0E
:105B200031EE022AB4EE431A9FED233AF1EE10FA59
:105B300032FE011A9FED1F2A31EE022AB4EE413ADD
:105B4000F1EE10FA32FE011A31EE000A90ED001A61
:105B500030EE01AAB0EE610AB0EE621AF0EE4A0A27
:105B600000F086F8B0EE40BAB0EE490AF0EE4A0A0C
:105B7000B0EE481A00F07CF894ED002A82FE4B1A31
:105B8000B4EE4B2AF1EE10FA08DCB4EE401AF1EE56
:105B900010FA03DBBDEC088B10BD00BF81FE000ACC
:105BA00084ED000ABDEC088B10BD00BFDB0FC9C03F
:105BB000DB0F4940DB0FC940DB0F49C0000000008C
:105BC00010B52DED0A8B002846D030EE600AB0EEFD
:105BD00041AA9FED231AB0EE429A9FED222A044675
:105BE00030EE011AF0EE4A0AB4EE420A9FED1F2A87
:105BF000F1EE10FAB0EE618A31FE000A9FED1A1A3A
:105C000030EE011AB4EE402AF1EE10FA31FE00CA6D
:105C100090ED000AB0EE491A3CEE00BAB0EE4B0A25
:105C200000F026F8B5EE400AF1EE10FA03DD3AEE88
:105C30004C0A84ED000AB0EE4B0AF0EE480AB0EED2
:105C4000491A00F015F8B5EE400AF1EE10FA03DA41
:105C500038EE4C0A84ED000ABDEC0A8B10BD00BF83
:105C6000DB0FC9C0DB0F4940DB0FC940DB0F49C068
:105C700030EE600AB5EE401AF1EE10FA16DDB6EE1F
:105C8000002A21EE022AB4EE420AF1EE10FA03DDF8
:105C900030EE410A704700BFB1EE422AB4EE420A2C
:105CA000F1EE10FAA8BF704730EE010A704700000D
:105CB00080B502A20DF098FF002080BD4369616CA1
:105CC0006C6FEFBD9E28E288A0E383BBCF893C20A8
:105CD00029E28C92E298850D0A0000000000000085
:105CE00040F63850C2F2004070470000000000004B
:105CF00042F22010C2F2004002F0F6BC00000000A8
:105D000042F21020C2F2004002F0EEBC000000009F
:105D100042F28820C2F2004002F0E6BC000000001F
:105D200042F20030C2F2004002F0DEBC000000008F
:105D300042F2F030C2F2004002F0D6BC0000000097
:105D400042F27830C2F2004002F0CEBC0000000007
:105D500040F20F42D0F800C0C4F20202944511DCB8
:105D60006F22C4F20202944522DC3F22C4F20202F6
:105D7000944539DC1022C4F2020294455AD02822FC
:105D800054E000BF40F26F42C4F2020294451BDCB3
:105D900040F23F42C4F2020294452DDC40F2104230
:105DA000C4F20202944545D040F228423EE000BFD2
:105DB0009F22C4F20202944528DC7022C4F202023F
:105DC000944537D0882231E040F29F42C4F202026B
:105DD000944523DC40F27042C4F20202944529D07B
:105DE00040F2884222E000BF4022C4F20202944501
:105DF00020D058221AE000BF40F24042C4F2020212
:105E0000944517D040F2584210E000BFA022C4F2DF
:105E1000020294450ED0B82208E000BF40F2B8421A
:105E2000C4F20202944505D040F2A042C4F202023C
:105E3000944519D16FF00F024AF6AB2352FA8CF257
:105E4000CAF6AA23A2FB03310AA35F2AC1F30211F7
:105E50005B5C40F2FF312CEA0101C36588BF04316D
:105E600081650846704700BF2CF0FF018165084638
:105E7000704700BF00061016000610160000000054
:105E800070B540F26F44D0F800C0C4F20204D0F8FC
:105E900058E0A4451ADC9F25C4F20205AC4533DC6A
:105EA0005725C4F20205AC455ADC1025C4F20205A0
:105EB000AC4500F098802825C4F20205AC4500F0FE
:105EC00092804025C4F202058AE000BF45F22F45CA
:105ED000C5F60205AC452DDC40F2B745C4F202051B
:105EE000AC454BDC40F27045C4F20205AC457AD0BB
:105EF00040F28845C4F20205AC4574D040F2A0459A
:105F0000C4F202056CE000BF40F22745C4F202056E
:105F1000AC4543DCA025C4F20205AC4563D0B825EE
:105F2000C4F20205AC455ED040F21045C4F2020551
:105F300056E000BF45F26B45C5F60205AC453FDCB7
:105F400045F23045C5F60205AC454CD045F2444516
:105F5000C5F60205AC4546D045F258453EE000BFC7
:105F60005825C4F20205AC453DD07025C4F20205A7
:105F7000AC4538D08825C4F2020531E040F2B8457E
:105F8000C4F20205AC452ED045F20845C5F602051F
:105F9000AC4528D045F21C4520E000BF40F2284522
:105FA000C4F20205AC451ED040F24045C4F20205E1
:105FB000AC4518D040F25845C4F2020510E000BFCD
:105FC00045F26C45C5F60205AC450CD045F294454A
:105FD000C5F60205AC4506D045F28045C5F602057A
:105FE000AC4540F0D580456EC66E002E866E6E6064
:105FF0001CBFD0E91C566E60A44515DC9F24C4F27A
:106000000204A4452CDC5724C4F20204A44551DC4C
:106010001024C4F20204A4457AD02824C4F2020455
:10602000A44575D040246FE045F22F44C5F6020424
:10603000A44529DC40F2B744C4F20204A44545DC7F
:1060400040F27044C4F20204A44561D040F2884496
:10605000C4F20204A4455BD040F2A04454E000BF67
:1060600040F22744C4F20204A4453FDCA024C4F259
:106070000204A4454CD0B824C4F20204A44547D07D
:1060800040F2104440E000BF45F26B44C5F6020404
:10609000A44555DC45F23044C5F60204A44561D060
:1060A00045F24444C5F60204A4455BD045F2584489
:1060B00054E000BF5824C4F20204A44528D0702440
:1060C000C4F20204A44523D088241DE040F2B84461
:1060D000C4F20204A4451BD045F20844C5F60204EC
:1060E000A4453FD045F21C4438E000BF40F22844AC
:1060F000C4F20204A4450BD040F24044C4F20204AE
:10610000A44505D040F25844C4F20204A4453FD14E
:106110008468C06D00F01F003F2505FA00F0CEF83E
:106120000800DCF80000402C20F48020CCF80000AF
:10613000CCF8043023D0CCF80810CCF80C2070BD7B
:1061400045F26C44C5F60204A4450BD045F28044E8
:10615000C5F60204A44505D045F29444C5F60204F0
:10616000A44515D1C46D806804F01F0401254028A2
:1061700005FA04F4CEF80440CCF8043004D1CCF88D
:106180000820CCF80C1070BDCCF80810CCF80C200E
:1061900070BD000000000000B0B5D8B141F2AC24E1
:1061A000C2F20044207818B1FD2568B2B0BD00BF2E
:1061B00014F0B6FC606068B146F2F9320020C0F617
:1061C000000203210025FDF733FE0120207068B294
:1061D000B0BD00BFFE2568B2B0BD000000000000E9
:1061E00010B538B13421002400F8244BFAF7C9FE69
:1061F00060B210BDFE2460B210BD000000000000BF
:10620000B0B508B30546044655F8100F01466FF3C4
:10621000DF21A1F5B671B1F5A56F11D8C0F3CA2180
:10622000A1F5B671B1F5A56F0AD8A988800D40EA2D
:1062300081206FF3DF20A0F5B670B0F5A56F07D908
:10624000FF2040B2B0BD00BFFE2040B2B0BD00BFD5
:1062500011F4405F4FF0FF0000F0C5808AB2B2F544
:10626000804FC0F0C080C1F34A01A1F5B671B1F50D
:10627000A56F00F2B88001202070FDF755FD2A6857
:1062800094F81CC013466FF3DF23BCF1000F00EE3F
:10629000103AA369C4E90201C2F3CA20A988B8EE82
:1062A000401A9FED520AE36331EE001A31EE012AE3
:1062B00001EE100A4FEA925040EA81206FF3DF208E
:1062C000B8EE413A04EE100A9FED491AC1F34A00B4
:1062D00082EE012A05EE100A33EE003AB8EE444A87
:1062E00084ED0B2A4FEA913284F83920B8EE455AF2
:1062F000E28A34EE004A4FF0000033EE033A606564
:10630000C1F3013135EE005A34EE044A84F83810F6
:1063100083EE013A628735EE052A84ED0C3A84EE6D
:10632000013A627F84ED093A82EE012A84ED0A2A5D
:1063300018BF4FF0010C002A84F840C018BF01229A
:10634000E38B84F852C084F84120DDB203F00101F0
:1063500084F84210C5F3400184F84310C5F380016E
:1063600084F84410C5F3C00184F84510C5F300114A
:1063700084F84610C5F3401184F84710C5F3801126
:1063800084F84810E90984F84910C3F3002184F81F
:106390004A10C3F3402184F84B10C3F38025218CAD
:1063A00084F84C5002EE101A84F85320C3F3C02135
:1063B00084F84D10C3F3003184F84E10C3F340311C
:1063C000B8EE422A84F84F10C3F3803184F850109D
:1063D00032EE000AD90B84F8511030EE000A80EE3C
:1063E000010A84ED0D0A40B2B0BD00BF000080C4B8
:1063F0000000A5440000000041F2AC200121C2F2DF
:106400000040406814F094BA10B504460020FDF72F
:10641000B3FC04F1100112220AF042F9002818BF5F
:106420004FF0FF3010BD000080B502460120012171
:1064300014F0C2FA0138B0FA80F0400980BD0000C3
:10644000704700000000000080B54FF4806004F049
:1064500023FB4FF48050BDE8804004F01DBB0000DA
:10646000EFF3108072B600BFFEE7000000000000EE
:1064700044F60400C5F60200816841F00201816023
:106480000168890409D4016889045CBF01685FEA76
:10649000814102D401688904F2D5704700000000F0
:1064A00042F26840C2F2004003F026BD0000000046
:1064B00042F26840C2F2004003F01EBD000000003E
:1064C00042F20850C2F2004003F016BD0000000086
:1064D00042F20850C2F2004003F00EBD000000007E
:1064E00042F2A850C2F2004003F006BD00000000D6
:1064F00042F2A850C2F2004003F0FEBC00000000CF
:1065000010B54FF0000CC2F800C08C4500F086803A
:10651000047844F02003202B28D0447844F0200352
:10652000202B11D0847844F02003202B14D0C47881
:1065300044F02003202B17D00430047844F02003CB
:10654000202BEAD112E000BF01305FFA84FEBEF1D9
:10655000200F10D01FE000BF02305FFA84FEBEF1B2
:10656000200F08D017E000BF033000BF5FFA84FEA1
:10657000BEF1200F0FD14478202C11D18478202C2B
:1065800016D1C478202C1BD110F8044F5FFA84FE7A
:10659000BEF1200FEFD0BEF1000F3FD00AE000BFE8
:1065A000E4B301300CF1010C8C45AED10EE000BF1C
:1065B000A4B302300CF1010C8C45A6D106E000BF5B
:1065C00064B303300CF1010C8C459ED1022144F0E0
:1065D0002003DBB2202B1ED043184C1E146013F88E
:1065E000014C44F02004202C1AD01160445C44F08B
:1065F0002004202C16D04C1C14605C7844F020043D
:10660000202C11D08C1C14609C78043144F02003A1
:10661000DBB2202BE0D1023907E000BF002010BD23
:10662000012102E0012100E00121002908BF084604
:1066300010BD0000000000002DE9F04741F2DC4AE7
:106640009046C2F2004A89460646DAF800307BB12D
:106650001C68A3684846414632469847002818BF40
:10666000BDE8F0870020CAF80000BDE8F08700BF51
:1066700041F2D805C2F20045CAF8005005E000BF5B
:106680006D68CAF80050002D61D02C682768384624
:10669000FAF764FB0246305C40F020002028EFD17E
:1066A00030463946FAF779FB0028E9D194F90CC055
:1066B000BCF1000FCDD40021334600221F78202FDB
:1066C00006D119E03944012204331F78202F13D05A
:1066D00087B3002201275878202817D050B3002212
:1066E00001279878202817D020B300220127D878D6
:1066F000202817D1E6E700BF012A4FF001024FF032
:10670000000718BF013158782028E7D13944012209
:10671000002798782028E7D1394401220027D8782B
:106720002028CFD030B1002204331F78202FCFD1C2
:10673000E2E700BF012A08BF0139C8B25FFA8CF155
:10674000884218BF002D0DD1002D7FF482AF4FF687
:10675000BD414846C0F601014246FAF739FC002027
:10676000BDE8F0874FF665414846C0F60101424654
:10677000FAF72EFC76E70000B0B5A8B10446082071
:1067800014F0E6FFD0B1054615F0C6FC40F2140047
:106790002C60C2F2004000226A60016805604D6012
:1067A00015F0E2FC0120B0BD4FF0500080F31188DD
:1067B000BFF36F8FBFF34F8FFEE700BF4FF0500066
:1067C00080F31188BFF36F8FBFF34F8FFEE7000098
:1067D00070B54FF0FE0608B30C46F9B158210546D6
:1067E000FAF7CFFB20890A222883002620686168F7
:1067F0006961286120782E706188FCF7D9FA2078C9
:10680000A1880A22FCF7D4FA2078E1880A22FCF752
:10681000CFFA20780A222189FCF7CAFA70B270BD3B
:10682000B0B5002818BF002A00D1B0BD438A8B4202
:1068300046D192F800C015795378547991789FED3C
:106840009A2A5B0192F803E043EA4C339FED904AA9
:1068500043EAD10C4FEA8E2300EE10CA61F3944351
:1068600043EA85019379D27941EA9411DB0101EE83
:10687000101A64F3D433B8EE400A43EA520203EE2E
:10688000102AB8EE411A20EE020AB8EE433A21EE81
:10689000021A80EE040A23EE022A9FED843A81EE6A
:1068A000041A30EE030A82EE042A80ED070A31EE64
:1068B000031A80ED081A32EE030A80ED090AB0BD12
:1068C000838A8B4244D111789FED752A53789FEDCE
:1068D000704A9578D4785B0143EA41311379A40278
:1068E00041EAD50C517965F394449579D27944EA1B
:1068F0008303ED0100EE10CA61F3D43543EA91132E
:1069000045EA520101EE103A03EE101AB8EE400AC1
:10691000B8EE411AB8EE433A20EE020A21EE021A0E
:1069200023EE022A9FED5F3A80EE040A81EE041AFC
:1069300082EE042A30EE030A31EE031A80ED0A0AD1
:1069400032EE030A80ED0B1A80ED0C0AB0BD00BFD9
:10695000C38A8B4248D111789FED4C2A53789578A1
:10696000D4785B0143EA41311379A40241EAD50CA2
:10697000517965F394449579D27944EA8303ED0122
:1069800000EE10CA43EA911361F3D43501EE103AD8
:1069900045EA5201B8EE400A03EE101AB8EE411A69
:1069A00020EE020A9FED3C2AB8EE433A21EE021A8D
:1069B00023EE022A9FED363A80EE030A81EE031A97
:1069C00082EE032A9FED333A30EE030A9FED333A0D
:1069D00080ED0E0A31EE030A80ED0D0A32EE030A55
:1069E00080ED0F0AB0BD00BF038B8B4218BFB0BD56
:1069F00051789FED251A9378BFEE005AD4789D0800
:106A000045EA8111157900EE101A210163F30D3169
:106A10005379947941EA15119B00D27965F38D235E
:106A200002EE101A43EA9413B8EE400A64F30D2202
:106A300003EE103A04EE102AB8EE422A30EE000AB5
:106A4000B8EE433AB8EE444A32EE022A33EE033A45
:106A500080EE010A34EE044A82EE012A83EE013A06
:106A600084EE011A30EE050A80ED100A32EE050AB6
:106A700080ED110A33EE050A80ED120A31EE050AA7
:106A800080ED130AB0BD00BF00FC7F460000344318
:106A9000F8FFFF490000B4C20000B443000034C353
:106AA0001F858B421F850BC23333EB4233336BC2DE
:106AB000002869D0F0B595B00446007C6D460023EF
:106AC000618A2A46FCF718F8B0FA80F14FEA5117AC
:106AD00078B905F10D0600BF618A20463246FFF7FE
:106AE0009FFE207C0023618A2A46FCF705F80028D7
:106AF000F2D0207CA18A6D4600232A46FBF7FCFFDA
:106B000080B905F10D0600BFA18A20463246FFF785
:106B100087FE207CA18A00232A46FBF7EDFF002890
:106B2000F2D00127207CE18A6D4600232A46FBF73C
:106B3000E3FF78B905F10D06E18A20463246FFF7FA
:106B40006FFE207CE18A00232A46FBF7D5FF002850
:106B5000F2D00127207C6D46218B00232A46FBF7CB
:106B6000CBFFA8B11FBBFDF7DFF8D4E90223801AE1
:106B700048F2A162C0F201029941801A71F100004D
:106B80001BD30020207018E0FE2040B2704700BFE9
:106B900005F10D06218B20463246FFF741FE207C91
:106BA0000023218B2A46FBF7A7FF0028F2D0012003
:106BB0002070FDF7B9F8C4E90201002015B0BDE866
:106BC000F04040B2704700002DE9F0412DED028BFE
:106BD00082B0044600284FF0FF0000F039810E46D5
:106BE000002900F035819046FDF79EF8D4E9002396
:106BF000801A994118F062FD00EE100A9FED971A75
:106C000080EE010A84ED020AFDF78EF83778257CC4
:106C1000C4E90001BD423DD004F17C000DF05CFFF1
:106C200004F1B8000DF058FF04F1F4000DF054FF2A
:106C300004F598700DF050FF9FED898A04F5BE7041
:106C4000B0EE480A0AF0DCFEB0EE480A04F5CE7059
:106C50000AF0D6FEE06808300AF00AFF04F170007E
:106C6000FBF79AF8012F08BF002D03D094ED730AAB
:106C70000AE000BF94ED5D0A94ED5E1A30EE010A61
:106C8000B6EE001A20EE010A84ED1D0AD4F8C40104
:106C90002067277496ED010A94ED021A20EE010A8E
:106CA000B7EE081AE06890ED2B2A20EE010AB5EE47
:106CB000402A8DED010AF1EE10FA10DDD4ED7A0ACA
:106CC000D4ED5B1A94ED1C0A94ED711A94ED5C2AD4
:106CD00001A8DFED642AFEF713FF9DED010A04F120
:106CE0007007DFED600A3846FEF7EAFEE06896EDD1
:106CF000020A94ED021A90ED2C2A20EE010AB5EE5C
:106D0000402A8DED000AF1EE10FA10DDD4ED7E0A76
:106D100094ED1D0AD4ED5D1A94ED5E2A94ED731A7C
:106D20006846DFED502AFEF7EBFE9DED000A04F108
:106D30007406DFED4C0A3046FEF7C2FE207C411E91
:106D4000022942D3032807D0002870D10020C4F8BC
:106D5000BC019FED430A68E0B8F1000F35D098F808
:106D6000000090B3E068D8F80410216790ED2B1A6A
:106D700098ED020AB5EE401AB1EE400AF1EE10FAB3
:106D800084ED1D0A0DDD94ED5B1AD4ED5C1AD4ED93
:106D9000710A94ED7A0A9FED332A3846FEF710FF08
:106DA000E06890ED2C0AB5EE400AF1EE10FA0CDD29
:106DB00094ED5D1AD4ED5E1AD4ED730A94ED7E0A5B
:106DC0009FED282A3046FEF7FBFE9FED258A04F151
:106DD0007C00B0EE481AD4ED021A94ED1C0AD4EDF2
:106DE000710A0DF07DFDB0EE481A04F1B800D4ED43
:106DF000021AD4ED760A0DF073FDB0EE481A84ED58
:106E00006F0A04F1F400D4ED021A94ED1D0AD4EDDA
:106E1000730A0DF065FDB0EE481A04F59870D4EDD4
:106E2000021AD4ED750A0DF05BFD84ED700A04F5CD
:106E3000BE7094ED6F0A0AF05BFD84ED6F0A04F5F5
:106E4000CE7094ED700A0AF053FD002084ED700AB4
:106E500040B202B0BDEC028BBDE8F0810024744961
:106E600000000000DB0FC940B0B52DED028B0028FB
:106E70006AD00446B0EE408AC16000250574FBF775
:106E800097FEB0EE480AE16804F17C0001F13C0293
:106E900000210DF0D5FDB0EE480AE16804F1B8001C
:106EA00001F11C0201210DF0CBFDB0EE480AE168B2
:106EB00004F1F40001F17C0200210DF0C1FDB0EEFF
:106EC000480AE16804F5987001F15C0201210DF0B7
:106ED000B7FDE168B0EE480A04F5BE70D1ED270AAF
:106EE0000AF036FDE168B0EE480A04F5CE70D1ED47
:106EF000270A0AF02DFDE06890ED290A90ED2A2A74
:106F000090ED2B1A90ED2C3A30EE011A84ED5C0ACC
:106F100084ED5B1A32EE031A84ED5D1A84ED5E2A6D
:106F20000BF0E2FFE06808300AF0D6FEE0680830B7
:106F30000AF09EFDE16804F118001031FFF748FCEB
:106F400068B2BDEC028BB0BDFF2568B2BDEC028B10
:106F5000B0BD00000000000010B586B00446C06857
:106F600094ED700A0CF054F8B1EE040A0020CDE95B
:106F7000030094ED6F1A029049F69A1021EE000A70
:106F8000C3F699600590E0688DED010A0BF0DCFE18
:106F9000E06801A908300AF0E3FD06B010BD00006A
:106FA00010B538B30446C0680CF0BEF8E0680BF0CA
:106FB00053FF48B100F1080304F5FC7C40690ECB97
:106FC0008CE80E00C4F80402E06808300AF00CFFF8
:106FD000E06808300AF098FD48B100F11C0304F5A0
:106FE000F47C806A0ECB8CE80E00C4F8F40100201B
:106FF00040B210BDFF2040B210BD000000000000F4
:1070000010B310B504461830FFF752FD606BC4F89A
:10701000DC01E16CC4F8C411216DC4F8C811616DC4
:10702000C4F8CC11216CC4F8D011616CC4F8D4112F
:10703000A16CC4F8D811A16BE06BC4E978100020F2
:10704000BDE8104040B27047FF2040B270470000DA
:1070500070470000000000007047000000000000C2
:1070600070470000000000007047000000000000B2
:107070007047000000000000B0B582B090F85C20BE
:10708000012A03D10221084602B0B0BD42F2083203
:1070900000230193C4F202020093A2F54274036834
:1070A000A34227D14FF6006C4FF60055CFF6FF7C78
:1070B000CFF6FF7552F80C40535923435B0719D4A0
:1070C000D1F800E01368BEF1000F23F440441DD056
:1070D0004B6823431360535952F80C502B43DB0782
:1070E00022D1136840F61F758968AB4341EA0E014F
:1070F000194316E0016E41F02001016601210022D2
:1071000080F85C20084602B0B0BD00BF1460515941
:1071100052F80C301943C90708D1116840F61F73A3
:10712000994311600021EAE70021E8E70021E6E742
:107130002DE9F04181B00022009290F85C20012AF4
:1071400004D10221084601B0BDE8F08103680122A4
:1071500080F85C209A68520700F1FC8246F2083CF5
:107160004FF6FF78C5F6020CC0F20F08ACF5427E70
:107170000A68734516D0B2F1FF3F13DD92FAA2F50B
:1071800012EA080FB5FA85F54FF0010608BF950E13
:10719000920E05F01F0506FA05F5DE693543DD613F
:1071A00001E000BF920E4D681F2402F01F02C5F3DC
:1071B000012605F01F05AC4003EB8606AA40376B9D
:1071C00027EA0404224332639A689C68E40844EA8C
:1071D0009202D20740F029810A6807268D6873451C
:1071E000C2F34064C2F3045203EB840406FA02F6CD
:1071F000676905FA02F227EA060642EA06026261B8
:1072000010D041F20002C5F60042126802F070424E
:10721000B2F1805F6ED14A69DC680E2505EA54063A
:107220009CE000BF4FF604540A69CFF6FF74042AAD
:107230004D695CF8046067D14FF65852CFF6FF7283
:107240005CF802201C6E0E68C4F3846416EA08021F
:10725000C6F3846596FAA6F6B6FA86F6374608BFF0
:107260002F46BC420CD11A6E22F000421A660C68FE
:1072700004EA0802C4F3846594FAA4F4B4FA84F628
:107280005C6E37465C6E002A08BF2F46C4F38464E8
:10729000BC420CD15A6E22F000425A660C6804EAD5
:1072A0000802C4F3846594FAA4F4B4FA84F69C6EDC
:1072B00037469C6E002A08BF2F46C4F38464BC4244
:1072C0000CD19A6E22F000429A660C6804EA080219
:1072D000C4F3846594FAA4F4B4FA84F6DC6E002A4C
:1072E000DC6E08BF2E46C4F38462B24200F099807F
:1072F0009BE000BFDC684A69DD68E4064FEA55059B
:107300002AD405F00E0629E00624ACF52A7704EA13
:1073100096040E6805FA04F406F0F8452C4357F875
:10732000226044F0004447F822400A69CC6957F8CB
:10733000225025F080752C4347F822400A6991F8C5
:10734000204057F82250012C25F0007508BF05F1A8
:10735000007547F8225068E005F008060F6903F150
:107360006005042F20D12A680C6802F0F842B2EBC5
:10737000846F4FEA846241D12C6824F000442C6071
:107380005C6E04F0F84494423DD09C6E04F0F844E6
:10739000944241D19C6E24F000449C66DC6E04F063
:1073A000F844944241D13CE00C68B24055F8276063
:1073B00004F0F84406F000462243324345F8272003
:1073C0000A6991F8214055F82260012C26F0004608
:1073D00008BF06F1004645F822600A7E0C691D6967
:1073E000013A04F01F04B2FA82F225F4F045520982
:1073F000D202A2402A431A6117E000BF5C6E04F07B
:10740000F8449442C1D15C6E24F000445C669C6EEA
:1074100004F0F8449442BDD0DC6E04F0F844944289
:1074200003D1DA6E22F00042DA669A68D20711D1EF
:1074300073450A68CD680FD005F01804D3F8C01062
:1074400028FA04F402EA0806B14314402143C3F8C1
:10745000C01012E0002182E14FF6A85105F0180695
:10746000CFF6FF7128FA06F602EA080716405CF824
:107470000140BC4334434CF801400021C4F2527136
:1074800001F52D04A54240F0138146F20004C5F633
:107490000204A3422CD042F20014C4F20204A3421C
:1074A0003CD042F20004C4F20204A34250D11F2493
:1074B000C1F2F044A24275DD40F2FF74C2F63064BE
:1074C000A2425FDD40F60004C2F63064A24200F042
:1074D000BF8041F20004C3F26024A24200F0B280F7
:1074E0000024C4F22134A24200F0CD80B6E000BFF7
:1074F0001F21C1F2F0418A422CDC0721C0F69041E5
:107500008A426DDC0221C0F230418A4254D004210B
:10751000C0F660018A4216D0AAE000BF1F21C1F266
:10752000F0418A4228DC0721C0F690418A4245DCBE
:107530000221C0F230418A423ED00421C0F66001EF
:107540008A4240F08B804021C1F620119BE000BFB1
:10755000002198E040F2FF71C2F630618A4253DCAC
:107560002021C1F2F0418A4234D040F20041C2F6FB
:1075700000218A4211D07BE040F2FF71C2F63061F7
:107580008A4253DC2021C1F2F0418A4222D040F2EB
:107590000041C2F600218A4260D140F60001C2F6E5
:1075A000306170E00721C0F690418A4206DC02217A
:1075B000C0F230418A42C0D1012164E00821C0F606
:1075C00090418A421CD01021C1F2C0018A4211D0E0
:1075D00044E000BF40F20021C2F2B05153E000BFCE
:1075E0000821C0F690418A420AD01021C1F2C001A0
:1075F0008A423DD140F20011C2F2801143E000BF47
:107600008021C1F650513EE040F60001C2F63061E3
:107610008A421DD042F20001C3F290618A4227D112
:1076200044F20001C3F6C0212DE000BF40F6000186
:10763000C2F630618A420BD041F20001C3F26021F0
:107640008A420BD142F20001C3F290611BE000BFFD
:1076500041F20001C3F2602115E000BF00240021C7
:10766000C4F68434A24204BF0021C4F6B8710AE013
:1076700044F200040021C3F6C024A24204BF48F231
:107680000001C3F6F061734512D091FAA1F44FF6F0
:10769000C135B4FA84F4C0F20A05294208BF8C0E41
:1076A00004F01F01012404FA01F1DC692143D961CE
:1076B000B2F1FF3F02DD002151E000BF42F20001C4
:1076C00042F20016C4F20201C4F2020601F580740F
:1076D00001F54275A342644608BF2C468B4208BFA1
:1076E0002C4643F48075B54225682BD18C68D1F8BF
:1076F00008112143C9072DD1002105F0E074CCF217
:1077000052718A4208BF15F400012FD00021CCF23B
:1077100021318A4208BF15F080712BD00021CCF6B0
:1077200084318A424FF0000119D115F4800208BF5C
:10773000734514D1DCF8001021F0E071214341F4CD
:10774000800156E04FF60051CFF6FF715CF8011052
:10775000C907D1D0016E41F020010166012100224C
:1077600080F85C20084601B0BDE8F081734505D083
:107770000021F4E7734535D00021F0E7DCF8001074
:1077800042F6635221F0E071C0F23E52214341F4CF
:107790000001CCF8001040F20C01C2F2004109686F
:1077A0008909A1FB02129109022202EB4101009119
:1077B000009919B3009901390091009901B300991A
:1077C000013900910099E9B10099013900910099BE
:1077D000D1B1009901390091009900294FF00001C1
:1077E000E8D1BCE7DCF8001021F0E071214341F062
:1077F0008071CCF800100021B1E700BF0021AEE796
:107800000021ACE70021AAE70021A8E70000000062
:1078100070470000000000007047000000000000FA
:107820002DE9F04F81B046F2083942F200080446D3
:107830000068C5F60209C4F2020808F5807B08F565
:1078400042774A460168584508BF3A464045436872
:1078500008BF3A4603EA0105A90716680CD5206E51
:10786000C00603D4206E40F4006020662046FFF777
:10787000EFFB20680221016015F00C0F06F01F0AD3
:1078800044D0216EC90603D4216E41F400712166F3
:10789000C16811F4406F33D10146584508BF4146D5
:1078A000814218BF0946BAF1000F08BF0146BAF17C
:1078B000050F08BF0146BAF1090F08BF0146C968A4
:1078C00089041DD4016809071AD5816849070FD4B6
:1078D000416821F00C014160206E20F48070206628
:1078E000206EC0040CD4206E40F00100206607E03A
:1078F000206E40F010002066606E40F0010060666F
:107900002046FFF785FF20680C21016015F0600F0D
:1079100022D0216EC90603D4216E41F400512166A4
:107920000146584508BF414606F01E02814218BF75
:107930000946BAF1000F08BF0146062A08BF0146F2
:10794000C26C12F4C07FC268C9686BD02046FFF7D2
:1079500083FB20686021016029060BD4E90515D45A
:10796000A90520D4E9062BD4690549D401B0BDE8A6
:10797000F08F00BF206E40F480302066204600F07B
:1079800003FA206880210160E905E9D5206E40F402
:10799000003020662046FFF767FB20684FF48071B7
:1079A0000160A905DED5206E40F4802020662046C7
:1079B000FFF75EFB20684FF400710160E906D3D544
:1079C000E16B69B1BAF1000F52D0584508BFB94612
:1079D000404508BFB946D9F8001011F4404F0BD00C
:1079E000206E40F480602066606E40F002006066A9
:1079F0002046FFF711FF2068102101606905B5D509
:107A0000216E41F480412166616E41F0080161669A
:107A10004FF480610160204601B0BDE8F04FFFF7F0
:107A20001FBB00BF8B0106D502F4406201F4005376
:107A3000D2187FF48BAF890201683FF587AF11F050
:107A400040013FF483AF8168090715D4416821F0F4
:107A500060014160206E20F480502066206EC005D9
:107A60003FF574AF206E40F0010020666EE700BF66
:107A7000C1688907B4D1BFE7206E40F010002066CE
:107A8000606E40F00100606660E7000000000000EA
:107A9000B0B582B0044600284FF00000019009D034
:107AA000206E58B120688168890012D48168C900AD
:107AB00019D54EE00125284602B0B0BD204600F0A1
:107AC00067F90020606684F85C002068816889009E
:107AD000ECD54FF6C0728168C5F6FF721140816027
:107AE0008168C90035D44FF6C0718268C5F6FF7150
:107AF00001F18051114042F6635201F180518160E1
:107B000040F20C01C0F23E52C2F2004109688909FC
:107B1000A1FB0212012101EB921101910199C1B166
:107B2000019901390191019900291FBF019901397A
:107B3000019101991FBF00290199013901911CBFD1
:107B40000199002905D00199013901910199002974
:107B5000E6D18168C90009D4216E012541F01001E8
:107B60002166616E41F00101616600E000258168D7
:107B7000226E02F01002C1F380018918216E07D035
:107B800041F0100001252066284602B0B0BD00BFBC
:107B900021F4817146F2100C023121668168C5F62C
:107BA000020CC90724D142F2001240F48071C4F2E1
:107BB0000202914242F20001C4F2020140F0A080B0
:107BC0008A68D1F808311A43D20711D101F58072C1
:107BD00001F5427390421A4618BF0CF53E72884276
:107BE00008BF1A466168136823F47C1319431160B7
:107BF000617EE36BACF1100E704543EA413121D058
:107C0000A268114394F82020012A41EA024306D1D8
:107C1000616A0022CFF6FE7202EB41410B43A16A7A
:107C200029B101F47871E26A194341EA020370450F
:107C300016D04CF20302C168CFF6F072114019431E
:107C4000C1601FE0D4E90232082B41EA02015DD095
:107C50000C2B5FD01C2B61D110231943D2E700BF3E
:107C600044F207025CF8041CCFF6F072114019438D
:107C70004CF8041CDCF80010626B21F040611143E9
:107C8000CCF8001081688268D20842EA9101C907E5
:107C900065D1217E70454FEA813103D0226B1143BB
:107CA00004E000BF94F8382041EA4201C26844F27F
:107CB00003039A431143C16094F84410012919D178
:107CC0004FF61E017045CFF600412DD0026902EA41
:107CD000010C0021D4E91223CFF6FF7101EB024120
:107CE0004CEA0302236D1143626D1943114341F0C5
:107CF000010102E0016921F00101016123E000BFFF
:107D00005CF8082CD2073FF461AF71E700231943F8
:107D100078E700BF0823194374E700BF182B18BF8A
:107D2000002319436EE700BFDCF800201140D4E9BE
:107D300012231143226D1943636D1143194341F01E
:107D40000101CCF800100169226C21F070417045EE
:107D500041EA0201016102D02046F9F789FE20685C
:107D60002169026B012922F00F0102D1E269013A77
:107D7000114301630121206E61F301002066284652
:107D800002B0B0BD0000000070470000000000001D
:107D90002DE9F04186B0044646F20002C5F6020223
:107DA0000020216805909142049067D042F20000C3
:107DB000C4F20200814240F0948044F2E040002589
:107DC000C5F60200C5F6020501AE4FF0030850F8F3
:107DD000081C002741F0200140F8081C50F8081C3E
:107DE00001F0200100910099016841F0010101605A
:107DF000016801F0010100910099016841F004015E
:107E000001600068314600F00400009000982020D6
:107E100001902846CDF80880039702F049FE102013
:107E20003146CDE9010805F50060039702F040FEF8
:107E300042F220151020C2F20045C4F20200286070
:107E40000920C5E901074FF4806028614FF4006004
:107E500068614FF40050A8614FF48070EF60C5E98D
:107E6000070728466F6201F05BF808B1FEF7F8FAE1
:107E7000A565AC6306B0BDE8F08100BF44F2E04107
:107E800042F29815C5F60201C2F200450A6842F0B6
:107E900080720A600A6801F6287102F0807200920E
:107EA000009A29601121E860C5E901104FF4806152
:107EB00029614FF4006169614FF400512862C5E9FE
:107EC0000610284601F02CF808B1FEF7C9FA7F2009
:107ED00005210022A565AC6302F0C6FF7F2002F0F9
:107EE000B3FF06B0BDE8F0812DE9F041044602F091
:107EF000E3FE0CB3054694F83500022820D140F289
:107F00000F472668C4F2020740F26F48BE42C4F22F
:107F100002081DDC6F20C4F2020086422ADC3F20EA
:107F2000C4F20200864241DC1020C4F20200864204
:107F300063D028205CE000BF0120BDE8F08100BFD5
:107F4000802060650120002184F83410BDE8F081B4
:107F500046451BDC40F23F40C4F2020086422DDC65
:107F600040F21040C4F20200864246D040F228405F
:107F70003EE000BF9F20C4F20200864228DC702051
:107F8000C4F20200864238D0882031E040F29F409F
:107F9000C4F20200864223DC40F27040C4F20200C8
:107FA00086422AD040F2884022E000BF4020C4F23E
:107FB0000200864221D058201AE000BF40F2404023
:107FC000C4F20200864218D040F2584010E000BFD0
:107FD000A020C4F2020086420FD0B82008E000BF03
:107FE00040F2B840C4F20200864206D040F2A040FF
:107FF000C4F20200864240F099813146306820F098
:108000001E0041F8140B6FF080000A68464500EA34
:10801000020008601ADC9F20C4F20200864233DCB2
:108020005720C4F2020086425ADC1020C4F202003B
:10803000864200F097802820C4F20200864200F0B9
:1080400091804020C4F202008AE000BF45F22F4038
:10805000C5F6020086422DDC40F2B740C4F20200B1
:1080600086424BDC40F27040C4F20200864279D076
:1080700040F28840C4F20200864273D040F2A04031
:10808000C4F202006CE000BF40F22740C4F20200DC
:10809000864243DCA020C4F20200864262D0B820AF
:1080A000C4F2020086425DD040F21040C4F20200E9
:1080B00056E000BF45F26B40C5F6020086423FDC49
:1080C00045F23040C5F6020086424BD045F24440AE
:1080D000C5F60200864245D045F258403EE000BF5A
:1080E0005820C4F2020086423CD07020C4F2020044
:1080F000864237D08820C4F2020031E040F2B84016
:10810000C4F2020086422DD045F20840C5F60200B6
:10811000864227D045F21C4020E000BF40F22840B4
:10812000C4F2020086421DD040F24040C4F2020078
:10813000864217D040F25840C4F2020010E000BF5F
:1081400045F26C40C5F6020086420BD045F29440E1
:10815000C5F60200864205D045F28040C5F6020011
:10816000864204D1206E016821F48071016030687C
:1081700020F00100306000BF3068C00710D002F06E
:108180009BFD401B0628F7D320206065032084F860
:1081900035000120002184F83410BDE8F08100BFD3
:1081A0002068B84210DC6F21C4F2020188421DDC55
:1081B0003F21C4F20201884234DC1021C4F20201E2
:1081C000884255D028214FE040451BDC40F23F411A
:1081D000C4F2020188422DDC40F21041C4F20201D7
:1081E000884245D040F228413EE000BF9F21C4F2C2
:1081F0000201884228DC7021C4F20201884237D093
:10820000882131E040F29F41C4F20201884223DC20
:1082100040F27041C4F20201884229D040F2884104
:1082200022E000BF4021C4F20201884220D0582140
:108230001AE000BF40F24041C4F20201884217D068
:1082400040F2584110E000BFA021C4F20201884270
:108250000ED0B82108E000BF40F2B841C4F20201DC
:10826000884205D040F2A041C4F20201884261D1A7
:10827000D4E9161202F01F023F2303FA02F28A60C9
:10828000404561DC9F21C4F20201884214DC572181
:10829000C4F20201884227DC1021C4F202018842A4
:1082A00000F0A8802821C4F20201884200F0A280D8
:1082B0004021C4F202019BE040F22741C4F20201D6
:1082C000884221DCA021C4F20201884200F09280A1
:1082D000B821C4F20201884200F08C8040F21041C3
:1082E000C4F2020184E000BF5821C4F202018842B6
:1082F00000F080807021C4F2020188427AD0882187
:10830000C4F2020174E000BF40F22841C4F202014D
:1083100088426FD040F24041C4F20201884269D0E5
:1083200040F25841C4F2020162E000BF6FF00E005B
:1083300031466AE6D4E9161202F01F02012303FA5D
:1083400002F24A6040459DDD45F22F41C5F602012B
:10835000884217DC40F2B741C4F20201884227DCB0
:1083600040F27041C4F20201884243D040F2884199
:10837000C4F2020188423DD040F2A041C4F20201A1
:1083800036E000BF45F26B41C5F6020188421FDCB2
:1083900045F23041C5F6020188422BD045F24441F6
:1083A000C5F60201884225D045F258411EE000BFC3
:1083B00040F2B841C4F2020188421BD045F20841A4
:1083C000C5F60201884215D045F21C410EE000BFFF
:1083D00045F26C41C5F6020188420BD045F294414A
:1083E000C5F60201884205D045F28041C5F602017A
:1083F00088420BD1616EA26EE06E4A6030B10168B6
:1084000021F480710160D4E91C014160012084F8ED
:1084100035000020002184F83410BDE8F081000010
:1084200080B5D8B190F83510022919D140F20F4229
:108430000168C4F20202914216DC6F23C4F2020307
:10844000994227DC3F23C4F2020399423EDC102309
:10845000C4F2020399425FD0282359E0012080BD75
:1084600080214165012080BD40F26F43C4F20203C8
:1084700099421BDC40F23F43C4F2020399422DDCD7
:1084800040F21043C4F20203994245D040F228431F
:108490003EE000BF9F23C4F20203994228DC702310
:1084A000C4F20203994237D0882331E040F29F435F
:1084B000C4F20203994223DC40F27043C4F2020387
:1084C000994229D040F2884322E000BF4023C4F201
:1084D0000203994220D058231AE000BF40F24043E3
:1084E000C4F20203994217D040F2584310E000BF93
:1084F000A023C4F2020399420ED0B82308E000BFC3
:1085000040F2B843C4F20203994205D040F2A043BE
:10851000C4F20203994275D191424FF0040280F8EF
:10852000352011DC6F20C4F20200814222DC3F20A2
:10853000C4F20200814239DC1020C4F20200814200
:1085400059D0282054E000BF40F26F40C4F202002E
:1085500081421BDC40F23F40C4F2020081422DDC2C
:1085600040F21040C4F20200814244D040F2284060
:108570003EE000BF9F20C4F20200814228DC702050
:10858000C4F20200814236D0882031E040F29F40A0
:10859000C4F20200814223DC40F27040C4F20200C7
:1085A000814228D040F2884022E000BF4020C4F23F
:1085B000020081421FD058201AE000BF40F2404024
:1085C000C4F20200814216D040F2584010E000BFD1
:1085D000A020C4F2020081420DD0B82008E000BF04
:1085E00040F2B840C4F20200814204D040F2A04000
:1085F000C4F202008142086820F0010008600020F7
:1086000080BD00BF0A6822F00E020A6045F25742A0
:10861000C5F6020291420A6822F001020A600FDCEC
:1086200045F22F42C5F60202914219DC45F208429A
:10863000C5F60202914229D045F21C4222E000BF59
:1086400045F27F42C5F60202914213DC45F25842E0
:10865000C5F60202914219D045F26C4212E000BF09
:1086600045F23042C5F6020291420FD045F2444233
:1086700008E000BF45F29442C5F60202914205D0DF
:1086800045F28042C5F6020291421AD1D0E9181C87
:10869000D0E916E30A6822F480720A6003F01F0131
:1086A000012202FA01F1CEF80410816ECCF8041018
:1086B000C16E31B10A6822F480720A60D0E91C12DE
:1086C0004A60012180F83510026D002180F83410D5
:1086D0000AB190470021084680BD0000000000005C
:1086E000406D7047000000002DE9F04782B0002186
:1086F000019140F20C010446C2F2004148F2B51269
:10870000C1F64E32A56D096840F26F490068C4F2A7
:108710000209A1FB021848452E68296816DC9F2132
:10872000C4F2020188422DDC5721C4F202018842C2
:1087300052DC1021C4F2020188427BD02821C4F20D
:108740000201884276D0402170E000BF45F22F42FE
:10875000C5F60202904229DC40F2B742C4F202029E
:10876000904245DC40F27041C4F20201884261D07F
:1087700040F28841C4F2020188425BD040F2A0413D
:1087800054E000BF40F22741C4F2020188423FDCBE
:10879000A021C4F2020188424CD0B821C4F20201E7
:1087A000884247D040F2104140E000BF45F26B42A2
:1087B000C5F60202904275DC45F23042C5F602026F
:1087C000904200F0818045F24442C5F60202904298
:1087D0007AD045F2584273E05821C4F2020188422F
:1087E00028D07021C4F20201884223D088211DE0E4
:1087F00040F2B842C4F2020290421BD045F2084255
:10880000C5F6020290425FD045F21C4258E000BF1C
:1088100040F22841C4F2020188420BD040F24041AC
:10882000C4F20201884205D040F25841C4F202016C
:10883000884261D1E16D082201F01F0140F20F4A28
:108840008A40C4F2020A324200F0E98050454FF0FB
:10885000040313DC6F27C4F20207B8426CDC3F2725
:10886000C4F20207B84200F3A7801027C4F202073F
:10887000B84200F0C8802827C0E000BF484567DC48
:1088800040F23F47C4F20207B84200F39D8040F235
:108890001047C4F20207B84200F0B58040F2284702
:1088A000ACE000BF45F26C42C5F6020290420BD02C
:1088B00045F28042C5F60202904205D045F294424C
:1088C000C5F60202904217D10268E36D570703F024
:1088D0001F0315D504279F4017EA010610D0110485
:1088E0006F6045D4910603D4016821F00401016052
:1088F000216C002940F0F68202B0BDE8F08700BF8D
:1089000097073DD502279F4017EA010638D011048A
:108910006F6000F1ED82910609D4016821F00A012F
:108920000160012084F83500002084F83400E16BF8
:10893000002940F0D782DFE79F27C4F20207B84240
:108940004CDC7027C4F20207B8425CD0882755E09F
:1089500040F29F47C4F20207B84247DC40F270473A
:10896000C4F20207B8424ED040F2884746E000BF4A
:10897000D00300F1C382A16C002940F0B382BBE7B1
:108980001207B9D508229A401140B5D0016821F0EC
:108990000E010160012000FA03F16960606584F84E
:1089A00035000020E16C84F834000029A4D0204672
:1089B000884702B0BDE8F0874027C4F20207B842FA
:1089C00021D058271AE000BF40F24047C4F2020706
:1089D000B84218D040F2584710E000BFA027C4F2B8
:1089E0000207B8420FD0B82708E000BF40F2A04706
:1089F000C4F20207B84206D040F2B847C4F20207F8
:108A0000B84218BF082307681F4208D0036823F044
:108A100004030360AA60626D42F0010262650122F4
:108A20008A4032426FD0504510DC6F23C4F20203FB
:108A300098421DDC3F23C4F20203984234DC102329
:108A4000C4F20203984256D028234FE048451BDC6D
:108A500040F23F43C4F2020398422DDC40F210433F
:108A6000C4F20203984246D040F228433EE000BFE1
:108A70009F23C4F20203984228DC7023C4F202034D
:108A8000984238D0882331E040F29F43C4F2020379
:108A9000984223DC40F27043C4F2020398422AD089
:108AA00040F2884322E000BF4023C4F20203984210
:108AB00021D058231AE000BF40F24043C4F2020321
:108AC000984218D040F2584310E000BFA023C4F2EF
:108AD000020398420FD0B82308E000BF40F2A04341
:108AE000C4F20203984206D040F2B843C4F2020333
:108AF000984240F00B8243691B0604D5AA60626D60
:108B000042F00202626504228A4032426FD0504530
:108B100010DC6F23C4F2020398421DDC3F23C4F231
:108B20000203984234DC1023C4F20203984256D068
:108B300028234FE048451BDC40F23F43C4F20203C8
:108B400098422DDC40F21043C4F20203984246D012
:108B500040F228433EE000BF9F23C4F20203984244
:108B600028DC7023C4F20203984238D0882331E015
:108B700040F29F43C4F20203984223DC40F2704368
:108B8000C4F2020398422AD040F2884322E000BF98
:108B90004023C4F20203984221D058231AE000BFB8
:108BA00040F24043C4F20203984218D040F25843C6
:108BB00010E000BFA023C4F2020398420FD0B823F4
:108BC00008E000BF40F2A043C4F20203984206D07E
:108BD00040F2B843C4F20203984240F09F81036818
:108BE0009B0704D5AA60626D42F004026265102200
:108BF00002FA01F1314200F0818050454FF0080245
:108C000010DC6F23C4F2020398421DDC3F23C4F240
:108C10000203984234DC1023C4F20203984256D077
:108C200028234FE048451BDC40F23F43C4F20203D7
:108C300098422DDC40F21043C4F20203984246D021
:108C400040F228433EE000BF9F23C4F20203984253
:108C500028DC7023C4F20203984238D0882331E024
:108C600040F29F43C4F20203984223DC40F2704377
:108C7000C4F2020398422AD040F2884322E000BFA7
:108C80004023C4F20203984221D058231AE000BFC7
:108C900040F24043C4F20203984218D040F25843D5
:108CA00010E000BFA023C4F2020398420FD0B82303
:108CB00008E000BF40F2A043C4F20203984206D08D
:108CC00040F2B843C4F20203984218BF042203687A
:108CD000134213D0A96001684903016808D4C9058B
:108CE00008D4016821F008010160216C21B905E078
:108CF00008034FD4216C09B120468847E06D00F08D
:108D00001F01202000FA01F2324200F0AB802068FF
:108D10001023504510DC6F27C4F20207B8421DDC57
:108D20003F27C4F20207B84238DC1027C4F202071A
:108D3000B8425AD0282753E048451BDC40F23F4751
:108D4000C4F20207B84231DC40F21047C4F2020715
:108D5000B8424AD040F2284742E000BF9F27C4F201
:108D60000207B8422CDC7027C4F20207B8423CD09C
:108D7000882735E040F29F47C4F20207B84227DC5B
:108D800040F27047C4F20207B8422ED040F2884742
:108D900026E000BFA16C0029AED1AFE74027C4F2A6
:108DA0000207B84221D058271AE000BF40F24047DE
:108DB000C4F20207B84218D040F2584710E000BF92
:108DC000A027C4F20207B8420FD0B82708E000BFBE
:108DD00040F2A047C4F20207B84206D040F2B847BA
:108DE000C4F20207B84218BF022307681F4239D0F5
:108DF000AA6094F83520042A02681BD122F01602DA
:108E00000260426922F080024261226C0AB9A26CBF
:108E10001AB1026822F0080202603F208840A86070
:108E2000012084F83500216D0020002984F83400E9
:108E300058D161E5510301680CD4C9050ED401680D
:108E400021F010010160012084F83500002084F831
:108E5000340003E0080301D4616C00E0E16B09B168
:108E600020468847606D00283FF446AD606DC0071E
:108E700034D0042084F8350020684FEA9821026835
:108E800022F001020260019A013201928A421AD84C
:108E90000268D20717D0019A013201928A4212D891
:108EA0000268D2070FD0019A013201928A420AD891
:108EB0000268D20707D0019A013201928A4202D891
:108EC0000268D207DFD10068C0074FF0030008BF77
:108ED000012084F83500002084F83400E16C00297A
:108EE0003FF40AAD2046884702B0BDE8F08700BFD6
:108EF000D00307D4616C0029F4D1FDE4216C002972
:108F0000F0D1F9E4E16B0029ECD1F5E40268042228
:108F10008A4032427FF4FBAD69E600BF026866E634
:108F20002DE9F04381B0044601F0C6FE002C00F0AC
:108F3000128140F26F4805462068C4F2020840459D
:108F400016DC9F21C4F2020188422DDC5721C4F2B5
:108F50000201884254DC1021C4F20201884200F070
:108F60007E802821C4F20201884278D0402171E03D
:108F700045F22F41C5F60201884229DC40F2B74193
:108F8000C4F20201884247DC40F27041C4F202019F
:108F9000884264D040F28841C4F2020188425ED027
:108FA00040F2A04156E000BF40F22741C4F2020166
:108FB000884241DCA021C4F2020188424FD0B8218E
:108FC000C4F2020188424AD040F2104142E000BFA0
:108FD00045F26B41C5F60201884200F3C18045F2BB
:108FE0003041C5F60201884200F0CD8045F244418F
:108FF000C5F60201884200F0C68045F25841BDE046
:109000005821C4F20201884229D07021C4F2020121
:10901000884224D088211DE040F2B841C4F2020108
:1090200088421CD045F20841C5F60201884200F092
:10903000AA8045F21C41A1E040F22841C4F202019D
:1090400088420CD040F24041C4F20201884206D06E
:1090500040F25841C4F20201884240F09782022156
:1090600084F83510002184F83410016821F00101E2
:1090700001600168C90708D001F01EFE401B0528E9
:1090800064D820680168C907F6D148F23F0204F1AC
:1090900008060168CFF610621140D4F818C06CCEF3
:1090A0001143D4F824901943E3692943256A0E43F8
:1090B000B9F1040F46EA0C0643EA060343EA050346
:1090C00003D1D4E90B6533432B43666843F4801125
:1090D000A6F13F07A6F12905042FA6F1470238BFE4
:1090E0000B46062DA6F14F0E38BF0B46022A26F07E
:1090F000030238BF0B46BEF1040F38BF0B46742A7B
:1091000008BF0B46B9F1040F0360416921F0070164
:1091100041EA090140F0F480D4E90A53002B41EA06
:10912000050100F0ED80BCF5005F00F0CF80BCF1E0
:10913000000F40F0D780022D00F0D780012D00F005
:10914000CB80002D00F0D180DAE000BF20206065E8
:10915000032084F83500012001B0BDE8F08300BF92
:1091600045F26C41C5F6020188420CD045F28041BF
:10917000C5F60201884206D045F29441C5F60201C7
:10918000884240F00382022184F83510002184F8DF
:1091900034100168A268A2F18003E768B3FA83F390
:1091A000402A4FEA53134FEA83336FF3101108BF7D
:1091B0001023226941EAD70167691943A36941EA8B
:1091C000D201E26941EAD70141EAD3014CF6CD432D
:1091D00041EAD2014AF6F832CAF2FD72276A024425
:1091E000CCF6CC43A2FB032341EA171101606FF0D8
:1091F000030000EA9300E0652046FCF7A9FDE16D5D
:10920000012201F01F0102FA01F14160206840458E
:1092100040F3858045F22F41C5F60201884217DCF4
:1092200040F2B741C4F20201884229DC40F27041A9
:10923000C4F20201884200F0BC8040F28841C4F2CE
:109240000201884200F0B58040F2A041ACE000BFCE
:1092500045F26B41C5F60201884223DC45F23041FC
:10926000C5F60201884200F0A48045F24441C5F6EB
:109270000201884200F09D8045F2584122E000BF83
:1092800040F2B841C4F20201884200F0928045F2F7
:109290000841C5F60201884200F08B8045F21C416E
:1092A00010E000BF45F26C41C5F60201884200F0B3
:1092B000808045F29441C5F60201884200F0798031
:1092C00045F28041C5F6020170E000BF032D17D8BA
:1092D000DFE805F00E0B0E02A3F1C072B2FA82F2C3
:1092E000520904E0032D03D30AD1C3F300623AB15B
:1092F00040206065012084F8350001B0BDE8F083AE
:1093000041612046FCF724FDE16D3F2201F01F0181
:1093100002FA01F18160206840453FF77BAF9F2151
:10932000C4F20201884211DC5721C4F202018842D2
:1093300020DC1021C4F2020188423AD02821C4F274
:109340000201884235D040212EE000BF40F2274183
:10935000C4F20201884219DCA021C4F20201884251
:1093600027D0B821C4F20201884222D040F2104135
:109370001AE000BF5821C4F20201884219D07021BE
:10938000C4F20201884214D088210DE040F2284145
:10939000C4F2020188420CD040F24041C4F2020102
:1093A000884206D040F25841C4F20201884240F09F
:1093B000E58045F2574C45F6FC0EC5F6020CC5F6A5
:1093C000020E604512DC45F22F41C5F602018842CB
:1093D00020DC45F20841C5F60201884234D045F24E
:1093E0001C41C5F6020188422ED085E045F27F413E
:1093F000C5F6020188421BDC45F25841C5F6020160
:10940000884221D045F26C41C5F6020188421BD04A
:1094100072E000BF45F23041C5F60201884213D028
:1094200045F24441C5F6020188420DD064E000BF18
:1094300045F29441C5F60201884205D045F28041CB
:10944000C5F60201884257D16FF007014CF6CD42B4
:1094500051FA80F1CCF6CC42A1FB0212AEF1FC0530
:10946000AEF17C061309A26803F01F01802A4FF0B9
:10947000010205EB8305256602FA01F26666A26623
:1094800002D10021616000E06168CBB20139072997
:109490002B60726016D85E1E082E19D260450EF140
:1094A000440219DC45F22F41C5F60201884245DC31
:1094B00045F20841C5F60201884255D045F21C41EB
:1094C0004EE000BF00206067C4E91B0056E000BF0B
:1094D000D4E91B02616F4EE045F27F41C5F60201FF
:1094E000884235DC45F25841C5F6020188423BD03E
:1094F00045F26C4134E000BF6FF00F014AF6AB2239
:1095000051FA80F1CAF6AA22A1FB021240F20F43DF
:10951000C4F2020308251109984203F1AA060B467A
:1095200088BF05EB121340F60005B042C4F20205F5
:1095300005F1800628BF0B4695E700BF45F2304194
:10954000C5F6020188420FD045F2444108E000BF51
:1095500045F28041C5F60201884205D045F29441AA
:10956000C5F60201884213D101210EEB8300B14000
:10957000E066226761670023036051600020606538
:10958000012184F8351001B0BDE8F0834020DEE50C
:1095900040F60000C4F2020000F1FC0E00F5A072DB
:1095A000E2E7000000000000B0B500283CD005460E
:1095B00090F83400012801D10220B0BD012085F8C7
:1095C000340095F83500012828D1022085F83500AF
:1095D000002068652868046824F0010404602846B7
:1095E000FCF74EFC40F20F422868C4F2020240F23F
:1095F0006F419042C4F2020118DC6F23C4F20203EF
:10960000984225DC3F23C4F2020398423CDC10233D
:10961000C4F2020398425ED0282357E04FF4006062
:109620006865002085F834000120B0BD88421BDC4D
:1096300040F23F43C4F2020398422DDC40F2104353
:10964000C4F20203984246D040F228433EE000BFF5
:109650009F23C4F20203984228DC7023C4F2020361
:10966000984238D0882331E040F29F43C4F202038D
:10967000984223DC40F27043C4F2020398422AD09D
:1096800040F2884322E000BF4023C4F20203984224
:1096900021D058231AE000BF40F24043C4F2020335
:1096A000984218D040F2584310E000BFA023C4F203
:1096B000020398420FD0B82308E000BF40F2B8433D
:1096C000C4F20203984206D040F2A043C4F202035F
:1096D000984240F02F8103680B2464F34403036035
:1096E0002B6C1BB1036843F008030360884219DC4C
:1096F0009F23C4F20203984232DC5723C4F20203D0
:10970000984259DC1023C4F20203984200F096807C
:109710002823C4F20203984200F090804023C4F250
:10972000020389E045F22F43C5F6020398422DDC7F
:1097300040F2B743C4F2020398424BDC40F270435C
:10974000C4F20203984279D040F28843C4F2020383
:10975000984273D040F2A043C4F202036CE000BF11
:1097600040F22743C4F20203984243DCA023C4F230
:109770000203984262D0B823C4F2020398425DD03B
:1097800040F21043C4F2020356E000BF45F26B43BF
:10979000C5F6020398423FDC45F23043C5F60203AA
:1097A00098424BD045F24443C5F60203984245D057
:1097B00045F258433EE000BF5823C4F202039842EA
:1097C0003CD07023C4F20203984237D08823C4F2FD
:1097D000020331E040F2B843C4F2020398422DD0B4
:1097E00045F20843C5F60203984227D045F21C43D0
:1097F00020E000BF40F22843C4F2020398421DD08B
:1098000040F24043C4F20203984217D040F258435A
:10981000C4F2020310E000BF45F26C43C5F6020338
:1098200098420BD045F29443C5F60203984205D006
:1098300045F28043C5F60203984274D12B6E1C6832
:10984000E40303D51C6844F480741C60EB6E1BB108
:109850001D6845F480751D60904211DC6F21C4F2D3
:10986000020188421EDC3F21C4F20201884235DC3D
:109870001021C4F20201884255D0282150E000BFD7
:1098800088421BDC40F23F41C4F2020188422DDCD9
:1098900040F21041C4F20201884244D040F2284113
:1098A0003EE000BF9F21C4F20201884228DC702103
:1098B000C4F20201884236D0882131E040F29F4153
:1098C000C4F20201884223DC40F27041C4F202017A
:1098D000884228D040F2884122E000BF4021C4F2F3
:1098E000020188421FD058211AE000BF40F24041D7
:1098F000C4F20201884216D040F2584110E000BF85
:10990000A021C4F2020188420DD0B82108E000BFB6
:1099100040F2B841C4F20201884204D040F2A041B2
:10992000C4F202018842016841F001010160002097
:10993000B0BD00BF0368052464F3430303602B6CD0
:10994000002B3FF4D3AE036843F00403CDE60000E0
:10995000B0B5044601F0B0F940F204010546C2F288
:109960000041621C097818BF0C4400BF01F0A4F943
:10997000401BA042FAD3B0BD90F89830013B012BB8
:109980000ED80068836D0B4212D0836D0B408B4262
:1099900016D1C36D43F00203C3658B0514D418E0E0
:1099A00000F19C01012002220B681A430A607047F3
:1099B000C36D43F00103C3658B0505D409E000BF07
:1099C0000323C3658B0504D5D0F8E0301343C0F8FA
:1099D000E0304B0504D5D0F8E4301A43C0F8E42059
:1099E0004FF6FF72436DC3F6CF720A401A434265C9
:1099F0008A0F4AF614010020C4F200010B681A43D2
:109A00000A607047000000002DE9F04390F898309C
:109A1000022B19D10668D6F8C03013F07C5F1DD038
:109A2000D6F8C4309B0223D4D6F8C4304D68002D3C
:109A30000D69C3F3044C8B6824D00C682B4323437B
:109A400043F0804E22E000BFD0F89C1041F00801A6
:109A5000C0F89C100120BDE8F08300BFD0F89C1036
:109A600041F02001C0F89C100120BDE8F08300BF48
:109A7000D0F89C1041F40071C0F89C100120BDE8A2
:109A8000F08300BF0C682B4343EA844E836ED0F80A
:109A90008450D1E907970CFB03F48B6949EA076707
:109AA000D1F81480D1F80C901F4305EB840347EAEA
:109AB000080745F824E047EA09475F60CF6887B1A7
:109AC0004FF6B035083303320024C0F6010500BF5D
:109AD000171957F8037C1F51CF680434EF5DBC425F
:109AE000F6D3012101FA0CF1C6F8D010C0F8941099
:109AF0000020BDE8F0830000704700000000000077
:109B000080B590F89820013A012A0BD80A68002AFB
:109B1000CA680FD00B69072A43EA427E18D18B69C5
:109B20001BE000BFD0F89C1041F00201C0F89C106F
:109B3000012080BD072A19D10A69D1F81CC012047E
:109B40008B6942EA0C221A4342F0605218E000BFCF
:109B5000D1F808C04B6943EA8C73006F496800EB89
:109B6000C10240F831E00020536080BD8B68D1F81D
:109B700010C09B0743EAC2624B6942EA0C421A4397
:109B80004968C06E40F82120002080BD0000000020
:109B900090F898C0BCF1010F0ED19200006842EA23
:109BA0000111DDF800C041EA430141EA0C01C0F8AF
:109BB00080100020704700BFD0F89C1041F00401D5
:109BC000C0F89C100120704710B34AF200010068F1
:109BD000C4F2000188420FD04DF20041C4F20001EE
:109BE00088420BD04AF20041C4F20001884218BFFB
:109BF0007047012003E000BF002000E0022041F296
:109C00002021C2F2004101EB4010C06A00B10047C0
:109C100070470000000000007047000000000000D6
:109C2000B422402908BFA4220068805800F07F00B9
:109C300070470000000000002DE9F04390F8987094
:109C4000022F11D1402919D10668D6F8A07017F457
:109C5000FE0F2FD0D6F8A4707F0635D0D6F8A470AA
:109C6000FF013BD400273CE0D0F89C1041F00801F4
:109C7000C0F89C100120BDE8F08300BF41290FD13E
:109C80000668D6F8B07017F4FE0F13D0D6F8B4708B
:109C90007F0619D0D6F8B470FF012BD400272CE032
:109CA000076D8F4206D900F17C04456D4FF0000C22
:109CB0000E462BE0D0F89C1041F02001C0F89C101B
:109CC0000120BDE8F08300BFD0F89C1041F4807102
:109CD000C0F89C100120BDE8F08300BFD6F8A0704A
:109CE000FF0FD6F8A46000F17404C6F30526F51939
:109CF000466C0AE0D6F8B070FF0FD6F8B46000F1F9
:109D00007804C6F30526F519C66CAC46754324687D
:109D100004EB850E54F8257017F08047576054F80F
:109D2000257027F0604608BFC7F38A46166054F8CE
:109D3000257007F00057976054F8254004F0004460
:109D40001461BEF80440D461BEF8064014F00F045C
:109D5000D460DEF8044004F480145461DEF804405A
:109D600004F4001494619EF8074004F07F04146228
:109D7000DEF804404FEAD474546229D04FF6B0386C
:109D80000024C0F6010800BF0EEB0406651C377AFC
:109D90001F55D76818F80770BD423FBF1F19757A65
:109DA0007D70D5683EBF18F80590A51C4D450FD2B3
:109DB000B57ABD70D56818F80590E51C4D4507D2F9
:109DC000F57A0434FD70D56818F80550AC42DBD341
:109DD000402905D10068C0F8A8C00020BDE8F08384
:109DE000412905D10068C0F8B8C00020BDE8F08363
:109DF0001F2909D80068012202FA01F1C0F8981061
:109E00000020BDE8F08300BF006801F01F010122BF
:109E100002FA01F1C0F89C100020BDE8F0830000B8
:109E200080B590F89820022A40D10268D2F8F0302C
:109E300013F47C1F42D0D2F8F4309B0646D0D2F8FF
:109E4000F430D0F88000C3F3042C50F83C3013F009
:109E500080434B6050F83CE02EF0604308BFCEF3E7
:109E60008A430B6050F83C3003F000538B6000EBEA
:109E7000CC0350F83C0000F0004008619888C861AD
:109E8000D88800F00F00C860586800F4801048615E
:109E9000586800F400108861586800F44000486277
:109EA000D87908620020C2F8F8C080BDD0F89C10B4
:109EB00041F00801C0F89C10012080BDD0F89C1032
:109EC00041F02001C0F89C10012080BDD0F89C100A
:109ED00041F48071C0F89C10012080BD000000009A
:109EE0000068D0F8C40000F03F0070470000000098
:109EF00070470000000000002DE9F04F87B00446D5
:109F00004AF61000C4F2000001684AF61400C4F2D8
:109F100000000268206802EA010A056DD0F854903A
:109F2000076DD0F85480036D0293436D0193036D68
:109F30000693436D0593036D0493436D0393436D43
:109F4000066D06EA030B5FEACB530BD54FF4807125
:109F500001654AF610010020C4F2000108602046A5
:109F6000FFF7C6FF05EA09064AF610095FEA4B50FB
:109F7000C4F200094FEA8A750ED52068D0F8DC10CB
:109F8000D0F8E42011404FF4806202650020C9F847
:109F90000000204600F0A8FC08EA070806F4704616
:109FA00055B12068002101650AF00300C9F80000DE
:109FB00020462946FFF7A0FDDDE9011000EA010770
:109FC00008F00F0546B12068314606650020C9F843
:109FD0000000204600F0D8FC07F0F00645B12068EC
:109FE000294605650020C9F80000204600F0F8FB6E
:109FF00046B12068314606650020C9F800002046B9
:10A0000000F016FC5FEA0B5000F1B6805FEA8B505F
:10A0100000F1C0805FEA0B3000F1CF805FEACB3007
:10A0200000F1D9805FEA4B30DDE9031000EA010559
:10A0300009D520684FF4802101650020C9F800008F
:10A04000204600F049FC5FEA8B30DDE9051000EAAC
:10A05000010005F060710CD522684FF400331365E0
:10A060000022C9F80020D4F89C2042F08002C4F8F5
:10A070009C2000F0715539B1206801650020C9F8B5
:10A0800000002046FFF7C8FD206845B105650021A6
:10A09000C9F80010D4F89C102943C4F89C10A9F505
:10A0A000016188425ED16068816889075AD0016A7F
:10A0B000426A036A476A114003EA070202F0300568
:10A0C000D0F82080D0F82490026A049211F00F0199
:10A0D000D0F824B0026A0692426A0592466AD0F825
:10A0E00020A003D00162204600F0EAFB08EA09073D
:10A0F0002DB1606829460562204600F0E9FB06EABA
:10A100000A0007F4C0754006049800EA0B060AD559
:10A1100060684023C16BC26B090C02F03F0203620E
:10A12000204600F0D1FBDDE9051000EA010706F446
:10A13000FC462DB1606829460562204600F0BCFB54
:10A1400007F4F02036B161680E62D4F89C103143F8
:10A15000C4F89C1030B161680862D4F89C100843C0
:10A16000C4F89C00D4F89C00002847D0204607B0D3
:10A17000BDE8F04FFFF728BD20684FF4006101658E
:10A180000020C9F80000204600F026FC5FEA8B5052
:10A190007FF540AF2068D0F8D810D0F8E02011400B
:10A1A0004FF4007202650020C9F80000204600F05C
:10A1B000C3FB5FEA0B307FF531AF20684FF400211D
:10A1C00001650020C9F80000204600F005FB5FEAA9
:10A1D000CB307FF527AF20684FF480310165002038
:10A1E000C9F80000204600F07BFB5FEA4B30DDE958
:10A1F000031000EA01053FF51CAF24E707B0BDE8F6
:10A20000F08F0000000000002DE9F04F85B0A8B3EA
:10A210004AF200080446C4F200080068404531D004
:10A2200094F89810A9B3816921F01001816100F0C0
:10A2300043FD054620688169090705D500F03CFD0E
:10A24000401B0B28F6D310E0816941F001018161C8
:10A2500000F032FD054600BF20688169C90721D1A1
:10A2600000F02AFD401B0B28F6D3D4F89C0040F0E8
:10A270000100C4F89C00032084F89800012005B078
:10A28000BDE8F08F08F58071616094F8981000299E
:10A29000C9D1002084F89900204600F0B9F920685F
:10A2A000C1E700BF816941F002018161217C8269BF
:10A2B00022F04002012918BF40328261617C82692C
:10A2C00022F48042012908BF02F580428261A17C0C
:10A2D000826922F48052012918BF02F580528261FE
:10A2E000816921F44073D4E902120B4383618369CD
:10A2F00023F0A4038361036923F010030361AAB16F
:10A30000022A0FD0012A03D1826942F004020CE034
:10A310008369032A43F080038361036943F01002D9
:10A32000026103D1826942F020028261D4E90572A0
:10A33000E369561E6FF0FF02256A02EB0323B1F5B5
:10A34000407F43EA4663A5F1010646EA030640F270
:10A350000003CFF6FF7303EB074746EA0701C1612D
:10A3600010D1D4E90B65D4E90917013F02EB0622AD
:10A370006FF00F063A4306EB05173A4303EB014132
:10A380001143C160236E2BB1616ED0F8C020114320
:10A39000C0F8C010E16DCDE90313D9424FF670014A
:10A3A000C0F6010109D0D0F8C820A36E22F0070240
:10A3B00051F823301A43C0F8C820D4F840A0BAF1AD
:10A3C000000F09D0D0F8BC20636C22F0070251F8CE
:10A3D00023301A43C0F8BC20A76C57B1D0F8BC207A
:10A3E000E36C22F0700251F8233042EA0312C0F805
:10A3F000BC20D4F850C0BCF1000F0AD0D0F8BC206B
:10A40000636D22F4E06251F8231042EA0121C0F8A2
:10A41000BC10404504D161688A6822F003028A605A
:10A420000021C4F89410C4F89C10012184F89810FD
:10A430004FF6FC72D0F88410D4F83C9021EA020365
:10A44000656CD4E90D120292019543EA8103C0F8CC
:10A450008430D0F8843023F47F0343EA0243C0F809
:10A4600084305318D0F888606FF38F0646EA83066D
:10A47000C0F88860D0F8886003EB490326F4FE0634
:10A4800046EA0946C0F88860D0F8A0606FF38F06EE
:10A4900046EA8306C0F8A060D0F8A06005FB0A3346
:10A4A00026F4FE0646EA0A46C0F8A060D0F8B0607E
:10A4B0006FF38F0646EA8306C0F8B060D0F8B0604C
:10A4C00026F4FE0646EA0746C0F8B060E66CD0F80F
:10A4D000AC506FF38F0506FB07337E4345EA8305D7
:10A4E000C0F8AC50D4F8548008FB0C35D0F8F030EC
:10A4F0006FF38F0308FB0CFC43EA8503C0F8F030D0
:10A50000D0F8F0E0A36D2EF47C1242EA0342C0F8CA
:10A51000F02005EB4302D0F8C0506FF38F0545EAF9
:10A520008202C0F8C020D0F8C020DDF80CB022F4C0
:10A530007C1242EA0B42C0F8C020019AD0F8C05009
:10A5400025F07C5502FB0AFE4AF20002C4F200022A
:10A55000DDF810A002EB8101029A01F5406145EAA5
:10A560000A6501EB8207C0F8C05007EBC902A56E6F
:10A5700002EB8E00626700EB86060BFB05F2276795
:10A5800006EB8C07C4E91E060AFB05F007EBC303C4
:10A5900003EB8202C4F884304DF2FC33E16602EB37
:10A5A0008000C4F200039842C4F88070C4F8882088
:10A5B000C4F8900004D9D4F89C0040F0200058E67C
:10A5C000814221D20A46002042F8040BD4F8903090
:10A5D0009A4215D2486001F10802D4F890309A42AC
:10A5E0003FBF0020886001F10C02D4F8903038BFE2
:10A5F0009A4205D2C8601031D4F890209142E1D33C
:10A6000005B0BDE8F08F00BF002005B0BDE8F08FB9
:10A61000B0B5B6B0044602A8B8210025CDE934553E
:10A62000CDE932553195F6F7ACFC4DF2004120688A
:10A63000C4F20001884241D04AF20041C4F2000154
:10A64000884273D04AF20001C4F20001884240F00F
:10A65000BF80002003904FF4004002904FF08050E4
:10A660001D9002A801F0ACFE08B1FBF7F9FE41F223
:10A67000205144F2E040C2F20041C5F602000A68EF
:10A68000002A02F101020A6008D1C16841F4807118
:10A69000C160C16801F480710191019901681524BC
:10A6A00041F0080101600068132500F008000190E6
:10A6B000019803203190092133E000BF4FF400409E
:10A6C00002904FF080501D9002A8039501F078FE93
:10A6D00008B1FBF7C5FE41F2205144F2E040C2F25E
:10A6E0000041C5F602000A68002A02F101020A6070
:10A6F00008D1C16841F48071C160C16801F4807102
:10A70000019101990168A02441F0080101600068ED
:10A710009F2500F008000190052101984FF440505A
:10A72000319040F60040C5F6020038E0002003906A
:10A730004FF4004002904FF080501D9002A801F0AD
:10A740003FFE08B1FBF78CFE41F2205144F2E0409D
:10A75000C2F20041C5F602000A68002A02F10102B5
:10A760000A6008D1C16841F48071C160C16801F418
:10A770008071019101990168162441F00201016084
:10A780000068142500F002000190019860203190CB
:10A7900040F60040C5F602000921A0F500603591A1
:10A7A00031A9022232920022CDE9332200F080F951
:10A7B00005210022284600F057FB284600F044FB04
:10A7C00005210022204600F04FFB204600F03CFB14
:10A7D00036B0B0BD0000000070470000000000006F
:10A7E00010B34AF200010068C4F2000188420FD0A1
:10A7F0004DF20041C4F2000188420BD04AF2004100
:10A80000C4F20001884218BF7047012003E000BF76
:10A81000002000E0022041F22021C2F2004101EBC1
:10A820004010C06900B10047704700000000000000
:10A8300010B34AF200010068C4F2000188420FD050
:10A840004DF20041C4F2000188420BD04AF20041AF
:10A85000C4F20001884218BF7047012003E000BF26
:10A86000002000E0022041F22021C2F2004101EB71
:10A870004010406A00B1004770470000000000002F
:10A8800090F8981001290DD1022180F898100168E4
:10A890008A6922F001028A610021C0F89C100846F2
:10A8A000704700BFD0F89C1041F00401C0F89C1024
:10A8B0000120704700000000704700000000000009
:10A8C000704700000000000070470000000000001A
:10A8D000704700000000000070470000000000000A
:10A8E000704700000000000010B34AF20001006849
:10A8F000C4F2000188420FD04DF20041C4F20001C1
:10A9000088420BD04AF20041C4F20001884218BFCD
:10A910007047012003E000BF002000E0022041F268
:10A920002021C2F2004101EB4010806900B10047D4
:10A93000704700000000000010B34AF200010068F8
:10A94000C4F2000188420FD04DF20041C4F2000170
:10A9500088420BD04AF20041C4F20001884218BF7D
:10A960007047012003E000BF002000E0022041F218
:10A970002021C2F2004101EB4010406900B10047C4
:10A98000704700000000000010B34AF200010068A8
:10A99000C4F2000188420FD04DF20041C4F2000120
:10A9A00088420BD04AF20041C4F20001884218BF2D
:10A9B0007047012003E000BF002000E0022041F2C8
:10A9C0002021C2F2004101EB4010006900B10047B4
:10A9D0007047000000000000704700000000000009
:10A9E000B0B541F2E0450446C007C2F2004502D0CE
:10A9F000286800B18047A00702D5686800B1804789
:10AA0000600702D5A86800B18047200702D5E86832
:10AA100000B18047E00602D5286900B18047A00652
:10AA200002D5686900B18047600602D5A86900B107
:10AA30008047200602D5E86900B18047E00502D5CD
:10AA4000286A00B18047A00502D5686A00B1804736
:10AA5000600502D5A86A00B18047200502D5E86AE2
:10AA600000B18047E00402D5286B00B18047A00404
:10AA700002D5686B00B18047600402D5A86B00B1B5
:10AA80008047200406D5E86B002808BFB0BDBDE8AC
:10AA9000B0400047B0BD00008821C5F600010A683B
:10AAA000024208BF70470860FFF79ABF000000002D
:10AAB0002DE9F04F85B00D680290002D00F0E68082
:10AAC00002988E4600F126420A2102F1FF7342F2FB
:10AAD0000042C5F60202002490424FEAB32208BFAA
:10AAE0000921082A4FF0010738BF4FEAB321002699
:10AAF0004FF000080091CDF80CE00DE0DEF80050BA
:10AB000008F1010835FA07F006F1020607F101071E
:10AB100004F1040400F0BA80A7F1010A012000FA50
:10AB20000AF315EA0309E9D0DEF804B00BF00305D7
:10AB30006A1E012A22D802984FEA4801D0F808C0BC
:10AB40000191032101FA06F203992CEA020CD1F8D3
:10AB50000CE00EFA06F1DDF80CE041EA0C01816030
:10AB600041686FEA020CCBF3001299430346019847
:10AB700002FA0AF2114359600CE000BF0320032DD2
:10AB800000FA06F0029B6FEA000C304602D1304614
:10AB9000032526E0D968DEF8082001EA0C0182408E
:10ABA000022D41EA0201D9601BD102466FF0030079
:10ABB00000EA5A010F20194404F01C0300FA03F5BF
:10ABC0001046D1F820E0039A2EEA0505DDF80CE0E6
:10ABD00012699A40029B2A430A62DEF804B00BF025
:10ABE0000305196805FA00F001EA0C011BF4403F67
:10ABF00040EA010018603FF481AF44F2F44140F2B2
:10AC00000845C5F60201C5F600050F23086840F0A7
:10AC100002000860086800F0020004902AF00300B7
:10AC2000049904F00C0142598B409A43009B03FAAB
:10AC300001F1114341514FF0B0452868DEF804108E
:10AC400040EA0902CB0258BF20EA09028B022A60BF
:10AC500040F20405C5F60005286840EA090258BF1D
:10AC600020EA09028B032A60D5F8800040EA090235
:10AC700058BF20EA0902C903C5F88020E86F40EAFE
:10AC8000090258BF20EA0902EA6737E705B0BDE8C4
:10AC9000F08F0000000000000069084018BF01208C
:10ACA0007047000000000000002A08BF090481610D
:10ACB000704700000000000046F25800C2F2014058
:10ACC000006870470000000040F2040046F258019E
:10ACD000C2F20040C2F2014100780A6810440860E4
:10ACE000704700000000000080B5032000F0ECF881
:10ACF00002F0A6FA44F218414FF6C803C5F6020165
:10AD0000C0F601030A68096801F00F01C2F30322CB
:10AD1000595C9A5C01F01F0102F01F02D04040F222
:10AD20001002C2F2004220FA01F1116040F20C015F
:10AD3000C2F2004108600F2000F00AF800281CBF92
:10AD4000012080BD00F054F8002080BD000000000C
:10AD5000B0B58AB00F283ED80446A1200022214673
:10AD6000002500F081F8A12000F06EF840F2080004
:10AD7000C2F20040046044F2EC40C5F602000168F3
:10AD800041F080710160006801A900F080700290BC
:10AD9000029802A802F0A0F902F022FA4DF68361AF
:10ADA0004000C4F21B314EF20002A0FB010142F64A
:10ADB0007C50C2F200404FF0FF33C4F20002026048
:10ADC00003EB9141C0E9011540F2E731C0E90315F9
:10ADD00003F096FF10B101200AB0B0BD42F67C50DE
:10ADE000C2F2004003F0C0FF0AB0B0BD0000000096
:10ADF00081B044F2F4400022C5F60200016841F03F
:10AE00000201016000680F2100F0020000906FF065
:10AE10000100009B01B000F027B800000000000016
:10AE2000002848BF70474EF2801300F01F01400910
:10AE3000CEF20003012202FA01F143F82010BFF321
:10AE40004F8FBFF36F8F7047002848BF704700F0E7
:10AE50001F01012202FA01F14EF200124009CEF266
:10AE6000000242F82010704770B54EF60C5C4FF0AF
:10AE7000FF36CEF2000C00F16045DCF80030C3F381
:10AE8000022E8EF00703042B28BF0423BEF1030417
:10AE900006FA03F321EA030100F00F0338BF002490
:10AEA000043BB0F1FF3F634406FA04F003F10C03E6
:10AEB00001FA04F1C8BF05F5644322EA0000084323
:10AEC0000001187070BD00004EF60C514FF6FF03E4
:10AED000CEF200010A681A4060F30A2242F0806054
:10AEE00040F0FD70086070472DE9F04F8EB04BF2D6
:10AEF00004430022C5F200230492CDE90222059208
:10AF000045F200090692C5F20029D0F800E01A685F
:10AF1000BEEB090C02F0030018BF4FF0010C012832
:10AF200076D10120029002F03000102875D002F492
:10AF30004070B0F5807F01D10120049002F4A02080
:10AF400040F20108B0F5803FC0F200186ED19003C6
:10AF5000404658BF4FF00110059002F0A060B0F1DC
:10AF6000807F68D05A6802F0030001286ED1022069
:10AF7000029002F0300010286CD002F44070B0F55E
:10AF8000807F01D10220049002F4A020B0F5803F20
:10AF900040F20200C0F2010005D19503054648BF0A
:10AFA00008F10105059502F0A065B5F1807F05D196
:10AFB0009201024648BF08F10102069200250C9555
:10AFC000CDE90A55CDE9085553F8042C1E68D2077F
:10AFD0004FF4007204BF40F22222C0F20442F7078D
:10AFE00005D086EA0207BF073CD401250895F7067D
:10AFF0003BD586EA0207BF0637D44FF0010BCDF8E8
:10B0000024B006F44077B7F5407F37D134E000BF75
:10B0100002F0300010287FF48AAF0120039002F480
:10B020004070B0F5807F3FF487AF87E702F0A06003
:10B03000B0F1807F96D19001404658BF4FF001108B
:10B0400006905A6802F00300012890D002F0300008
:10B05000102892D10220039002F44070B0F5807F56
:10B0600090D091E70025F706C3D44FF0000B06F40B
:10B070004077B7F5407F01D101270A97F7030DD537
:10B0800086EA02077F0309D4B70319D44FF0011AE7
:10B09000CDF82CA0F70118D504E000BF4FF0000A4E
:10B0A000F70112D586EA02077F010ED4B70141D419
:10B0B0004FF001140C945F68FE070AD10FE000BF47
:10B0C000CDF82C80C246F701ECD400245F68FE075F
:10B0D00005D087EA0206B60701D402250895FE06C8
:10B0E00007D587EA0206B60603D44FF0020BCDF867
:10B0F00024B007F44076B6F5407F01D102260A96C7
:10B10000FE0307D587EA0206760303D4BE0319D4EB
:10B1100082460B90FE011BD57A40520118D4BA0129
:10B120001ED404460C90D9F80000C007AEEB09000D
:10B1300014D01EE0CDF8308044465F68FE07CED0C4
:10B14000C7E700BF08F1010ACDF82CA0FE01E3D447
:10B15000D9F80000C007AEEB09000AD100220FE0C9
:10B1600008F101040C94D9F80000C007AEEB090007
:10B17000F4D0D9F8002022F00102C9F80020012201
:10B180004AF200060192B0FA80F7C5F20026D046D6
:10B19000CA463268CDF800E0D207A646484606D037
:10B1A000306820F0010030600198023001900CEB13
:10B1B0004C000DF108097F0909EBC006B26803EBEA
:10B1C000820252F804CC2CF4807442F8044C53F8F8
:10B1D000042CD2072AD159F8300000285BD003EBA9
:10B1E000800050F8042C22F0010240F8042C706812
:10B1F00038B103EB800050F8042C22F0100240F824
:10B20000042CF06840B1012222EA000053F820200B
:10B2100022F4803243F820203069E0B3012222EA90
:10B22000000053F8202022F0807232E053F8040C22
:10B23000009A524520F0010043F8040C2BD103EB97
:10B240008500BBF1000F50F8042C42F0020240F8D8
:10B25000042C07D003EB8B0050F8042C42F02002A2
:10B2600040F8042CB8F1000F08D0012020EA0800B3
:10B2700053F8202042F4802243F82020BEF1000F32
:10B2800009D00120724620EA0E0053F8202042F037
:10B29000806243F8202007EB4705086859F83560BD
:10B2A00009EBC502B04215D148685768B842DDF8CD
:10B2B00000E034D1CF68D468A7422FD10F6912695A
:10B2C000974207462BD153F8040C40F0010043F895
:10B2D000040C57E088689768B84203D15768DDF8D6
:10B2E00000E01CE04868576860B1B8420AD103EB3F
:10B2F000860252F8047C27F0010742F8047CDDF84E
:10B3000000E016E0C868D468A042DDF800E006D08E
:10B3100008691269904202D034E000BF074603EB8F
:10B32000860050F8042C22F0010240F8042C384624
:10B330003FB103EB800050F8042C22F0100240F8DB
:10B34000042C09EBC500826803EB820252F8047CEE
:10B3500027F4807742F8047CC26842B1012727EACB
:10B36000020253F8227027F4803743F822700069F4
:10B3700040B1012222EA000053F8202022F080721E
:10B3800043F8202088684FF44072D64503EB8000D4
:10B3900050F8047C08BF4FF4807227F440773A4499
:10B3A00040F8042C486953F8042C471EC2F30742A6
:10B3B00097420BD9002753F8042CCFF6FF7722F4DD
:10B3C0007F0207EB0040104343F8040C53F8042CB1
:10B3D000086801384AF20005D207C5F2002553F883
:10B3E000207027F003022BD10327D64508BF012781
:10B3F0003A4343F82020486860B103EB80003022D4
:10B40000D64550F8047C08BF102227F020073A43A5
:10B4100040F8042CC868C2032AD4019ED0B301228C
:10B42000D64522EA000053F8202003EB80044FF0B9
:10B43000A06022F0E06208BF4FF0807028E000BFFB
:10B4400042F0010243F82020486840B103EB80003D
:10B45000012750F8042C67F3051240F8042CC86843
:10B46000C20329D4A8B34FF080726FF0E06727E0E1
:10B470000122D64522EA000003EB800453F8202085
:10B480004FF4A02022F4E02208BF4FF48030019E48
:10B49000104320600869C1032AD4C8B30121D645EE
:10B4A00021EA00004FF0E06153F8202022F0E06232
:10B4B00008BF4FF0407128E04FF480326FF4E0276E
:10B4C000012626EA000053F8206037403A4343F84B
:10B4D00020200869C10323D4019EC8B101210322A1
:10B4E00021EA000053F8201062F31A610EE000BF59
:10B4F0000121D64521EA00004FF4E02153F8202035
:10B5000008BF4FF4403122F4E022114443F82010E8
:10B51000F00712D1B00718D400200EB0BDE8F08FAC
:10B520000121032221EA000053F8201062F31241A6
:10B5300043F82010019EF007ECD0DAF8000040F04C
:10B540000100CAF80000B007E6D5286840F0010005
:10B55000286000200EB0BDE8F08F00000000000061
:10B56000F0B581B00446FFF7A7FB002C00F08980FE
:10B57000054600206065216D11B101B0F0BD00BF2E
:10B58000204600F081F8206841F28836A6654FF623
:10B59000F40ED4E903C263698168CFF6E00E002798
:10B5A000CFF6FF7701EA0E0107EB024241EA0C01F8
:10B5B0006FF0FF0E676B11430EEB03223943E36913
:10B5C000114319438160C168226A21F4E0211143CB
:10B5D000C160216BA26B42EA01410161E16B4161F3
:10B5E0000168626821F4F8510EEB022211430160F8
:10B5F000016A890609D500BFFFF75EFB401BB04218
:10B6000038D82068016A8906F6D4C168A268D4E9EE
:10B61000097621F0FF01013FA3693943C160022B84
:10B62000016821F0400141EA02010160D0F80811EF
:10B63000E26A21F0A04141EA060141EA0201C0F8B4
:10B640000811016841F00101016003D1816841F0F6
:10B6500002018160E068B0F1806F05D101202065B2
:10B66000002001B0F0BD00BF02202065002001B025
:10B67000F0BD00BF4FF400702065606D40F0010028
:10B680006065012001B0F0BD2DE9F04FB5B0044672
:10B6900002A80830B02100253095CDE93355CDE919
:10B6A0003155F5F76EFC45F200012068C5F2002126
:10B6B000884203D035B0BDE8F08F00BF4FF0007076
:10B6C000029002A80395159500F07AFE08B1FAF7EA
:10B6D000C7FE44F2E04040F20008C5F60200C5F69D
:10B6E000020830AC022750F80C1C4FF0000941F45E
:10B6F000001140F80C1C50F80C1C4FF0030B01F427
:10B7000000110191019950F80C1C41F4804140F85E
:10B710000C1C50F80C1C4FF0090A01F480410191F7
:10B720000199016841F001010160016801F0010126
:10B7300001910199016841F002010160016801F085
:10B74000020101910199016841F010010160016855
:10B7500001F0100101910199016841F008010160B7
:10B760000068214600F00800019001984046CDE9AC
:10B770003077CDF8C890CDF8CCB0CDF8D0A0FFF799
:10B7800097F930A9082081E8810A062034904046C4
:10B790002146FFF78DF930A9012008F580660425C0
:10B7A00081E8810A304621463495FFF781F930A8B7
:10B7B0002146CDF8D0A080E8A00A3046FFF778F9FE
:10B7C00030A84FF40065214680E8A00A0B20349091
:10B7D00008F58050FFF76CF930A82146CDF8D0A0CD
:10B7E00080E8A00A08F54060FFF762F935B0BDE8CF
:10B7F000F08F00000000000001680122C0F8D8248A
:10B80000002280F8CC24886940F000608861486D8F
:10B8100040F08052002042F003024A657047000069
:10B82000F0B581B0002800F02781044690F8950417
:10B8300028B9002084F89404204600F035F903204C
:10B8400084F8950420680DF0C7F9D4E90001267C3E
:10B85000D4E9022300960CF0FFFE002840F0098195
:10B86000206800210DF0C0F9002840F00281217904
:10B87000002900F0F580A1F1010C01F0030EBCF1EC
:10B88000030F4FF0000345D301F0FC0204F19A00CE
:10B890000126002500F8865C6F1C20F86C5C00F81F
:10B8A000627C20F8487CAF1C00F83E7C20F8247CA9
:10B8B000EF1C043500F8856C00F8823CAA4240F881
:10B8C0007E3C40F87A3C40F8763C00F8616C00F829
:10B8D0005E3C40F85A3C40F8563C40F8523C00F878
:10B8E0003D6C00F83A3C40F8363C40F8323C40F8B9
:10B8F0002E3C00F8196C00F81A7C078000F8163C02
:10B9000040F8123C40F80E3C40F80A3C00F1900030
:10B91000C0D12B46BEF1000F2DD003EBC300012296
:10B92000BEF1010F04EB80054FF000006A752B7526
:10B93000EB852876C5E9070068621CD05D1CBEF166
:10B94000020F05EBC50604EB860672753575F585A5
:10B950003076C6E9070070620DD0981C012300EB19
:10B96000C00204EB820253751075D085002010765A
:10B97000C2E907005062BCF1030F4FF0000237D359
:10B9800001F0FC0004F53471002300BF01F87C3C99
:10B990005F1C01F8587C9F1C01F8347CDF1C0433C9
:10B9A00001F87B2C01F8782C984241E91D2241F8DE
:10B9B0006C2C01F8572C01F8542C41E9142241F861
:10B9C000482C01F8332C01F8302C41E90B2241F8C6
:10B9D000242C01F80F2C01F8107C01F80C2C41F8F4
:10B9E000082C41F8042C0A6001F19001CED11A46CE
:10B9F000BEF1000F34D002EBC200BEF1010F04EB28
:10BA000080014FF0000081F8550281F8542281F83E
:10BA10005802C1E99700C1F8640221D0511CBEF15F
:10BA2000020F01EBC10304EB830383F8550283F893
:10BA3000541283F85802C3E99700C3F864020FD088
:10BA4000901C002200EBC00104EB810181F855221B
:10BA500081F8540281F85822C1E99722C1F8642282
:10BA6000D4E90001277CD4E9022300970CF01CFFE5
:10BA700030B1022084F89504012001B0F0BD00BF70
:10BA800000206074012084F89504207B012802D1F5
:10BA90002046FFF7B1FE20680CF0F6FE002001B052
:10BAA000F0BD00000000000010B5B0B002A90446CF
:10BAB00001F10800B021F5F764FA00212068C4F212
:10BAC0000401884202D030B010BD00BF00200390B6
:10BAD0004FF4802002904FF44010239002A800F011
:10BAE0006FFC08B1FAF7BCFC00F03AF844F2D84019
:10BAF000C5F60200016841F000710160006800F0C5
:10BB000000700190019830B010BD000000000000EE
:10BB1000B0B544F60C05C5F6020529684907296841
:10BB200006D401F00701081A18BF0120B0BD00BFFC
:10BB300021F0070108432860FFF7BEF8044600BF64
:10BB400055F8080C800407D4FFF7B6F8001BB0F5D1
:10BB50007A7FF5D90120B0BD0020B0BD0000000003
:10BB600044F60C00C5F60200016841F080710160E6
:10BB7000704700000000000080B501F0D9FA44F2DF
:10BB800020414FF6C802C5F60201C0F6010209685D
:10BB9000C1F30211515C01F01F01C84080BD0000DB
:10BBA00080B544F2304EC5F6020E5EF8083C5EF8F1
:10BBB000081CC1F3051C5EF8041CBCF1000FDEF884
:10BBC000042017D0C2F3CC0201F00101514303F06D
:10BBD0000303022B00EE101AB8EE400A10D0012B1E
:10BBE00012D01BB95EF8301C890611D49FED361AAD
:10BBF0001CE000BF00218160C0E9001180BD00BFD2
:10BC00009FED301A12E000BF9FED2D1A0EE000BF2D
:10BC10005EF8301C49F20002C0F2D032C1F3C1011B
:10BC200022FA01F101EE101AB8EE411ADEF8001006
:10BC30009FED263A6FF35F2102EE101ADEF8001036
:10BC4000C1F34621B8EE422A00EE032A00EE10CAE4
:10BC5000B7EE003AB8EE400A81EE000A32EE031A5F
:10BC600002EE101AB8EE422A20EE010A32EE031A52
:10BC700080EE011ABCEEC11A80ED001ADEF8001049
:10BC8000C1F3064101EE101AB8EE411A31EE031A63
:10BC900080EE011ABCEEC11A80ED011ADEF8001028
:10BCA000C1F3066101EE101AB8EE411A31EE031A23
:10BCB00080EE010ABCEEC00A10EE101A816080BD51
:10BCC0000024744A001BB74B0024744C0000003958
:10BCD00080B544F2384EC5F6020E5EF8103C5EF8B0
:10BCE000101CC1F3053C5EF80C1CBCF1000FDEF823
:10BCF000042015D0C1F30011C2F3CC02514300EE71
:10BD0000101A03F003010229B8EE400A0ED089B9D7
:10BD10005EF8381C890611D49FED361A1CE000BF6E
:10BD200000218160C0E9001180BD00BF9FED301A85
:10BD300012E000BF9FED2D1A0EE000BF5EF8381C28
:10BD400049F20002C0F2D032C1F3C10122FA01F17E
:10BD500001EE101AB8EE411ADEF800109FED263AF7
:10BD60006FF35F2102EE101ADEF80010C1F34621D6
:10BD7000B8EE422A00EE032A00EE10CAB7EE003AEF
:10BD8000B8EE400A81EE000A32EE031A02EE101AF3
:10BD9000B8EE422A20EE010A32EE031A80EE011AB2
:10BDA000BCEEC11A80ED001ADEF80010C1F30641A6
:10BDB00001EE101AB8EE411A31EE031A80EE011AA4
:10BDC000BCEEC11A80ED011ADEF80010C1F3066165
:10BDD00001EE101AB8EE411A31EE031A80EE010A94
:10BDE000BCEEC00A10EE101A816080BD0024744AB7
:10BDF000001BB74B0024744C000000390000000009
:10BE000080B544F2404EC5F6020E5EF8183C5EF86E
:10BE1000181CC1F3055C5EF8141CBCF1000FDEF8C1
:10BE2000042015D0C1F30021C2F3CC02514300EE2F
:10BE3000101A03F003010229B8EE400A0ED089B9A6
:10BE40005EF8401C890611D49FED361A1CE000BF35
:10BE500000218160C0E9001180BD00BF9FED301A54
:10BE600012E000BF9FED2D1A0EE000BF5EF8401CEF
:10BE700049F20002C0F2D032C1F3C10122FA01F14D
:10BE800001EE101AB8EE411ADEF800109FED263AC6
:10BE90006FF35F2102EE101ADEF80010C1F34621A5
:10BEA000B8EE422A00EE032A00EE10CAB7EE003ABE
:10BEB000B8EE400A81EE000A32EE031A02EE101AC2
:10BEC000B8EE422A20EE010A32EE031A80EE011A81
:10BED000BCEEC11A80ED001ADEF80010C1F3064175
:10BEE00001EE101AB8EE411A31EE031A80EE011A73
:10BEF000BCEEC11A80ED011ADEF80010C1F3066134
:10BF000001EE101AB8EE411A31EE031A80EE010A62
:10BF1000BCEEC00A10EE101A816080BD0024744A85
:10BF2000001BB74B0024744C0000003900000000D7
:10BF300010B584B0024641F6FF7300209B1A70EBE7
:10BF400001032DDA47F6FF739B1A70EB010380F2B1
:10BF5000798082F400430B4300F0A08082F48033A8
:10BF60000B4300F0E38082F40022114340F01E8175
:10BF700044F20040C5F60200816D01F44031B1F594
:10BF8000003F00F01F81B1F5803F00F0FD800029E7
:10BF900040F0E1810068000100F17D81DBE100BF3C
:10BFA00040F2FF739B1A70EB010325DB82F4807370
:10BFB0000B4300F0878082F48062114340F0F680EA
:10BFC00044F20041C5F60201886DC0F34252042AD2
:10BFD00000F2C18148F20000C0F2BB00DFE812F0BD
:10BFE000060000010601E6000C0100BF08688001A0
:10BFF00040F1B181E0E000BF82F400630B4300F048
:10C000007B8082F48052114340F0D08044F20041A2
:10C01000C5F60201086DC0F30232042A00F29B81CA
:10C0200048F20000C0F2BB00DFE812F00600F800A2
:10C03000FE00C000040100BF0868800140F18B8150
:10C04000BAE000BF82F400530B4300F07B8082F41F
:10C050008042114340F0AA8044F20044C5F6020435
:10C06000A06DC0F30270052800F27581DFE810F0C2
:10C070000600420146014A015001520101F058F800
:10C08000216A4FF6C802C0F60102C1F30211515CE9
:10C0900001F01F01C84004B010BD00BF44F20040D1
:10C0A000C5F60200016D01F04051B1F1005F00F0F2
:10C0B0007580B1F1805F00F07B80002940F04B81FA
:10C0C00060E000BF44F20041C5F60201086D00F0D7
:10C0D0000702042A00F23F8148F20000C0F2BB00D0
:10C0E000DFE802F004BAC064C40000BF0868800141
:10C0F00040F1318160E000BF44F20041C5F6020129
:10C10000886DC0F30262042A00F2258148F2000023
:10C11000C0F2BB00DFE802F004BCC64AD00000BF9A
:10C120000868800140F1178146E000BF44F20040FA
:10C13000C5F60200C16C0068C90319D4800140F142
:10C140000A8139E044F20040C5F60200016DC1F3F6
:10C150000241052900F2FF80DFE811F00600E60049
:10C16000F000FA000001140001F00AF804B010BD5C
:10C17000000140F1F08001A8FFF7AAFD039804B088
:10C1800010BD00BF0068C6E00068800040F1E38099
:10C1900001A8FFF735FE039804B010BD0068000148
:10C1A00040F1D98001A8FFF793FD029804B010BDBB
:10C1B0000068800140F1CF8001A8FFF7F1FC0298F0
:10C1C00004B010BDC16C036811F04051026840F02A
:10C1D000CF8013F0040300F0CB80C2F3C100D6E09F
:10C1E0000868000140F1B78055E000BF0868800092
:10C1F00040F1B18059E000BFC86C0B6810F04052AC
:10C20000086803D113F0040340F0BF80B2F1805FEF
:10C2100061D110F4807040F0B1805CE008680001EA
:10C2200040F1998037E000BF0868800040F19380BA
:10C230003BE000BFC86C0B6810F04052086803D1A7
:10C2400013F0040340F0A180B2F1805F43D110F4F9
:10C25000807040F093803EE00868000140F17B80F0
:10C2600019E000BF0868800075D51EE0C86C0B6837
:10C2700010F04052086803D113F0040340F08580A9
:10C28000B2F1805F27D110F4807077D123E000BF36
:10C29000086800015FD501A8FFF71AFD019804B0F6
:10C2A00010BD00BF0868800055D501A8FFF7A8FDA4
:10C2B000019804B010BD00BFC86C0B6810F040526C
:10C2C000086802D113F004035FD1B2F1805F02D19C
:10C2D00010F4807052D1086810F400301CBF43F293
:10C2E0000060C0F26E10B2F1005F18BF002004B011
:10C2F00010BD00BF206800012DD518E02068800027
:10C3000029D51EE02068400725D520683DE000BF04
:10C31000206824E0206843F200618003C0F26E11BF
:10C3200001EAE07004B010BD0068000113D501A857
:10C33000FFF7CEFC029804B010BD00BF006880007B
:10C3400009D501A8FFF75CFD029804B010BD00BF3D
:10C350000168490718D4002004B010BD006840F6F9
:10C360000011C005C0F23D0101EAE07004B010BD4B
:10C37000B1F1805F14D112F4807211D040F6001038
:10C38000C0F23D0004B010BD0068C0F3C10049F226
:10C390000001C0F2D03121FA00F004B010BD00BF9E
:10C3A000006810F400301CBF43F20060C0F26E1051
:10C3B000B1F1005F18BF002004B010BD0000000004
:10C3C0002DE9F0470446C07844F22C480007C5F632
:10C3D000020833D5606E4FEA305103290CD8DFE8EC
:10C3E00001F003111D2600BFD8F8001041F4003100
:10C3F000C8F800101BE000BF01266078C0070BD012
:10C4000020E000BF04F10800022108F0BDFB064651
:10C4100060B16078C00715D1354646E004F12800C8
:10C42000022108F045FC06460028F2D1606ED8F8DB
:10C43000241021F440110843C8F824000026607835
:10C44000C007E9D0A06D04280ED83546DFE800F01B
:10C450000412181E1E0000BFD8F80000354640F434
:10C460000030C8F8000011E001250127607840077E
:10C470001FD453E004F10800002108F085FB04E01C
:10C4800004F12800002108F013FC05462F461DB1D9
:10C49000607840070DD441E0D8F82400A16D20F069
:10C4A000070000250843C8F8240037466078400795
:10C4B00034D5D4F8A4004FEA705005280CD8DFE832
:10C4C00000F00311171D1D1DD8F8000040F40030C6
:10C4D000C8F8000012E000BF0125012660780007BF
:10C4E00020D455E004F10800002108F04DFB04E0E1
:10C4F00004F12800002108F0DBFB05462E461DB1A3
:10C50000607800070ED443E0D8F82C00D4F8A410CB
:10C5100020F4600000250843C8F82C003E466078EF
:10C52000000735D5D4F8A8004FEA306005280DD8AB
:10C53000DFE800F00412181E1E1E00BFD8F800002D
:10C5400040F40030C8F8000012E000BF01250127C8
:10C55000E078800720D44EE004F10800002108F0C4
:10C5600013FB04E004F12800002108F0A1FB0546BC
:10C570002F461DB1E07880070ED43CE0D8F82C009F
:10C58000D4F8A81020F0E06000250843C8F82C007B
:10C590003746E07880072ED5E06C4FEA301003284C
:10C5A0000ED8DFE800F00903130900BFD8F8000037
:10C5B00040F40030C8F800002E467DB912E000BFFC
:10C5C000012501266078C00619D44CE004F108006A
:10C5D000022108F0D9FA05462E461DB16078C00642
:10C5E0000DD440E0D8F82000E16C20F030000025A8
:10C5F0000843C8F820003E466078C00633D5E06D99
:10C600004FEA303004280DD8DFE800F00412181E7D
:10C610001E0000BFD8F8000040F40030C8F8000049
:10C6200012E000BF01250127607880061FD44EE08C
:10C6300004F10800002108F0A7FA04E004F1280042
:10C64000002108F035FB05462F461DB160788006B5
:10C650000DD43CE0D8F82400E16D20F4E040002542
:10C660000843C8F824003746607880062FD5206E2E
:10C670004FEA3040052809D8DFE800F0040E140422
:10C68000040400BF2E46ADB918E000BF0125012605
:10C69000607840061FD44FE004F10800012108F043
:10C6A00073FA04E004F12800012108F001FB0546BB
:10C6B0002E461DB1607840060DD43DE0D8F8240028
:10C6C000216E20F4E02000250843C8F824003E46EF
:10C6D0006078400630D5D4F8AC004FEA30700528B9
:10C6E00008D8DFE800F0030D130303032F46ADB9AC
:10C6F00018E000BF012501276078000620D442E041
:10C7000004F10800012108F03FFA04E004F12800D8
:10C71000012108F0CDFA05462F461DB160780006CC
:10C720000ED430E0D8F82C00D4F8AC1020F0E04063
:10C7300000250843C8F82C0037466078000622D54B
:10C74000E06E58B1B0F1005F0CD0B0F1805F2FD136
:10C75000D8F8000040F40030C8F800002E469DB91B
:10C7600008E000BF04F10800012108F00DFA0546B9
:10C770002E464DB9D8F82400E16E20F04050002537
:10C780000843C8F824003E46E078C00733D0A06CC8
:10C79000032813D8DFE800F008021A08D8F80000D0
:10C7A00040F40030C8F80000A946BDB91AE000BF47
:10C7B00001250126E078C007E9D11CE001254FF0F2
:10C7C0000109A07840061AD51CE000BF04F108005A
:10C7D000022108F0D9F90546A9461DB1A078400606
:10C7E0000DD50FE0D8F82000A16C20F00300002543
:10C7F0000843C8F82000B146A078400602D44F464E
:10C8000018E000BFD8F8D40340F48070C8F8D4030F
:10C81000FEF752FA064600BFD8F8D403C00507D485
:10C82000FEF74AFA801B6428F6D90325032701E0A6
:10C830002F468DB12078C00761D0A06F4FEAF0007D
:10C8400005283BD8DFE800F004404604040400BF9C
:10C85000002D2E4646D149E0D8F84410D4F8B00057
:10C86000414011F4407F11D0D8F84410D8F844204A
:10C8700042F48032C8F84420D8F8442021F44071B2
:10C8800022F48032C8F84420C8F84410B0F5807F04
:10C8900040F0D082FEF710FA064641F2883A0325AE
:10C8A000032700BFD8F84400800700F1C182FEF7DB
:10C8B00003FA801B5045F5D9BCE700BF01250126CE
:10C8C000207880071FD44CE004F10800012108F013
:10C8D0005BF904E004F12800012108F0E9F90546BC
:10C8E0002E461DB1207880070DD43AE0D8F82800F4
:10C8F000A16F20F0380000250843C8F828003E4604
:10C90000207880072DD5606F052809D8DFE800F072
:10C91000040E1404040400BF2F46ADB918E000BF94
:10C9200001250127207840071FD44DE004F10800BD
:10C93000012108F029F904E004F12800012108F0A0
:10C94000B7F905462F461DB1207840070DD43BE0CE
:10C95000D8F82800616F20F0070000250843C8F8C8
:10C9600028003746207840072ED5D4F890000528B7
:10C9700008D8DFE800F0030D130303032E46ADB91A
:10C9800018E000BF012601252078800620D451E060
:10C9900004F10800012108F0F7F804E004F1280090
:10C9A000012108F085F905462E461DB12078800644
:10C9B0000ED43FE0D8F82C00D4F8901020F00700F7
:10C9C00000250843C8F82C003E462078800631D563
:10C9D000D4F88C004FEA3070052809D8DFE800F061
:10C9E000040E1404040400BF2F46ADB918E000BFC4
:10C9F000012701252078400620D451E004F10800E9
:10CA0000002108F0C1F804E004F12800022108F038
:10CA10004FF905462F461DB1207840060ED43FE061
:10CA2000D8F82800D4F88C1020F0E0400025084306
:10CA3000C8F8280037462078400631D5D4F8980049
:10CA40004FEAB020052809D8DFE800F0040E1404EE
:10CA5000040400BF2E46ADB918E000BF0126012531
:10CA60002078000620D454E004F10800002108F0EA
:10CA70008BF804E004F12800022108F019F90546BA
:10CA80002E461DB1207800060ED442E0D8F82C00C6
:10CA9000D4F8981020F4E05000250843C8F82C0082
:10CAA0003E462078000634D5D4F89C004FEA70301A
:10CAB00005280FD8DFE800F004141A04040400BFAE
:10CAC0002F46E5B12068010727D4C1063ED40003F4
:10CAD00055D475E00127012520680107F5D51CE034
:10CAE00004F10800002108F04FF804E004F12800E8
:10CAF000022108F0DDF80546002D2F46E2D1D8F8D6
:10CB00002C00D4F89C1020F4604000250843C8F89D
:10CB10002C00374620680107D7D5D4F88010B1F52E
:10CB2000805F0AD104F12800022108F0C1F8002832
:10CB300018BF01272068D4F88010D8F8282022F4E4
:10CB400040521143C8F82810C106C0D5D4F894103B
:10CB5000B1F5807F0AD104F12800022108F0A8F87D
:10CB6000002818BF01272068D4F89410D8F82C208A
:10CB700022F440721143C8F82C10000320D5D4F8D9
:10CB8000A000B0F5003F0FD0B0F5803F06D078BBD5
:10CB900004F10800002107F0F7FF04E004F1280089
:10CBA000022108F085F805462E4655B9D8F82C0024
:10CBB000D4F8A01020F4403000250843C8F82C0019
:10CBC0003E46A07840072BD5D4F88400B0F5401F2E
:10CBD0000BD0B0F5001F11D0B0F5801F2AD1D8F8C6
:10CBE000000040F40030C8F800002F46CDB90DE039
:10CBF00001260125A0784007E6D411E004F12800C1
:10CC0000012108F055F805462F4655B9D8F82800F7
:10CC1000D4F8841020F4401000250843C8F82800F8
:10CC20003746A078C0070AD13E462168880016D54D
:10CC300033E000BF01270125A078C007F4D0206DA4
:10CC4000B0F5803F10D018BBD8F8000040F4003099
:10CC5000C8F800002E4685B1216888001DD46068A0
:10CC60008A0326D467E000BF04F10800022107F020
:10CC70008BFF0546002D2E46EED1D8F82000216D01
:10CC800020F4803000250843C8F82000CCE700BF1E
:10CC90000126012521688800E1D504F12800022140
:10CCA00008F006F8002818BF0126D4E900108A030E
:10CCB00041D5E26F6FF0010303EB3223022B0BD35C
:10CCC0004FEA322343B1012B40F0AC80D8F800305A
:10CCD00043F40033C8F8003035B3CA022ED48A02B8
:10CCE00036D44A003ED4B1F1FF3F4BDD090253D4A4
:10CCF000C1075CD1810765D441076ED4010778D4A0
:10CD0000C10600F18280800607D504F128000221C7
:10CD100007F0CEFF002818BF0125002D18BF012500
:10CD20002846BDE8F08700BFD8F8283023F44073C8
:10CD30001A43C8F828203546CA02D0D5D8F824208E
:10CD4000236F22F000421A43C8F824208A02C8D573
:10CD5000D8F82420A36E22F080721A43C8F8242049
:10CD60004A00C0D558F81C2C22F4004248F81C2C6C
:10CD7000D4F8B42058F81C3C1A4348F81C2CB1F1E4
:10CD8000FF3FB3DCD8F82020636D22F040521A43F5
:10CD9000C8F820200902ABD5D8F82810D4F888208C
:10CDA00021F440011143C8F82810C107A2D004F1B2
:10CDB0000800002107F0E8FE002818BF054660685B
:10CDC000810799D504F10800012107F0DDFE002854
:10CDD00018BF05466068410790D504F1080002219C
:10CDE00007F0D2FE002818BF0546606801077FF5EE
:10CDF00087AF04F12800002107F05AFF002818BF70
:10CE000005466068C1067FF57EAF04F12800012168
:10CE100007F04EFF002818BF0546606880067FF5C2
:10CE20007CAF72E70125CA027FF559AF86E700BFE4
:10CE3000D4F8B0004FF6CF7358F81C2CC0F2FF03A3
:10CE400000F4407122F47C5203EA10136FF31F3098
:10CE5000B1F5407F08BF1A43002548F81C2CD8F8CC
:10CE600044100843C8F84400FFF7C9BC00000000A4
:10CE70002DE9F04381B0002800F02A8142F2000839
:10CE80000446C5F200288946D8F8000000F00F00DB
:10CE900088420ED2D8F8000020F00F0040EA0900C6
:10CEA000C8F80000D8F8000000F00F00484540F036
:10CEB0000F81206844F218474107C5F602070AD5DA
:10CEC00021693A6802F07002914204D93A6822F06E
:10CED00070021143396001070AD561697A6802F06E
:10CEE0007002914204D97A6822F07002114379608D
:10CEF000C1060AD5A1697A6802F4E062914204D9B8
:10CF00007A6822F4E0621143796081060AD5E1690A
:10CF1000BA6802F07002914204D9BA6822F0700235
:10CF20001143B96010F002010AD0E2683B6803F0D7
:10CF30000F039A4204D93B6823F00F031A433A6067
:10CF4000C20746D0386820F47061D4E90102012894
:10CF500041EA0201396009D003280DD0022811D11D
:10CF600057F8181C890340F1B38010E057F8181CDB
:10CF7000C90540F1AD800AE057F8181C890140F15D
:10CF8000A78004E057F8181C490740F1A18057F822
:10CF9000081C21F00701084347F8080CFDF78CFE38
:10CFA000064641F2883500BF57F8080C616800F06A
:10CFB0003800B0EBC10F09D0FDF77EFE801BA84200
:10CFC000F2D9032001B0BDE8F08300BF206800F073
:10CFD000020151B1E1683A6802F00F02914204D2B5
:10CFE0003A6822F00F0211433960D8F8001001F0BE
:10CFF0000F0149450DD9D8F8001021F00F0141EA81
:10D000000901C8F80010D8F8001001F00F014945D7
:10D010005ED141070AD521693A6802F07002914257
:10D0200004D23A6822F070021143396001070AD530
:10D0300061697A6802F07002914204D27A6822F043
:10D04000700211437960C1060AD5A1697A6802F4B9
:10D05000E062914204D27A6822F4E062114379607E
:10D0600080060AD5E069B96801F07001884204D2EF
:10D07000B96821F070010843B86000F0E1F8396840
:10D080004FF6C8033A68C0F60103C1F3032102F06A
:10D090000F02595C9A5C01F01F0120FA01F102F0C5
:10D0A0001F0040F2100221FA00F0C2F200421060AC
:10D0B00040F2080040F20C02C2F20040C2F200420C
:10D0C0000068116001B0BDE8F043FDF741BE00BF4C
:10D0D000012001B0BDE8F0833F22026044F2184213
:10D0E000C5F6020252F8083C03F0070343601368D8
:10D0F00003F470638360136803F00F03C360136865
:10D1000003F070030361536803F0700343615368D5
:10D1100003F4E0638361926802F07002C26142F23C
:10D120000000C5F20020006800F00F0008607047A2
:10D1300080B500F085F844F218414FF6C803C5F6F3
:10D140000201C0F601030A68096801F00F01C2F389
:10D150000322595C9A5C02F01F0220FA02F201F0ED
:10D160001F0040F2100122FA00F0C2F200410860F4
:10D1700040F20C01C2F200410A6080BD00000000D4
:10D1800080B500F05DF844F2184C4FF6C801C5F6C2
:10D19000020CC0F60101DCF80020DCF8003003F0DE
:10D1A0000F03C2F30322CB5C8A5C02F01F02D04063
:10D1B00003F01F0240F2100320FA02F2C2F2004311
:10D1C0001A6040F20C03C2F200431860DCF804005D
:10D1D000C0F30210085C00F01F0022FA00F080BDCE
:10D1E00080B500F02DF844F2184C4FF6C801C5F692
:10D1F000020CC0F60101DCF80020DCF8003003F07E
:10D200000F03C2F30322CB5C8A5C02F01F02D04002
:10D2100003F01F0240F2100320FA02F2C2F20043B0
:10D220001A6040F20C03C2F200431860DCF80400FC
:10D23000C0F30220085C00F01F0022FA00F080BD5D
:10D2400044F20041C5F602010869C0F3C200032898
:10D2500010D002282CD088BB0868800649F2000054
:10D26000C0F2D03058BF70470968C1F3C101C8404F
:10D27000704700BF8A6A886AC0F3051CC86ABCF19F
:10D28000000F4B6B20D0C3F3CC0300F001005843D8
:10D2900002F00302022A00EE100AB8EE400A15D08E
:10D2A000C2B90868800619D49FED281A23E000BF90
:10D2B00043F20060C0F26E10704700BF40F60010ED
:10D2C000C0F23D00704700BF002070479FED1E1A5E
:10D2D00011E000BF9FED1B1A0DE000BF086849F286
:10D2E0000002C0F2D032C0F3C10022FA00F001EE19
:10D2F000100AB8EE411A086B9FED153A6FF35F20E4
:10D3000002EE100A086BC0F34620B8EE422A013044
:10D3100000EE032A00EE10CAB7EE003AB8EE400A5B
:10D3200081EE000A32EE031A20EE010A01EE100A25
:10D33000B8EE411A80EE010ABCEEC00A10EE100AE7
:10D34000704700BF0024744A001BB74B0024744C84
:10D35000000000390000000070B586B0002844F2DB
:10D36000E04640F2000014460D46C5F60206C5F63A
:10D3700002001DD0316800F5006041F00401316009
:10D38000316801F00401019101994FF4007101919C
:10D39000022102910321049100210391059101A929
:10D3A000FDF786FB56F8D00CE40120F07E4019E032
:10D3B000316841F001013160316801F001010191F2
:10D3C00001994FF48071019102210291032104918E
:10D3D00000210391059101A9FDF76AFB56F8D00CD5
:10D3E00020F0FE7044EA0501084346F8D00C06B070
:10D3F00070BD000000000000F0B581B0002800F012
:10D40000D5800446007844F20046C007C5F60206FF
:10D4100022D12078800768D5306910F03801B06AD1
:10D4200042D0182908BF5FEA80703DD0E0683168BB
:10D43000002800F0258121F0190108433060FDF734
:10D440003BFC05463068400748D4FDF735FC401BDF
:10D450000228F7D977E100BF306900F03801B06ADF
:10D46000102905D018290BD100F00300022807D19C
:10D4700030688003CDD560680028CAD196E000BF2F
:10D480006068002800F03281B0F5A02F00F04681DE
:10D49000B0F5803F00F04681306820F48030306085
:10D4A000306820F4802040E130684007E06801D512
:10D4B00000287BD0316821F0190108433060FDF766
:10D4C000FBFB05463068400708D4FDF7F5FB401B21
:10D4D00002284FF00300F5D901B0F0BD7068216952
:10D4E00020F0FE4040EA016070602078C00619D547
:10D4F000306900F03801B06A082906D0182940F0D8
:10D50000818000F0030001287CD13068C00502D57D
:10D51000E06980284AD1F068216A20F07C5040EA16
:10D520000160F0602078000744D42078800655D44C
:10D530002078400700F17E80656A9DB3306900F075
:10D540003800182840F01481012DB16A306B2DD0BD
:10D5500001F00302A36A9A4228D1C1F30511E26ADD
:10D56000914223D10146226B6FF35F21013A914230
:10D570001CD1C0F34622616B01398A4216D1C0F337
:10D580000642A16B01398A4210D1C0F30660E16BFB
:10D59000013988420AD1706BA16CC0F3CC00814282
:10D5A00040F09C81002001B0F0BD00BF012001B01F
:10D5B000F0BD00BF60690028706F4FD040F00100DF
:10D5C0007067FDF779FB0546706F8007ADD4FDF7F6
:10D5D00073FB401B0228F7D9B5E000BFA069002803
:10D5E000306871D040F480503060FDF765FB05462F
:10D5F000306880049CD4FDF75FFB401B0228F7D9FC
:10D60000A1E000BFE0690028306800F09F8040F092
:10D6100080003060FDF750FB054600BF3068C00554
:10D620003FF579AFFDF748FB401B02284FF00300A0
:10D63000F4D951E7D6F8000440F48070C6F800042D
:10D64000FDF73AFB054600BFD6F80004C00529D413
:10D65000FDF732FB401B6428F6D974E020F001008E
:10D660007067FDF729FB0546706F80077FF55DAF9A
:10D67000FDF722FB401B02284FF00300F4D92BE7F3
:10D6800021F001003060FDF717FB054630684007C8
:10D690007FF52BAFFDF710FB401B02284FF0030076
:10D6A000F4D919E7A068002800F08480052800F06C
:10D6B0009B80012800F09C80306F20F001003067D3
:10D6C000306F20F0040096E020F480503060FDF7C9
:10D6D000F3FA0546306880047FF52AAFFDF7ECFACF
:10D6E000401B02284FF00300F4D9F5E6306820F41F
:10D6F00080303060306820F480203060FDF7DCFA44
:10D70000054600BF306880037FF583AEFDF7D4FA8D
:10D71000401B64284FF00300F4D9DDE6306840F484
:10D7200080203060306840F480303060FDF7C4FA0B
:10D73000054600BF306880033FF56BAEFDF7BCFACD
:10D74000401B6428F6D9032001B0F0BD20F0800012
:10D750003060FDF7B1FA05463068C0057FF5E2AEEE
:10D76000FDF7AAFA401B02284FF00300F4D9B3E6F4
:10D77000306820F080703060FDF79EFA022D05467B
:10D780000CD100BF3068800148D5FDF795FA401BE9
:10D7900002284FF00300F5D99EE600BF30688001F3
:10D7A0007FF500AFFDF788FA401B02284FF0030019
:10D7B000F4D991E6306F20F001003067306F20F02F
:10D7C00004003067FDF778FA054641F28837306F7C
:10D7D00080077FF5B1AEFDF76FFA401BB8424FF0FE
:10D7E0000300F4D978E600BF306F40F004003067E2
:10D7F000306F40F001003067FDF75EFA054641F2F8
:10D80000883700BF306F80073FF596AEFDF754FABA
:10D81000401BB8424FF00300F4D95DE604F128073D
:10D82000B06A40F2F33188438ECF0843591E40EA74
:10D8300002104FF47E426FF35F21B06202EB47208B
:10D840004FF4FE0280B2E36B0844A16B02EB01418E
:10D850004FF0FE4201F4FE0102EB0362084402F0C5
:10D86000FE4108443063F06A4FF6F87120F0010081
:10D87000F062706BA26C884340EAC2007063F06A89
:10D88000216C20F00C000843F062F06A616C20F01B
:10D8900002000843F062F06A40F48030F062F06AFF
:10D8A00040F40030F062F06A40F48020F062F06AE8
:10D8B00040F00100F062306840F080703060FDF7A9
:10D8C000FBF90446306880013FF56CAEFDF7F4F9D2
:10D8D000001B02284FF00300F4D9FDE5F06A20F0A8
:10D8E0000100F062FDF7E8F90546FDF7E5F9A84209
:10D8F000FBD0706B4FF6F871A26C884340EAC2000F
:10D900007063F06A40F00100F062002001B0F0BDE9
:10D91000F0B581B0F8B10446D0F888001E4615462F
:10D920000F4628B9002084F88400204602F0A0FCAD
:10D930002420C4F888002068A16A0268002922F027
:10D940000101016002D0204608F0F2FD204609F0F6
:10D950008FFE012802D1012001B0F0BD206881684E
:10D9600041F480418160816821F400413943816044
:10D970003104026841EA45516FF3194211430160D5
:10D98000016841F001010160204601B0BDE8F040AE
:10D9900008F03EBE0000000043F600010068C4F23B
:10D9A0000001884208D141F22850C2F2004080694B
:10D9B000002808BF704700477047000000000000C3
:10D9C0002DE9F04381B00446066830697169D6F8E4
:10D9D000089094F8818002070CD511F4006209D0F8
:10D9E000B06940F40060B061204601B0BDE8F0438A
:10D9F00000F0E2BD01EA000505F06407042F05D13F
:10DA0000616F20468847216F2046884705F0450012
:10DA1000012807D1216F2046884705F026000228FB
:10DA200004D00BE005F02600022805D1616F2046E6
:10DA300001B0BDE8F0430847042F03D101B0BDE8B1
:10DA4000F08300BF280715D415F4587FF6D015F0E1
:10DA5000400065D1A80570D4E80505F020007CD40D
:10DA6000002840F08880D4F88400002840F093809B
:10DA7000E4E700BF2068816941F0080181618169A4
:10DA800041F010018161816941F4006181610169A6
:10DA900021F008010161806810F4404F27D0204632
:10DAA00007F0A2F9012084F88100D4F8840000284E
:10DAB00040F0AB80B8F1030F00F0AE80B8F1040F76
:10DAC00000F0B080B8F1050FB8D1204601B0BDE834
:10DAD000F04301F015B800BF2068616E006B41F89B
:10DAE000040B6166B4F86A000138A4F86A00B4F85F
:10DAF0006A000028D3D0E0681028EDD2082805D3AA
:10DB0000308E616E21F8020BEBE700BF206890F8C1
:10DB10003000616E0870606E01306066E2E700BF41
:10DB20002068D4F8841041F00401C4F8841081699D
:10DB300041F040018161A8058ED52068D4F8841099
:10DB400041F00101C4F88410816941F400718161E0
:10DB5000E80505F020007FF583AF2168D4F8842024
:10DB600042F00802C4F884208A6942F480728A6113
:10DB700000283FF478AF2068D4F8841041F0800189
:10DB8000C4F88410816941F020018161D4F88400D7
:10DB900000283FF453AF206809F4404240F26B3351
:10DBA000B2F5404F016821F001010160016921EAED
:10DBB0000301016126D1816844F6B96521F4404131
:10DBC0008160E06FC0F6010548B10565FAF728FCF1
:10DBD00028B1D4F8840040F04000C4F88400A06F5D
:10DBE00000283FF42BAF0565FAF71AFC00283FF434
:10DBF00025AFD4F8840040F04000C4F8840001B0A0
:10DC0000BDE8F083012084F88100204601B0BDE822
:10DC1000F043FFF7C1BE00BF204601B0BDE8F043AE
:10DC200000F046BF204601B0BDE8F04300F09CBCC8
:10DC30002DE9F047002858D043F600030446006859
:10DC4000C4F2000343F2000E43F6004C9842C4F2C3
:10DC5000010EC4F2000C4FF00001A16203D0604538
:10DC600018BF70453ED1E16B0122E568984202EB96
:10DC7000511105F108024FEAD20202FB01F118BF6F
:10DC8000704525D1102930D894F8811031B9002081
:10DC900084F88000204600F09FF82068022184F874
:10DCA0008110016821F0010101608168D4F81880B9
:10DCB000B8F1806F01F4F81ED4F804A020D1BAF1B5
:10DCC000000F15D0BAF5800F1AD1A36B03BB13E078
:10DCD000604518BF082908D8704518BF6045D1D0E5
:10DCE000D2E700BFE1680F29BDD90120BDE8F08768
:10DCF000A36BB3F1805F06D1036843F480530360E4
:10DD00005FEA4A2304D4D4F80C904FF0010C0FE0E2
:10DD1000D4F80C90B9F1070F08D3056825F4807C7E
:10DD2000256D45EA0C054FF0000C04E04FF0000CA7
:10DD3000056825F480750560BAF1000FE769A26AED
:10DD400047EA0E07E36B42EA0702A56842EA0302CC
:10DD50002669676942EA090282604AEA0803626B3F
:10DD6000616A42EA0302A36B41EA020141EA03014C
:10DD7000226A41EA0601E36C41EA070141EA020135
:10DD8000A26C41EA0301A36D41EA050141EA0201E7
:10DD900041EA0301C16009D18168012262F3CC210B
:10DDA00081608168022262F34A218160016DBCF1C9
:10DDB000000F21F00101016505D1C168626D21F0FC
:10DDC00000411143C1600020C4F88400012184F89F
:10DDD0008110BDE8F08700002DE9F04FB5B0044692
:10DDE00002A8B8210025CDE93355CDE9315530954C
:10DDF000F3F7C7F843F600012068C4F20001884237
:10DE000056D043F20001C4F20101884240F0DF80A5
:10DE10004FF48050029002A84FF00008CDF80C801B
:10DE2000CDF86480FEF7CCFA08B1F8F719FB44F29C
:10DE3000E04040F20044C5F60200C5F6020430ADF1
:10DE40004FF002090169032641F480510161016923
:10DE5000052701F4805101910199016841F0080101
:10DE60000160016801F0080101910199016841F028
:10DE7000020101600068294600F00200019001984B
:10DE80008020309004F50060CDE9319833963497C6
:10DE9000FCF70EFE08202946CDE9300920463497CC
:10DEA000CDE93286FCF704FE35B0BDE8F08F00BF47
:10DEB0004FF48050029002A803951995FEF780FA5E
:10DEC00008B1F8F7CDFA44F2E04040F20045C5F65B
:10DED0000200C5F6020530AE40F228088168C4F29F
:10DEE000020841F48041816081684FF0020901F429
:10DEF000804101910199016841F0040101600168CC
:10DF0000002701F0040101910199016841F002012B
:10DF100001600068314600F002000190019806207F
:10DF2000309005F58060CDF8C4904FF0030A329729
:10DF30004FF0050BCDF8CCA0CDF8D0B0FCF7B8FD74
:10DF40004FF400503146CDE9300932A880E8800C0A
:10DF50002846FCF7ADFD42F210252720C2F200450D
:10DF60004FF48066C5E901072846C5F80080EF60D8
:10DF7000C5E90467C5E90677C5E90877FAF7D0FF70
:10DF800008B1F8F76DFAE56708F11800AC6342F2E2
:10DF90008825C2F200452860282068604020C5E935
:10DFA00002072846C5E90467C5E90677C5E9087789
:10DFB000FAF7B6FF08B1F8F753FA2420052100223A
:10DFC000A567AC63FCF750FF2420FCF73DFF35B09C
:10DFD000BDE8F08F000000002DE9F04F81B09946B8
:10DFE00017460E460446D0F800A0C56BFCF764FE49
:10DFF00094F8811001290DD180460120002E18BF10
:10E00000002F03D101B0BDE8F08F00BF94F880006D
:10E01000012803D1022001B0BDE8F08FA346012002
:10E0200084F88000042084F881000020C4F8840073
:10E030004BF8646F2646A4F8687026F86A7FE0659E
:10E04000A4F86000A4F86200A168B1F5C02FC4E98B
:10E050001C00206804D1016821F40061016004E023
:10E06000C168022262F35241C16041684FF6FF72FB
:10E07000914339444160016841F0010101606168E8
:10E08000B1F5800F4FF0010103D1026842F4007234
:10E090000260E36801EB5511102B4BD33288002A44
:10E0A00000F085818DB219F1010225D041694269E4
:10E0B000D20704D1328809040CD5AA420AD2016BD6
:10E0C000DBF8000001600430CBF800003088013834
:10E0D000308006E0FCF7F0FDA0EB0800484580F03A
:10E0E000C7803088002800F0628120684169426959
:10E0F000D207DFD0E3E700BF41694269D20704D10C
:10E10000328809040ED5AA420CD2006BDBF800104D
:10E1100041F8040BCBF8001030880138308030888B
:10E1200030B944E1FCF7C8FD3088002800F03F8199
:10E130002068E1E73288072B44D9002A00F03781B4
:10E1400019F1010200F0A8808FB24FF6FF72551E40
:10E1500041694069C00716D130880A040ED5B8421B
:10E160000CD2BAF83010DBF8000020F8041BBAF823
:10E17000301020F8021C29460DE000BF30888904C9
:10E1800018D5012816D1BAF83010DBF8000020F8B5
:10E19000021B4FF6FF71CBF8000030880844308036
:10E1A0003088002800F00381206841694069C00779
:10E1B000D2D0E8E7FCF780FDA0EB08004845EFD39C
:10E1C00056E000BF002A00F0F28019F1010200F0D1
:10E1D0009F808FB24FF6FF72A2F1030A4169426934
:10E1E000D20725D132880B041CD5BA421AD290F836
:10E1F0003000616E08702068616E4A1C626690F89B
:10E20000300048702068616E4A1C626690F83000E9
:10E2100048702068616E4A1C626690F83000487051
:10E2200050460CE0328811F4C04F1BD0032A19D895
:10E2300090F83000DBF8001008704FF6FF70DBF844
:10E2400000100131CBF8001031880844308030884C
:10E25000002800F0AC80206841694269D207C1D033
:10E26000E6E700BFFCF728FDA0EB08004845EED329
:10E27000204606F0B9FDD4F8840040F48070C4F85C
:10E280008400012084F88100002084F880000320AD
:10E2900001B0BDE8F08F00BF8DB241694069C00791
:10E2A0001BD130880A0413D5A84211D2BAF8300025
:10E2B000DBF8001021F8040BBAF83000CBF800109E
:10E2C00021F8020C308802383080308898B96EE02E
:10E2D0003088890416D5012814D1BAF83000DBF84B
:10E2E000001021F8020BCBF8001030880138308084
:10E2F000308800285BD0206841694069C007D0D0D1
:10E30000EBE700BFFCF7D8FC30880028F3D14EE0E3
:10E310008FB241694269D2072ED132880B0425D5CC
:10E32000BA4223D290F83000616E08702068616EA6
:10E330004A1C626690F8300048702068616E4A1C82
:10E34000626690F8300048702068616E4A1C626610
:10E3500090F830004870606E01306066B4F86A0072
:10E360000438A4F86A003088A8B920E0328811F493
:10E37000C04F17D0032A15D890F83000DBF80010F2
:10E380000870DBF800000130CBF80000308801385D
:10E390003080308858B1206841694269D207BCD0CA
:10E3A000EAE700BFFCF788FC30880028F3D120465C
:10E3B00006F01AFD012084F88100002084F8800016
:10E3C000D4F88400002818BF012001B0BDE8F08F08
:10E3D00070B5044690F8810001280BD115460A4615
:10E3E00004F180060120002918BF002D08D100216A
:10E3F000317070BD04F1800602200021317070BDC3
:10E400003078012802D1022070BD00BF012084F8BD
:10E410008000042084F881000020C4F88400626633
:10E42000A4F86850A4F86A50C4E91C00A4F860007D
:10E43000A4F86200A068B0F5C02F21681AD108685E
:10E4400020F400600860E06810281BD2082829D357
:10E45000E06F8069B0F5005F18BFB0F5804F1DD147
:10E46000886820F480408860E06F8369B3F5804F4E
:10E4700024D02FE0C868022363F35240C860E068EC
:10E480001028E3D3E06F8069B0F5804F06D188682B
:10E4900020F480408860E06F1CE000BF0120002174
:10E4A000317070BD886820F480408860E06F8369B7
:10E4B000B3F5804F08D0B3F5005F0BD1B4F86A30E4
:10E4C00001335B0804E000BFB4F86A3003339B08F3
:10E4D000A4F86A3044F6117344F6017CC0F60103D7
:10E4E000C0F6010CC0E90F3C44F6D1633031C0F6F0
:10E4F0000103C36400230365B4F86A30FBF754F8E2
:10E5000060B1D4F8840040F01000C4F88400012009
:10E5100084F881000021317070BD00BFE16FD4E943
:10E520000002C9694FF6FF744368B1F5807F23EAA2
:10E53000040318BF2B44B2F5800F4360816841F497
:10E5400080418160016941F450710161016841F0CD
:10E550000101016003D1016841F4007101600020F4
:10E560000021317070BD000043F600010068C4F264
:10E570000001884208D141F22850C2F200404068B0
:10E58000002808BF704700477047000000000000E7
:10E5900043F600010068C4F20001884208D141F24C
:10E5A0002850C2F200400069002808BF70470047A9
:10E5B00070470000000000007047000000000000ED
:10E5C0002DE9F04381B01D4617460E460446D0F8AB
:10E5D0000090FCF771FB94F8811001290CD1804662
:10E5E0000120002E18BF002F02D101B0BDE8F0833A
:10E5F00094F88000012803D1022001B0BDE8F08327
:10E60000012184F88010032084F881000020C4F8E0
:10E610008400E665A4F86070A4F862706066A4F8EF
:10E620006800A4F86A00A2682067B2F5C02F60678E
:10E63000206805D10168034641F4006205E000BF8F
:10E64000034653F80C2F61F352421A604FF6FF72E3
:10E650004168914339444160016841F00101016022
:10E660006168B1F5800F03D1016841F40071016068
:10E67000E268102A3CD3B4F86210002900F01A8135
:10E68000691C1ED04169890706D4FCF715FBA0EB75
:10E690000800A8420AD339E1E16D51F8042B026267
:10E6A000E165B4F862000138A4F86200B4F86200D1
:10E6B000002800F0FF80206841698907E5D5EBE775
:10E6C00020684169890703D4FCF7F6FA0AE000BF25
:10E6D000E16D51F8042B0262E165B4F86200013883
:10E6E000A4F86200B4F862000028E9D1E2E000BFBB
:10E6F000B4F86210072A5DD9002900F0DB80691C9C
:10E7000031D04FF6FE714E1C4169890706D4FCF7E3
:10E71000D3FAA0EB0800A8421AD3F7E0B4F86210CD
:10E72000022909D3E16B39B1E16D51F8042B026282
:10E73000E1654FF6FE7006E0E06D30F8021BA9F8C7
:10E740002010E0653046B4F862100844A4F8620076
:10E75000B4F86200002800F0AD80206841698907A4
:10E76000DCD4D4E720684169890703D4FCF7A4FA14
:10E770001BE000BFB4F8621002290BD3E16B49B172
:10E78000E16D51F8042B0262E165B4F862000238D1
:10E7900009E000BFE06D30F8021BA9F82010E06529
:10E7A000B4F862000138A4F86200B4F862000028EE
:10E7B000D8D17FE0002900F07D80691C43D04FF65E
:10E7C000FE718E1E4F1C4169890707D4FCF774FA4D
:10E7D000A0EB0800A8422CD398E000BFB4F8621068
:10E7E000042909D3E16B402906D9E16D51F8042BC6
:10E7F0000262E165304617E0B4F8621002290BD3DB
:10E80000E16B49B1E06D30F8021BA9F82010E0651A
:10E810004FF6FE7008E000BFE16D097880F8201027
:10E82000E06D0130E0653846B4F862100844A4F8A1
:10E830006200B4F8620000283CD020684169890772
:10E84000CCD4C3E720684169890703D4FCF734FAC4
:10E850002CE000BFB4F8621004290BD3E16B41290E
:10E8600008D3E16D51F8042B0262E165B4F862004F
:10E87000043819E0B4F8621002290BD3E16B49B1F6
:10E88000E06D30F8021BA9F82010E065B4F86200D2
:10E89000023809E0E16D097880F82010E06D013060
:10E8A000E065B4F862000138A4F86200B4F86200D0
:10E8B0000028C7D1681C13D020684069000713D412
:10E8C000FCF7FAF9A0EB0800A842F5D3D4F88400CD
:10E8D00040F02000C4F8840006E000BFFCF7ECF92B
:10E8E000206840690007F9D5204606F07DFA01202E
:10E8F00084F88100002084F88000D4F88400002887
:10E9000018BF012001B0BDE8F08300BF204606F02B
:10E910006BFAD4F8840040F48070C4F884000120BD
:10E9200084F88100002084F88000032001B0BDE855
:10E93000F083000000000000F0B581B0044690F8BC
:10E94000810001280CD100294FF0010000F0AE80B9
:10E950001546002A00F0AA8094F88000012803D10F
:10E96000022001B0F0BD00BF012084F88000032226
:10E9700084F881200022C4F88420E165A4F8605066
:10E98000A4F862506266C4E91C22A4F86820A4F8C6
:10E990006A20A268B2F5C02F266813D130683246CB
:10E9A00040F400631360E268102A14D2A06F082AB2
:10E9B00082691BD3B2F5005F2AD0B2F5804F1BD01D
:10E9C0000EE000BF324652F80C3F60F35243136032
:10E9D000E268102AEAD3A06F8269B2F5804F17D09F
:10E9E000002084F88000012001B0F0BDB2F5804F16
:10E9F00008D0B2F5005F0BD1B4F8622001325208A2
:10EA000004E000BFB4F8622003329208A4F8622048
:10EA100044F6397244F60973C0F60102C0F60103E8
:10EA2000C0E90F2344F6D1620027C0F60102C26498
:10EA30000765B26822F40042B260B4F8623006F1B1
:10EA40002002FAF7B1FD68B1D4F8840040F010005C
:10EA5000C4F88400012084F8810084F8807001B03B
:10EA6000F0BD00BFA16F4FF6FF77D4E90002C9697E
:10EA70004368B1F5807F23EA070318BF2B44B2F542
:10EA8000800F4360816841F400418160016941F475
:10EA900048710161016841F00101016003D1016821
:10EAA00041F400710160002084F8800001B0F0BDE5
:10EAB00043F600010068C4F20001884208D141F227
:10EAC0002850C2F200400068002808BF7047004785
:10EAD000704700000000000043F600010068C4F227
:10EAE0000001884208D141F22850C2F20040C068BB
:10EAF000002808BF70470047704700000000000072
:10EB000043F600010068C4F20001884208D141F2D6
:10EB10002850C2F200408068002808BF70470047B4
:10EB2000704700000000000040F20442C5F60002F9
:10EB3000136823EA000008431060704700000000DB
:10EB40007047000000000000704700000000000057
:10EB50007047000000000000B0B590F83C20012A8A
:10EB600002D10220B0BD00BFD1E9022323F47C53BF
:10EB700022F4705242EA030548F2FF73D1E900CE55
:10EB8000CEF6F0730EEA030203F5006445EA020EC6
:10EB90000CEA04050C6903F5C05245EA0E05224053
:10EBA0002A434D692A4303F560550C6B03F5F04386
:10EBB0002A4023401343026840F2004C42F480652F
:10EBC000C4F2010C8C69654540F2000CCEF6FF7C66
:10EBD000CD690CEA044443EA050343EA040318D16F
:10EBE0004FF6FF7540F2000CCDF60F458C6ACDF65E
:10EBF000F04C03EA050E0D6A0CEA04544B6A44EA31
:10EC00000E0425F0085523F000532543C96A2B4311
:10EC10000B430021536480F83C100846B0BD00004F
:10EC2000B0B590F83C20012A4FF0020263D080F882
:10EC30003D2040F2004C0268C4F2010C42F48063B3
:10EC400063455368D2F808E002BF23F470034C68B0
:10EC500023434DF6FF740D68C4F2000423F07003E3
:10EC6000A24243EA0503536014DC40F2FF73C4F28E
:10EC700000039A4222DD40F60003C4F200039A42E8
:10EC80002ED040F60043C4F200039A4228D041F649
:10EC9000000321E04FF6FF73C4F200039A4213DD34
:10ECA0000023C4F201039A421AD044F20003C4F2D2
:10ECB00001039A4214D0624512D016E0B2F1804F9F
:10ECC0000ED040F2004307E04EF20003C4F200030E
:10ECD0009A4205D04EF20043C4F200039A4204D196
:10ECE0002EF080038968194391600022012180F889
:10ECF0003D1080F83C201046B0BD00000000000030
:10ED000060B310B5044690F83D0028B9002084F89F
:10ED10003C00204600F024F8022084F83D002068E2
:10ED2000211D06F0A5FE012084F8480084F83E006D
:10ED300084F83F0084F8400084F8410084F84200E1
:10ED400084F8430084F8440084F8450084F84600C1
:10ED500084F8470084F83D00002010BD0120704772
:10ED6000704700000000000090F83D10012923D1F9
:10ED7000022180F83D1001684DF6FF70C4F20000DA
:10ED80008142C86840F00100C86017DC40F2FF70A3
:10ED9000C4F20000814227DD40F60000C4F200000A
:10EDA000814233D040F60040C4F2000081422DD0B1
:10EDB00041F6000026E000BF012070474FF6FF70CB
:10EDC000C4F20000814215DD0020C4F2010081423E
:10EDD0001CD044F20000C4F20100814216D040F27F
:10EDE0000040C4F201000FE0B1F1804F0ED040F2BC
:10EDF000004007E04EF20000C4F20000814205D05E
:10EE00004EF20040C4F2000081420BD10722886814
:10EE1000C0F2010202400020062A18BFB2F5803F6E
:10EE200000D17047086840F001000860002070477A
:10EE30007047000000000000F0B581B00446006893
:10EE4000C768066906EA0705A9071BD468072FD417
:10EE5000280745D4E8065BD4E80772D117F080078D
:10EE600018BF16F402507AD1002F18BF16F4807024
:10EE700040F08280680600F18980A80600F1908049
:10EE800001B0F0BD6FF002010161012121778069BD
:10EE9000800703D02046FFF7CBFF05E0204600F0B7
:10EEA00033F9204600F01CFC002020776807CFD5FE
:10EEB00020686FF00401016102212177806910F45C
:10EEC000407F03D02046FFF7B3FF05E0204600F067
:10EED0001BF9204600F004FC002020772807B9D554
:10EEE00020686FF00801016104212177C069800763
:10EEF00004D02046FFF79CFF06E000BF204600F04C
:10EF000003F9204600F0ECFB00202077E806A3D5AB
:10EF100020686FF01001016108212177C06910F4A9
:10EF2000407F03D02046FFF783FF05E0204600F036
:10EF3000EBF8204600F0D4FB00202077E8073FF4F0
:10EF40008DAF20686FF001010161204600F028FDBF
:10EF500017F0800718BF16F402503FF485AF206801
:10EF60006FF4025101612046FFF7EEFD002F18BF3C
:10EF700016F480703FF47EAF20686FF480710161F9
:10EF80002046FFF7DDFD68067FF577AF20686FF05C
:10EF900040010161204600F00FFDA8067FF570AF2B
:10EFA00020686FF020010161204601B0BDE8F0400B
:10EFB000FFF7CEBD0000000070B586B041F2FF72D1
:10EFC0000068C4F20002002190420591CDE90311CE
:10EFD000CDE9011136DCB0F1804F5BD040F2004149
:10EFE000C4F20001884240F08D8044F2E0400024E9
:10EFF000C5F60200C5F6020402250026016841F0AC
:10F0000001010160016801F00101009100990168AE
:10F0100041F002010160006801A900F002000090C7
:10F0200000988020019020460295CDE90366059561
:10F03000FBF73EFDCDE90155CDE90366059504F5E5
:10F0400080605CE041F60001C4F2000188423BD0E0
:10F050000021C4F20101884254D144F2E040C5F6D7
:10F060000200016841F0100101600068002100F019
:10F0700010000090C5F6020100984FF4085001906E
:10F08000022002900020CDE903000120059001F547
:10F09000805034E044F2E040C5F60200016841F0DF
:10F0A00001010160006800F0010000900098052057
:10F0B0000190022002900020CDE90300012005907C
:10F0C0000020C5F602001AE044F2E040C5F6020056
:10F0D000016841F0020101600068002100F00200B7
:10F0E000009000984FF40040CDE9031100210190F9
:10F0F000C5F6020102200290059001F5806001A989
:10F10000FBF7D6FC06B070BD7047000000000000A1
:10F110002DE9F04190F83C30012B03D10220BDE8ED
:10F12000F08100BF4FEAB202052A31D8DFE812F0C1
:10F13000060038007600B400DA000001036843F6E8
:10F14000FF76C4F201061C6AB3421A6A24F0020474
:10F1500022F001021A621A46D3F804E052F818CFDE
:10F160008D6844EA0504D1F8008040F3078144F239
:10F170000007C4F20107BB4200F00B8144F6000710
:10F18000C4F20107BB4200F0048144F20047FCE0F6
:10F190000121002280F83C200846BDE8F08100BF34
:10F1A000036840F2004E43F48067C4F2010E1C6A0B
:10F1B00077451A6A24F0200422F010021A621A46D7
:10F1C0005D6852F818CF8E6844EA061407D1CE68FD
:10F1D0006FF0400724F0C00407EA0616344343F6F4
:10F1E000FF76D1F80080C4F20106B34240F3EC8010
:10F1F00044F20007C4F20107BB4200F0EC8044F681
:10F200000007C4F20107BB4200F0E58044F200476A
:10F21000C4F20107BB4200F0DE80E4E0036840F284
:10F22000004E43F48067C4F2010E1C6A77451A6AE7
:10F2300024F4007422F480721A621A465D6852F84F
:10F240001CCF8E6844EA062407D1CE6840F2FF47FF
:10F25000360224F44064BE43344343F6FF76D1F8CB
:10F260000080C4F20106B34240F3D48044F20007A8
:10F27000C4F20107BB4200F0D48044F60007C4F298
:10F280000107BB4200F0CD8044F20047C4F2010701
:10F29000BB4200F0C680CCE0036843F6FF77C4F2BF
:10F2A0000107D3F820C0BB421A6A22F480521A62C6
:10F2B0001A465C6852F81C6F0D68D1F808E040F3FC
:10F2C000CF8044F20007C4F20107BB4200F0D380B4
:10F2D00044F60007C4F20107BB4200F0CC8044F2C0
:10F2E0000047C4E0036843F6FF77C4F20107D3F890
:10F2F00020C0BB421A6A22F480321A621A465C6845
:10F3000052F8546F0D68D1F808E040F3D38044F20E
:10F310000007C4F20107BB4200F0D78044F60007A3
:10F32000C4F20107BB4200F0D08044F20047C8E0BD
:10F33000036843F6FF77C4F20107D3F820C0BB424D
:10F340001A6A22F480121A621A465C6852F8546FE4
:10F350000D68D1F808E040F3D98044F20007C4F208
:10F360000107BB4200F0DD8044F60007C4F201074C
:10F37000BB4200F0D68044F20047CEE00027C4F242
:10F380000107BB4205D040F20047C4F20107BB426F
:10F3900005D1CF6824F00C0427F004073C43B342A6
:10F3A00040F3E28044F20006C4F20106B34200F0EA
:10F3B000E68044F60006C4F20106B34200F0DF80A6
:10F3C00044F20046D7E000BF0027C4F20107BB4269
:10F3D00001D0734507D14F6925F440658E6945EA30
:10F3E000870747EA860548F6FF475D60CFF6FF6767
:10F3F00007EA0C0747EA08279F614F6809699F637E
:10F400001C629F6947F400679F619F6927F48067CA
:10F410009F61A6E00027C4F20107BB4201D07345FB
:10F4200007D14F6925F440558E6945EA071747EA29
:10F4300006154FF68C775D60CFF6FE7707EA0C076E
:10F4400047EA0807DF614F680969DF631C62DF690B
:10F4500047F00807DF61DF6927F00407DF61ACE0F0
:10F460000027C4F20107BB4205D040F20047C4F2B6
:10F470000107BB4204D14F6924F4804444EA871455
:10F4800048F6FF475C60CFF6FF673E402CF400571C
:10F4900046EA0524DC614E6809691E6447EA0E37B6
:10F4A0001F62DF6947F40067DF61DF6927F4806767
:10F4B000DF6156E00027C4F20107BB4205D040F2ED
:10F4C0000047C4F20107BB4204D14F6924F48034E1
:10F4D00044EA07244FF68C775C60CFF6FE7703375B
:10F4E0003E402CF4003746EA05045C654E68096925
:10F4F0009E6547EA0E471F625F6D47F008075F652C
:10F500005F6D27F004075F6557E000BF0027C4F276
:10F510000107BB4205D040F20047C4F20107BB42DD
:10F5200004D14F6924F4802444EA872448F6FF4735
:10F530005C60CFF6FF6707F540773E402CF400177C
:10F5400046EA05245C654E680969DE6547EA0E57A0
:10F550001F625F6D47F400675F655F6D27F480672A
:10F560005F65090229E000BF0026C4F20106B3422C
:10F5700005D040F20046C4F20106B34206D12EF493
:10F580004077D1E90565374347EA050E4FF68C759C
:10F59000C3F804E0CFF6FE750CEA050747EA080752
:10F5A0009F614F6809695F631C629F6947F00807A4
:10F5B0009F619F6927F004079F61136819431160D9
:10F5C0000021002280F83C200846BDE8F0810000C0
:10F5D00060B310B5044690F83D0028B9002084F8C7
:10F5E0003C00204600F024F8022084F83D0020680A
:10F5F000211D06F03DFA012084F8480084F83E0001
:10F6000084F83F0084F8400084F8410084F8420008
:10F6100084F8430084F8440084F8450084F84600E8
:10F6200084F8470084F83D00002010BD0120704799
:10F6300081B041F2FF710068C4F20001884217DC1A
:10F64000B0F1804F2AD040F20041C4F2000188425C
:10F6500041D144F2E840C5F60200016841F00201E0
:10F660000160006800F002000090009801B070474F
:10F6700041F60001C4F2000188421FD00021C4F20B
:10F680000101884227D144F2E840C5F602008168B2
:10F6900041F001018160806809E000BF44F2E84068
:10F6A000C5F60200016841F001010160006800F048
:10F6B00001000090009801B0704700BF44F2E8409C
:10F6C000C5F60200016841F040010160006800F0E9
:10F6D00040000090009801B070470000000000005A
:10F6E000704700000000000071B10A1F4FEAB2022B
:10F6F000032A11D8DFE802F002161E2400F13F03AE
:10F700001B78012B13D120E090F83E20012A0ED166
:10F71000022280F83E2032E000F143031B78012BE7
:10F7200005D112E000F140031B78012B0DD0012020
:10F73000704700BF00F141031B78012B05D0F6E7AD
:10F7400000F142031B78012BF1D1032A08D8DFE82E
:10F7500002F0030B0F1300BF022280F83F200EE0DF
:10F76000022280F843200AE0022280F8402006E0CE
:10F77000022280F8412002E0022280F84220026842
:10F7800001F01F00012101FA00F0116A81431162AA
:10F790004EF2FF31C4F200018A42116A40EA0100D0
:10F7A000106215DC40F6FF30C4F20000824227DC14
:10F7B000B2F1804F4ED040F20040C4F200008242CD
:10F7C00048D040F60000C4F20000824242D053E02C
:10F7D00043F6FF700021C4F20100C4F2010182422D
:10F7E00044F20000C4F201001EDC4EF20043C4F2F9
:10F7F00000039A422ED08A4224D040F200431DE0FA
:10F8000040F60040C4F20000824223D041F60000DE
:10F81000C4F2000082421DD04EF20000C4F200008B
:10F82000824217D028E000BF82420BD044F600038A
:10F83000C4F201039A4205D044F20043C4F201032A
:10F840009A4219D1536C8A4243F40041516418BF63
:10F8500082420BD107219068C0F2010101400020D3
:10F86000062918BFB1F5803F06D1704740F200402D
:10F87000C4F201008242EDD0106840F00100106037
:10F880000020704700000000026801F01F0C0123F7
:10F8900003FA0CFC136A23EA0C0343F6FF7CC4F260
:10F8A000010C13626245136A136213DD44F2000314
:10F8B000C4F201039A4218D044F60003C4F20103D3
:10F8C0009A4212D044F20043C4F201039A420CD08F
:10F8D00019E000BF0023C4F201039A4205D040F2B0
:10F8E0000043C4F201039A420DD1D2F820C041F284
:10F8F00011131CEA030F06D1D2F820C040F2444392
:10F900001CEA030F12D0D2F820C041F211131CEAF6
:10F91000030F16D1D2F820C040F244431CEA030F73
:10F920000FD1136823F0010313600AE0536C23F432
:10F9300000435364D2F820C041F211131CEA030FB4
:10F94000E8D04FEAB10104290AD8DFE801F0030F3B
:10F95000151B2100012180F83E100020704700BFD8
:10F96000012180F843100020704700BF012180F87A
:10F970003F100020704700BF012180F84010002098
:10F98000704700BF012180F841100020704700BF80
:10F99000012180F8421000207047000000000000A4
:10F9A0004EF200010068C4F20001884218BF70479F
:10F9B000FBF78AB90000000070470000000000005B
:10F9C00090F88410012901D1022070472421C0F849
:10F9D000881002681368116823F0005321F00101B8
:10F9E00011600021416613602022C0F8882080F851
:10F9F00084100846704700007047000000000000B7
:10FA0000704700000000000070B590F88420012AC3
:10FA100002D1022070BD00BF2422C0F888200268F5
:10FA2000D0F864E0BEF1000FD2F800C0136823F0F4
:10FA300001031360936823F0606341EA030191605E
:10FA40001AD091684FF6004E9368C0F6010E5B0F16
:10FA50004FF60845C1F34266C0F601051EF80340A3
:10FA6000E95C2301B3FBF1F11EF80630AE5D1B012A
:10FA7000B3FBF6F302E000BF01210123A0F86A10F6
:10FA80002021A0F86830C2F800C0C0F8881000211A
:10FA900080F88410084670BD70B590F88420012A63
:10FAA00002D1022070BD00BF2422C0F88820026865
:10FAB000D0F864E0BEF1000FD2F800C0136823F064
:10FAC00001031360936823F0604341EA03019160EE
:10FAD0001AD091684FF6004E9368C0F6010E5B0F86
:10FAE0004FF60845C1F34266C0F601051EF8034013
:10FAF000E95C2301B3FBF1F11EF80630AE5D1B019A
:10FB0000B3FBF6F302E000BF01210123A0F86A1065
:10FB10002021A0F86830C2F800C0C0F88810002189
:10FB200080F88410084670BD704700000000000097
:10FB3000704700000000000045F200010068C4F2B8
:10FB40000001032301F54042904208BF0123401AFF
:10FB500018BF1846032808BF704700EBC00041F2E9
:10FB60004851C2F2004101EB8000006900B100473A
:10FB70007047000000000000B0B50446006840F681
:10FB80002F01C26905681140D0F808E020290BD187
:10FB900005F020010EF08053C91823D0616FD1B356
:10FBA0002046BDE8B040084740F60F010A4219D090
:10FBB000012140F22013C1F20001C0F200430EEA1D
:10FBC000010C05EA030111EB0C010BD0D10718BFA2
:10FBD00015F4807140F0C68191070EF0010300F129
:10FBE000CD81D4E105EA0203D906E16E14D50129DD
:10FBF00012D1102101628168490600F19D80B4F89C
:10FC00005C10B4F85E20B4F85E30002B1CBF891A7B
:10FC10005FEA01422FD1B0BDD10240F159811EF4FB
:10FC2000800100F055814FF4801101622046BDE84B
:10FC3000B040FFF77DBF00BF206850E8000F22688A
:10FC400020F4907042E80003002B1FBF206850E8AA
:10FC5000000F226820F490701CBF42E80003002BC4
:10FC600012D0206850E8000F226820F4907042E81B
:10FC700000034BB1206850E8000F226820F4907018
:10FC800042E80003002BD7D14FF6FE70CEF6FF708E
:10FC9000226852E8022F2368024043E80225002D23
:10FCA0001FBF226852E8022F236802401CBF43E8AE
:10FCB0000225002D10D0226852E8022F236802404E
:10FCC00043E8022545B1226852E8022F236802402A
:10FCD00043E80225002DDBD12020C4F88C00002051
:10FCE000E0666067206850E8000F226820F010008E
:10FCF00042E80003002B1FBF206850E8000F226875
:10FD000020F010001CBF42E80003002B12D0206836
:10FD100050E8000F226820F0100042E800034BB1C9
:10FD2000206850E8000F226820F0100042E800032D
:10FD3000002BD7D189B227E2D4F8803019684A68FD
:10FD4000B4F85CC091B2002900F01682614580F0E1
:10FD50001382A4F85E20D969B1F5807F00F0AC80F1
:10FD600050E8000F216820F4807041E80002FAB1E9
:10FD7000206850E8000F216820F4807041E80002FC
:10FD8000002A1FBF206850E8000F216820F480700F
:10FD90001CBF41E80002002A0AD0206850E8000F8A
:10FDA000216820F4807041E800020AB12068D7E79A
:10FDB000206850E8020F216820F0010041E80202AB
:10FDC000002A1FBF206850E8020F216820F00100C0
:10FDD0001CBF41E80202002A26D0206850E8020F2A
:10FDE000216820F0010041E80202EAB1206850E8F1
:10FDF000020F216820F0010041E80202002AD7D159
:10FE000012E000BF206850E8020F216820F0400097
:10FE100041E80202EAB1206850E8020F216820F0B0
:10FE2000400041E80202A2B1206850E8020F2168B8
:10FE300020F0400041E80202002A1FBF206850E87D
:10FE4000020F216820F040001CBF41E80202002A96
:10FE5000D8D12020C4F88C000020E066206850E84B
:10FE6000000F216820F0100041E80002002A1FBFA7
:10FE7000206850E8000F216820F010001CBF41E806
:10FE80000002002A12D0206850E8000F216820F0FC
:10FE9000100041E800024AB1206850E8000F2168D4
:10FEA00020F0100041E80002002AD7D1D4F88000E9
:10FEB000F8F71AF8B4F85CC002202067B4F85E00C6
:10FEC000ACEB000081B22046BDE8B040FFF794BD26
:10FED00011060BD505F0800C0EF4000111EB0C019E
:10FEE00004D0A16F00297FF45BAE94E659060BD4D1
:10FEF000100240F17D8115F0804000F079812046AC
:10FF0000BDE8B040FFF710BE50E8000F216820F0B8
:10FF1000400041E80002002A00F04681206850E8D5
:10FF2000000F216820F0400041E80002002A1FBFB6
:10FF3000206850E8000F216820F040001CBF41E815
:10FF40000002002A00F03081206850E8000F21688C
:10FF500020F0400041E80002002A00F025812068DE
:10FF6000D2E700BF01210162D4F8901041F00101F5
:10FF7000C4F8901091070EF0010308D53BB102219F
:10FF80000162D4F8901041F00401C4F890105107B8
:10FF900008D53BB104210162D4F8901041F0020170
:10FFA000C4F8901011070CD505F0200151EA0C019E
:10FFB00007D008210162D4F8901041F00801C4F87C
:10FFC000901011050BD515F0806108D04FF4006139
:10FFD0000162D4F8901041F02001C4F89010D4F8D8
:10FFE000901000293FF417AE12F020010AD005F05E
:10FFF00020010EF08052891804D0616F11B12046A3
:020000040801F1
:1000000088472068D4F89010826802F0400201F01E
:100010002801891800F0C08050E8000F216820F402
:10002000907041E80002FAB1206850E8000F2168A2
:1000300020F4907041E80002002A1FBF206850E8B9
:10004000000F216820F490701CBF41E80002002AD4
:100050000AD0206850E8000F216820F4907041E831
:1000600000020AB12068D7E74FF6FE70CEF6FF70A7
:10007000216851E8021F2268014042E80213002B68
:100080001FBF216851E8021F226801401CBF42E8DF
:100090000213002B10D0216851E8021F2268014092
:1000A00042E8021343B1216851E8021F226801406F
:1000B00042E80213002BDBD1E06E012828D100BFFB
:1000C000206850E8000F216820F0100041E800028D
:1000D000002A1FBF206850E8000F216820F01000A0
:1000E0001CBF41E80002002A12D0206850E8000F2F
:1000F000216820F0100041E800024AB1206850E871
:10010000000F216820F0100041E80002002AD7D13A
:100110002020C4F88C000021E166206861678168B6
:1001200049065FD550E8020F216820F0400041E801
:100130000202002A42D0206850E8020F216820F015
:10014000400041E80202002A1FBF206850E8020F69
:10015000216820F040001CBF41E80202002A2DD097
:10016000206850E8020F216820F0400041E80202B8
:1001700022B32068D6E700BF8C457FF44CADD86928
:10018000B0F5807F7FF447AD022020672046BDE8B0
:10019000B040FFF731BC00BF2046FFF7CDFC002088
:1001A000C4F89000B0BD00BF2020C4F88800002033
:1001B000A0672046BDE8B04000F00ABDD4F880003A
:1001C00080B146F28971C0F601010165F8F728F99E
:1001D00000283FF420ADD4F88000016DBDE8B040A8
:1001E000084700BF2046BDE8B040FFF7A5BC00BFF0
:1001F000D0017FF510ADB5F1FF3FC8BFB0BD2046BF
:10020000BDE8B040FFF7FCBB10B5E0B10446D0F844
:10021000880028B9002084F88400204600F028F8DF
:100220002420C4F888002068A16A0268002922F00E
:100230000101016002D0204606F07AF9204607F05D
:1002400017FA012802D1012010BD00BF20684168C3
:1002500021F490414160816821F02A0181600168A8
:1002600041F0010101602046BDE8104006F0D0B920
:100270002DE9F043B5B000210446CDE93311CDE9B5
:100280003111309102A8B821F0F77BFE47F2FF71DF
:100290002068C4F20001884200F3808044F20041EB
:1002A000C4F20001884200F0CF8044F60001C4F29D
:1002B0000001884200F0FA8045F20001C4F200011A
:1002C000884240F0EA8102A8002703974FF0020815
:1002D000CDF808801F97FCF773F808B1F6F7C0F85F
:1002E00044F2E04040F60045C5F60200C5F60205BE
:1002F00030AE4FF00809816841F480118160816857
:1003000001F4801101910199016841F0040101603B
:10031000016801F0040101910199016841F00801AF
:1003200001600068314600F00800019001984FF428
:100330008050CDE93008A5F58060CDF8D090CDE9AA
:100340003277FAF7B5FB04203146CDE9300828466C
:10035000CDF8D090CDE93277FAF7AAFB42F200351A
:100360005820C2F20045C4F2020028604120C5E9CD
:1003700001074FF48060EF60C5E904072846C5E92E
:100380000677C5E90877F8F7CBFD08B1F6F768F806
:10039000C4F88050AC63352477E100BF47F6000114
:1003A000C4F20001884200F0CD8041F20001C4F2A5
:1003B0000101884200F0FA8041F60041C4F20101D7
:1003C000884240F06A810120029002A8002603962C
:1003D0002096FBF7F5FF08B1F6F742F844F2E0404B
:1003E00030ADC5F602000227016941F080010161CC
:1003F000016901F0800101910199016841F010014A
:1004000001600068294600F0100001900198042066
:100410003090349040F60040C5F60200339600F567
:1004200080642046CDE93176FAF742FB0820294660
:10043000CDE930070B2034902046CDE93266FAF73B
:1004400037FB9C2421E100BF02A80024039402256D
:1004500002951F94FBF7B4FF08B1F6F701F844F2D8
:10046000E040C5F60200816841F400318160816896
:1004700001F4003101910199016841F00801016026
:10048000006830A900F00800019001987020CDE9C3
:1004900030050720349040F60040C5F60200CDE953
:1004A0003244FAF705FB2624EFE000BF02A800263D
:1004B00003964FF00208CDF808801F96FBF780FFE7
:1004C00008B1F5F7CDFF44F2E04040F60044C5F630
:1004D0000200C5F6020430AD0727816841F480218F
:1004E0008160816801F4802101910199016841F0E6
:1004F00002010160016801F00201019101990168A6
:1005000041F0080101600068294600F008000190F0
:1005100001984FF48040CDE93008A4F5006034978D
:10052000CDE93266FAF7C4FA4FF440702946CDE9B6
:10053000300820463497CDE93266FAF7B9FA272415
:10054000A3E000BF02A800240394022502951F9493
:10055000FBF736FF08B1F5F783FF44F2E040C5F63C
:100560000200816841F080418160816801F0804132
:1005700001910199016841F010010160006840F6A5
:10058000004100F010000190C5F6020101984FF4FF
:10059000C070CDE930050720349001F5806030A9A6
:1005A000CDE93244FAF784FA52246EE00120029039
:1005B00002A8002603962096FBF702FF08B1F5F784
:1005C0004FFF44F2E04040F25808C5F60200C4F282
:1005D0000208016941F010010161016901F0100197
:1005E00001910199016841F001010160006840F644
:1005F000004100F001000190C5F6020101984FF49E
:10060000C060309002203396CDE931060720349047
:10061000A1F5406030A9FAF74BFA42F2F03508F143
:100620001800C2F200454FF4806728602A206860F5
:100630004020C5E902062846C5E90476C5E90666F4
:10064000C5E90866F8F76CFC08B1F5F709FFE5673E
:1006500008F13000AC6342F27835C2F20045286000
:10066000292068600020C5E90200C5E90470C5E9D9
:100670000600C5E908002846F8F752FC08B1F5F76E
:10068000EFFEC4F88050AC632524052100222046EB
:10069000FAF7EAFB2046FAF7D7FB35B0BDE8F0835E
:1006A000B0B50446D0F88C00202807D115460A467C
:1006B0000120002918BF002D02D1B0BD0220B0BD1D
:1006C0004FF0000CC4F86CC040F600402168C5F63D
:1006D0000000814234D04868000231D551E8000F53
:1006E000D4F800E040F080604EE8000141B300BF64
:1006F000206850E8000F216840F0806041E8000366
:10070000002B1FBF206850E8000F216840F0806078
:100710001CBF41E80003002B12D0206850E8000FF6
:10072000216840F0806041E800034BB1206850E848
:10073000000F216840F0806041E80003002BD7D112
:10074000A2652220A4F85C50C4F890C0C4F88C00C4
:10075000D4F88000F0B146F6B11146F63133C0F658
:100760000101C0F60103C0E90F1346F2997100239D
:10077000C0F60101C1642168036524312B46F8F7F6
:1007800013FF38B11020C4F890002020C4F88C006A
:100790000120B0BD206938B3206850E8000F2168FF
:1007A00040F4807041E80002002A1FBF206850E832
:1007B000000F216840F480701CBF41E80002002A4D
:1007C00012D0206850E8000F216840F4807041E8A2
:1007D00000024AB1206850E8000F216840F48070A0
:1007E00041E80002002AD7D1206850E8020F2168B2
:1007F00040F0010041E80202002A1FBF206850E8D3
:10080000020F216840F001001CBF41E80202002AEB
:100810001DD0206850E8020F216840F0010041E837
:100820000202A2B1206850E8020F216840F00100E6
:1008300041E80202002AD7D109E000BF206850E851
:10084000020F216840F0400041E80202EAB120684E
:1008500050E8020F216840F0400041E80202A2B1D6
:10086000206850E8020F216840F0400041E8020291
:10087000002A1FBF206850E8020F216840F04000A6
:100880001CBF41E80202002AD8D10020B0BD000000
:1008900080B5D0F88C30202B06D10123002918BF59
:1008A000002A03D1184680BD022080BD0023C36604
:1008B00040F60043D0F800C0C5F600039C4503D0C5
:1008C000DCF804301B0205D407F0F2F900231846C7
:1008D00080BD00BF5CE800CFD0F800E04CF0806342
:1008E0004EE8003CBCF1000FEED0036853E800CFA7
:1008F000D0F800E04CF080634EE8003CBCF1000F03
:100900001FBF036853E800CFD0F800E04CF08063CD
:100910001CBF4EE8003CBCF1000FD5D0036853E883
:1009200000CFD0F800E04CF080634EE8003CBCF112
:10093000000FC9D0036853E800CFCDE700000000E6
:1009400045F200010068C4F20001032301F54042B2
:10095000904208BF0123401A18BF1846032808BF59
:10096000704700EBC00041F24851C2F2004101EB78
:100970008000C06800B10047704700000000000020
:1009800045F200010068C4F20001032301F5404272
:10099000904208BF0123401A18BF1846032808BF19
:1009A000704700EBC00041F24851C2F2004101EB38
:1009B0008000806800B10047704700000000000020
:1009C000B0B50446D0F88800202831D100294FF076
:1009D000010061D0002A134608BFB0BD2165002583
:1009E000A4F854302120A4F85630C4F89050C4F82C
:1009F0008800E06FF0B146F2997246F6513CC0F6BD
:100A00000102C264226846F6114E2832C0F6010C7B
:100A1000C0F6010E0565C0E90FCEF8F7C5FD48B177
:100A20001020C4F890002020C4F888000120B0BD38
:100A30000220B0BD20684021016250E8020F216809
:100A400040F0800041E8020242B300BF206850E855
:100A5000020F216840F0800041E80202F2B12068F4
:100A600050E8020F216840F0800041E80202AAB17C
:100A7000206850E8020F216840F0800041E802023F
:100A800062B1206850E8020F216840F0800041E820
:100A900002020020002AD9D1B0BD00BF0020B0BDA5
:100AA000D0F88830202B07D10123002918BF002A55
:100AB00004D11846704700BF02207047016500212D
:100AC000A0F85420A0F85620C0F890102121C0F8BA
:100AD0008810416EB1F1005F816835D1B1F5805F5A
:100AE00002D10169002963D048F2B911C0F60101B1
:100AF0008167016851E8021F026841F4000142E881
:100B00000213002B52D0016851E8021F026841F421
:100B1000000142E80213002B1FBF016851E8021FC9
:100B2000026841F400011CBF42E80213002B3DD0D3
:100B3000016851E8021F026841F4000142E8021313
:100B4000002BD6D132E000BFB1F5805F01D1016941
:100B5000A1B348F2E901C0F601018167016851E8DB
:100B6000001F026841F0800142E8001363B301688E
:100B700051E8001F026841F0800142E80013002B99
:100B80001FBF016851E8001F026841F080011CBFCF
:100B900042E80013002B09D0016851E8001F0268E9
:100BA00041F0800142E80013002BD7D100207047AC
:100BB00047F6F971C0F601019AE700BF47F62971BF
:100BC000C0F60101C9E700BF0023184670470000C6
:100BD00045F200010068C4F20001032301F5404220
:100BE000904208BF0123401A18BF1846032808BFC7
:100BF000704700EBC00041F24851C2F2004101EBE6
:100C00008000406800B1004770470000000000000D
:100C100045F200010068C4F20001032301F54042DF
:100C2000904208BF0123401A18BF1846032808BF86
:100C3000704741F2485100EBC000C2F2004151F848
:100C4000200008B1004700BF70470000000000000E
:100C5000FEE700000000000010EE100AB6EE001AD9
:100C600045F6DF11B7EE083AC5F6377120EE010AF6
:100C7000A1EB6000B0EE434A01EE100A20EE012A1B
:100C800002EE414A24EE011A20EE010A01EE403A3A
:100C900021EE030A704700002DE9F04381B048B10E
:100CA000044690F82A0058B1002040B201B0BDE8D7
:100CB000F08300BFFF2040B201B0BDE8F08300BF69
:100CC00004F1780704F180093846494608F04AFEE5
:100CD000264684F8C800B4F8780004F1580826F8CD
:100CE000A80FB4F85A00A4F8AA0038464146324684
:100CF00008F040FD274684F8C8003088494627F8A8
:100D0000B00FB4F88200A4F8B20030463A4608F0BA
:100D100031FD2146254684F8C800384651F8902F09
:100D200045F8A02F2A4608F05BFB84F8C800284647
:100D3000394608F0B9FB84F8C800B4F85800308090
:100D4000B4F88200A4F8AA0040464946324608F0AA
:100D500011FD84F8C800A5F108023046394608F0B4
:100D600009FD84F8C800002040B201B0BDE8F0835E
:100D7000002800F095812DE9F04F83B004460173FF
:100D800042739A468373002020741846154688469D
:100D9000EFF75CFB51466061F0F7D1F84FEA8A0B40
:100DA0005846EFF753FB5946A061F0F7EAF858466A
:100DB000EFF74CFB5946E061F0F7E3F84FEA88099A
:100DC0004846EFF743FB49462062F0F7DAF8504611
:100DD000EFF73CFB51466062F0F7B1F84846EFF799
:100DE00035FB49462060F0F7CCF85846EFF72EFB6C
:100DF00059466060F0F7C5F8AE003046EFF726FBC5
:100E00003146A060F0F7BDF84846EFF71FFB4946B2
:100E10000746C4F8E800F0F7B4F804F13000012206
:100E200041463B4608F03BFB4846EFF70FFB49467F
:100E30000746C4F8EC00F0F7A4F8217B04F1380071
:100E400001223B4608F02BFB01957DB13046EFF7C0
:100E5000FDFA31460746C4F8F000F0F792F8617BDE
:100E600004F1400001223B4608F019FB5846EFF719
:100E7000EDFA59460646C4F8F400F0F782F8A17B73
:100E800004F148000122334608F009FB09FB08F68B
:100E9000CDF808803046EFF7D9FA31460746C4F856
:100EA000F800F0F76EF8217B04F150003B460A464B
:100EB00008F0F5FA3046EFF7C9FA31460746C4F8AC
:100EC000FC00F0F75EF8217B04F158003B460A462F
:100ED00008F0E5FA3046EFF7B9FA0746C4F8000122
:100EE0003046EFF7B3FA8046C4F80401384631467D
:100EF000F0F747F840463146F0F743F8217B04F11C
:100F000060003B460A4608F0CAFA217B04F16800FB
:100F1000D4F804310A4608F0C2FA019888B109FBF6
:100F200000F73846EFF792FA39460546C4F808014B
:100F3000F0F727F8217B04F17000627B2B4608F064
:100F4000AEFA02980BFB00F52846EFF77FFA09FB93
:100F50000AF80746C4F80C014046EFF777FACDF8D7
:100F600008A08246C4F8100138462946F0F709F86F
:100F700050464146F0F705F8227B04F17800A17B4A
:100F80003B4608F08CFA217B04F18000A27BD4F868
:100F9000103108F084FA3046EFF758FA314605462A
:100FA000C4F81401EFF7EDFF217B04F188002B4614
:100FB0000A4608F074FA02980BFB00F52846EFF792
:100FC00045FA29460746C4F81801EFF7DAFFA17B76
:100FD00004F190003B460A4608F061FA4046EFF7FC
:100FE00035FA41460546C4F81C01EFF7CAFF217BDC
:100FF00004F19800A27B2B4608F051FA3046EFF737
:1010000025FA0546C4F820013046EFF71FFAC4F868
:1010100024013046EFF71AFAC4F828014846EFF7E2
:1010200015FAC4F82C014846EFF710FA217BC4F8F2
:10103000300104F1A0002B460A4608F030FA217B6B
:1010400004F1A800D4F824310A4608F028FA217BDC
:1010500004F1B000D4F828310A4608F020FA217BC8
:1010600004F1B800D4F82C31012208F018FA217BE1
:1010700004F1C000D4F83031012208F010FA002049
:1010800084F82C00A062C4E93300C4E93500C4E947
:101090003700C4F8E40003B0BDE8F04F40B2704739
:1010A000FF2040B270470000002800F08B8070B530
:1010B0000646C07B002800F08980B27B0020307497
:1010C000D6F8F40071689200EFF7F7FEB17B706814
:1010D0008900EFF756FFB07B00FB00F1D6F818014E
:1010E0008900EFF74EFF307BB17B4143D6F80C010E
:1010F0008900EFF746FF96F80EC0BCF1000F2BD029
:101100000020002104E000BF01310430614523D2FA
:10111000D6F8F4301A1892ED000AB5EE400AF1EE56
:1011200010FAF1D0327C746A03EB820383ED000A7B
:10113000A1547269347C337BB569525C96F80EC059
:1011400014FB0322D6F80C3103EB82022B5842F831
:10115000043C621C3274D7E796F810C0BCF1000F53
:101160001BD0716AD6F81801D6F81CE0BCF1010F4B
:101170000A785EF8222002600FD00423CCF100022E
:1011800003EB8C03013918448C78013201315EF88D
:1011900024400460541C1844F6D1307BA6F878C073
:1011A000A6F87A00A6F88000A6F882C0A6F890C03B
:1011B000A6F892C0A6F89800A6F89AC0A6F848C06B
:1011C00010E000BFFF2040B2704700BFB27BD6F8EE
:1011D000F40071689200EFF770FEB17B70688900CF
:1011E000EFF7CFFE727BD6F8F000B1689200EFF710
:1011F00064FE0020BDE8704040B27047000000006F
:10120000002808BF704710B5017B0446D0F8E800FD
:101210008900EFF7B6FE217BD4F8EC008900EFF7E8
:10122000B0FE217B20688900EFF7ABFE0020207420
:10123000BDE8104070470000002800F01D812DE936
:10124000F04381B00446FFF72FFFD4F8CC1009B16A
:101250002046884794F8280030BB607B002800F0C7
:1012600025812546207B04F13001012725F8B80FA0
:1012700004F160002A46A4F8BA7008F07BFA26460A
:10128000217B26F8C01FA6F180013072A6F1500024
:101290003246778008F06EFA3072A6F1880228464E
:1012A000314608F09DF83072D4F8D01009B12046CC
:1012B000884794F8290050BB04F1600504F16806E2
:1012C0002846314608F04EFB04F1580784F8C80060
:1012D00004F1500128463A4608F04CFA2546B4F885
:1012E000581084F8C80025F8A81F314635F83E0C80
:1012F0002A466880384608F03DFA84F8C800A5F10F
:10130000200128463A4608F06BF884F8C800D4F863
:10131000D41009B120468847207C002800F0AE8018
:101320002046FFF7B9FCD4F8D81009B12046884709
:1013300094F82B00A0BB2046254604F138084FF056
:10134000010930F8781FA4F8BA9025F8B81F414673
:101350002A4608F00FFA84F8C80020462746A4F869
:10136000C29030F8481F27F8C01F29463A4608F0B7
:1013700099FA264684F8C80039462A4636F8980F66
:10138000A4F8BA902880304608F0F4F984F8C80030
:10139000A6F168024046294608F022F884F8C80001
:1013A000D4F8DC1009B12046884794F82C0030BBF3
:1013B0002046254630F8982F25F8A82F2E4635F8D8
:1013C0002E3CA5F1300126F8082F35F84E2C6A8105
:1013D0002A466B80A5F1500708F0CCF985F820006B
:1013E00028463946324608F0C5F985F82000A5F1AF
:1013F00058023846314608F055FA85F82000D4F8EE
:10140000E01009B120468847227B32B3236AD4F822
:10141000F81093ED000A91ED001AB4EE401AF1EEC7
:1014200010FAB8BF81ED000A012A16D00420043357
:1014300000EB82000127014491ED001A93ED000AB0
:101440000137B4EE401AF1EE10FAB8BF81ED000A90
:10145000BA42014403F10403EED120689200D4F8AB
:10146000E810EFF72AFDD4F8E41009B120468847C8
:10147000206801B0BDE8F08300207047E07B0028C1
:101480003FF44EAF227BD4E93A019200EFF715FD0D
:10149000207B00FB00F2D4E93E019200EFF70DFD46
:1014A000D4F8E0100029ADD1AEE700BF04F1600030
:1014B00004F1300104F1380208F05CF984F8C80046
:1014C000D4F8D01000297FF4F2AEF2E6000000005C
:1014D000002800F0ED800168002900F0E9809FED10
:1014E000761A80FE410A9FED751A80FE010A80ED92
:1014F000150A91ED013A91ED004A20EE002A20EE06
:10150000021A22EE033A01EE043A91ED024A00EE8D
:10151000043A91ED034A34EE033A80ED163A91ED28
:10152000053A91ED044A22EE033A01EE043A91EDB8
:10153000064A00EE043A91ED074A34EE033A80ED94
:10154000173A91ED093A91ED084A22EE033A01EE7D
:10155000043A91ED0A4A00EE043A91ED0B4A34EE5A
:10156000033A80ED183A91ED0D3A91ED0C4A22EED6
:10157000033A01EE043A91ED0E4A00EE043A91ED81
:101580000F4A34EE033A80ED193A91ED113A91ED9C
:10159000104A22EE033A01EE043A91ED124A00EEAF
:1015A000043A91ED134A34EE033A80ED1A3A91ED84
:1015B000153A91ED144A22EE033A01EE043A91ED08
:1015C000164A00EE043A91ED174A34EE033A80EDE4
:1015D0001B3A91ED193A91ED184A22EE033A01EEC9
:1015E000043A91ED1A4A00EE043A91ED1B4A34EEAA
:1015F000033A80ED1C3A91ED1D3A91ED1C4A22EE22
:10160000033A01EE043A91ED1E4A00EE043A91EDE0
:101610001F4A34EE033A80ED1D3A91ED213A91EDE7
:10162000204A22EE033A01EE043A91ED224A00EEFE
:10163000043A91ED234A34EE033A80ED1E3A91EDDF
:10164000253A91ED244A22EE033A01EE043A91ED57
:10165000264A00EE043A91ED274A34EE033A80ED33
:101660001F3A91ED293A91ED284A22EE033A01EE14
:10167000043A91ED2A4A00EE043A91ED2B4A34EEF9
:10168000033A80ED203A91ED2D3A22EE032A91EDB6
:101690002C3A01EE032A91ED2E1A00EE012A91ED6B
:1016A0002F0A30EE020A80ED210A002040B2704776
:1016B000FF2040B2704700BFCDCCCC3ECDCCCC3D5E
:1016C00000284BD090F88810002947D090ED170AD9
:1016D00090ED0E1A90ED1D2A20EE010A21EE021A5D
:1016E00090ED162A90ED0D3A90ED1C4A02EE030A99
:1016F00090ED182A03EE041A90ED0F3A02EE030A59
:1017000090ED1E2A03EE021A90ED192A90ED103A80
:1017100002EE030A90ED1F2A03EE021A90ED1A2A38
:1017200090ED113A02EE030A90ED202A03EE021A20
:1017300090ED1B2A90ED123A02EE030A90ED212A59
:1017400003EE021AB1EE400A80ED130AB1EE410A2F
:1017500080ED140A002040B2704700BFFF2040B265
:101760007047000000000000B0B5044600284FF0AC
:10177000FF0012D00D4681B1201D8821EFF701FC3A
:10178000B5EE000A4FF07A50606520462560FFF7FD
:101790009FFE012084F88800002040B2B0BD000008
:1017A00050B180B504305021EFF7EBFB0020BDE8CD
:1017B000804040B2704700BFFF2040B27047000039
:1017C000FF22002818BF002902D150B2704700BF85
:1017D00010B591E80C50D1E90441C26190ED010AC5
:1017E000036290ED021AC0F824C090ED032AC0F8FD
:1017F00028E090ED043AC0E90B4190ED076A90EDC6
:10180000087A30EE460A90ED096A31EE471A90EDFB
:101810000A7A90ED054A90ED065AD0ED0B0AD0ED0C
:101820000C1A80ED0D0A32EE460A80ED0E1A33EEE8
:10183000471A80ED0F0A34EE600A80ED101A35EE7B
:10184000611A002280ED110A80ED121ABDE81040E5
:1018500050B2704700000000FF22002818BF002986
:1018600002D150B2704700BF10B591E80C50D1E9D9
:101870000441426090ED076A836090ED087AC0F8F9
:101880000CC0D0ED0B0AC0F810E0D0ED0C1AC0E986
:10189000054190ED010A90ED021A90ED032A90EDBA
:1018A000043A30EE460A90ED096A31EE471A90ED9F
:1018B0000A7A90ED054A90ED065A80ED0D0A32EE57
:1018C000460A80ED0E1A33EE471A80ED0F0A34EE09
:1018D000600A80ED101A35EE611A002280ED110ABF
:1018E00080ED121ABDE8104050B2704700000000B1
:1018F00030B3B0EE403A90ED011A90ED062A90ED2B
:10190000074A80ED072A02EE413A90ED021A04EEF2
:10191000413A13EE101A21F00041B1F1FF4F00FEE1
:10192000031A90ED030A90ED043A80ED061A20EEBA
:10193000010A02EE030A90ED053A04EE030A70472D
:101940009FED010A704700BF00000000000000008A
:10195000002808BF704710B50446F5EE400AC0EDF8
:10196000000A0020F1EE10FAA061E06132DD80EEA5
:10197000200A9FED201A81EE000A0DF07BFB9FEDFF
:101980001E1AB7EE002A20EE011A20EE004A31EEB0
:10199000023A32EE410ABFEE002A34EE031A34EE68
:1019A000022A34EE000A84EE013A32EE022A84ED75
:1019B000033A80EE010A84ED053A33EE034A82EEE3
:1019C000011A84ED044A84ED011A84ED020ABDE88F
:1019D000104070474FF07E516061C4E903106060B1
:1019E0009FED030A84ED020ABDE81040704700BF76
:1019F00000000000DB0F4940F304B53F0000000089
:101A000080B390ED031A90ED042A31EE023A90ED86
:101A1000054AB0EE406A90ED015A33EE043A80EE8A
:101A2000033A13EE101A01F0FF41B1F1FF4F00FE2F
:101A3000033A80ED073A03EE456A90ED025A03EE51
:101A4000456A16EE101A21F00041B1F1FF4F00FE79
:101A5000065A80ED065A21EE050A02EE030A04EE4C
:101A6000030A70479FED010A704700BF00000000A5
:101A700010B592B0002841D090F800C0BCF1020F20
:101A800038D841F29051C2F2004151F82C1089B37C
:101A900091F8842072B30B1D04E000BF013A03F1FA
:101AA000040327D0D3F800E0BEF1000FF6D09EF873
:101AB00000106145F2D1BEF802104488A142EDD178
:101AC000BEF804006946009008208DF804004FF02D
:101AD000FF30CDF805000290FC208DF80C009EF838
:101AE0000000F1F771FE002818BF4FF0FF3040B240
:101AF00012B010BDFC2040B212B010BDFE2040B2AA
:101B000012B010BD00000000B0B518B390F800C0CE
:101B1000BCF1020F1ED841F29051C2F2004151F8BF
:101B20002C10B9B191F88430A3B101F1040E002258
:101B300003E000BF01329A420ED25EF82210002963
:101B4000F8D00C786445F5D14C884588AC42F1D189
:101B50000846B0BD0020B0BD00210846B0BD000061
:101B6000B0B592B0FE22002818BF002902D150B2B1
:101B700012B0B0BD90F800C0BCF1020F00F29C8022
:101B800041F29052C2F2004252F82C20002A00F09A
:101B9000938092F88430002B00F08E80043204E0B1
:101BA000013B02F1040200F08780D2F800E0BEF1B0
:101BB000000FF5D09EF800406445F1D1BEF8024018
:101BC0004588AC42ECD1B3EE0E2A91ED020A9FEDAE
:101BD0003C1AB2EE084A30EE010A91ED011A31EEDC
:101BE000021A9FED383A9FED392A91ED035A20EE03
:101BF000030A9FED353A21EE021A91ED046A25EEB3
